:020000040800F2
:10000000F0FF00102DF30608596B06086104020882
:10001000CDF30608CDF30608CDF306080000000076
:100020000000000000000000000000005D6B0608FA
:10003000616B060800000000656B060879A40008E3
:10004000CDF30608CDF30608CDF30608CDF3060878
:10005000CDF30608CDF3060859BD00087DBD0008A4
:10006000A1BD0008C5BD0008E9BD0008E9B700084A
:10007000FDB7000811B8000825B8000839B8000815
:100080004DB8000861B80008CDF30608CDF30608A6
:10009000CDF30608CDF30608CDF306080DBE000823
:1000A00009D1000869D0000819D1000859D000080A
:1000B00091D00008A1D00008B1D00008FDB100081F
:1000C000A9C7000805B20008ADC70008CDF30608AF
:1000D000CDF30608893A0608893B0608AD3C0608B8
:1000E00049BE0008CDF3060871C0060829D10008F2
:1000F000E1D0000839D10008D1D0000875B8000857
:10010000CDF30608CDF30608C1D00008CDF30608EC
:10011000D13D0608F53E0608CDF30608CDF30608E6
:1001200089B800089DB80008B1B80008C5B8000833
:10013000D9B80008CDF30608CDF30608CDF30608BC
:10014000CDF30608CDF30608CDF30608696B060863
:10015000EDB8000801B9000815B9000819400608F3
:100160000DB20008B1C70008CDF30608CDF30608AC
:10017000CDF30608CDF30608CDF30608CDF3060847
:08018000CDF30608CDF30608DB
:1080000010B40C4B4FF0E02C1A68DCF8180019681B
:108010008A42F9D159688842F6D89C684FF47A713F
:1080200001FB04F31B1AB3FBF4F35DF8044B01FBF3
:1080300002307047281C0020074BD0F8E4105B6822
:10804000D0F8F0205B1A9A42B8BFC0F8F030012394
:1080500080F81C3100207047001000E0B04A00EBAF
:10806000800102EBC1012DE9F041CB685B68B3F8F8
:1080700014C01CF0010F4FEA800E40F082805FFABE
:108080008CF4A6074DD5BFF35F8F91F82840012CE3
:10809000E5B200F0F7804FEA400C198BBFF35F8F19
:1080A0000EEB000102EBC10191F82840022C00F018
:1080B00017810EEB000102EBC10191F82840032C5F
:1080C0000AD191F82A1039B10CEB0001114491F852
:1080D0008440002C40F06381998889B241F480612A
:1080E00099800CEB0001114491F986100EEB00040D
:1080F00002EBC40494F8284001348C420FD184442C
:10810000944400218CF884109CF88510002940F0DC
:10811000E080704402EBC000002380F82530BDE809
:10812000F08165076BD400EB4007174414F040045E
:108130001FFA8CF697F986504FEA400C00F0E68063
:108140001E8A0C6BF6B26655EEB2741C64B291F8DE
:10815000288087F88640E51CA845214600F0458127
:108160000EEB000502EBC50595F82850AC42BDD1D9
:108170000CEB00011144023676B281F8866031467C
:10818000B4E71C8824F400642404240C1C801C889C
:10819000A4B244F480641C8000EB4004144491F8C1
:1081A0002A50002684F886604FEA400C002D56D0F5
:1081B00094F88440002C4ED00EEB000102EBC1017C
:1081C000844491F828109444012402298CF88440B6
:1081D00004D1198889B241F4006119800EEB0001C5
:1081E00002EBC10191F8261041F0010119820EEB5A
:1081F000000302EBC30292F82830BDE8F08100EBE7
:108200004005154491F82A40012685F8856000FA5A
:1082100006FC002C7ED095F88440002C40F0828033
:108220000EEB000102EBC10191F82910002900F0CA
:10823000B98019880CEB0004144489B241F4007130
:10824000198094F88610013149B284F886101C8890
:10825000E705FCD44AE791F82710FF29ACD00EEBD4
:10826000000102EBC10191F8264004F0FE041C82DB
:1082700091F82730FF2BBAD084449444FF238CF824
:108280008630B4E791F82A1000293FF404AF00EBE0
:10829000400111444FEA400C91F88440002C3FF417
:1082A000FCAE1C8824F480642404240C1C80BFF3DE
:1082B0005F8F1C8B1C8881F88550A4B244F4007435
:1082C0001C809C8891F98610A4B244F480649C8040
:1082D0000CE7998821F440710904090C998018E78A
:1082E00091F82A1000293FF4E4AE0CEB0001114490
:1082F00091F88440002C3FF4DCAE1C8891F9861084
:1083000024F480642404240C1C8041E036062FD41D
:108310002946EBE695F88410002981D089E700BF53
:10832000281C002091F828400E6B022C1C8847D98D
:1083300024F480642404240C1C801F8A95F9864050
:10834000FFB237550F6B198889B241F4007119805B
:10835000E4B21E8A611C49B2F6B27E54A11C9C880C
:10836000A4B249B244F4806485F886109C806EE71C
:108370006E1C41D0CC6A665D6C1CF5B21D8291F812
:10838000285064B2A54287F8864021467FF4AEAEFD
:108390009C8824F480642404240C9C80A6E691F933
:1083A0008610F5E7198889B241F4807119800CEBC9
:1083B00000011144012481F8844091F9861046E7B8
:1083C000A4B244F400741C801F8A95F98640FFB261
:1083D0003755E4B20F6B1E8A611C49B2F6B27E5467
:1083E000E11C49B285F8861031E79D8825F4806547
:1083F0002D042D0C9D80B3E687F8864091F8274028
:10840000E4B21C8291F82A4024B991F8281000297E
:108410007FF4EDAE998821F480610904090C9980FC
:10842000E5E600BF10B404698269E468416814603D
:1084300000234024C2E90234446993630C31C2E949
:108440000433C2E90633C2E90833C2E90A33C2E998
:108450000C33516094B1C269E46893634FF4803087
:10846000C2E90041C2E90233C2E90433C2E906337A
:10847000C2E90833C2E90A03C2E90C335DF8044BD0
:10848000704700BFD0E9001300221A60037D1F2B44
:1084900007D9203B202202FA03F343F01803CB60F4
:1084A0007047202202FA03F343F018038B607047F1
:1084B0001B4B016803F57D7C02E02C3363452CD017
:1084C0001A688A42F9D170B593F804E0427996456A
:1084D0000BD02C33634505D01A688A42F4D02C3374
:1084E0006345F9D14FF0FF3070BD9E468468DEF8D9
:1084F0000C50A5424FF0000208D00132032A0EF1C1
:108500000C0EE6D0DEF80C50A542F6D1DEF8105085
:10851000C668B542F1D150B270BD4FF0FF30704720
:10852000181E0708002A4FEA014C30B503460ABF5F
:10853000E6468E468C4600F1C005002419689A680C
:1085400041EA0C0142EA0E029A60C3E900140C33BE
:10855000AB42F3D1D0F8C030C0F8C44043EA0E03B8
:10856000C0F8C030C0F8C84030BD00BF8369196989
:10857000B3F80CC00A6830B49C6822F00102246889
:108580000A60A28992B222EA0C02A281027D0068EE
:108590001F2A06D94568203A082494402C4245D029
:1085A000FEE70568082494402C42F9D1202404FAFF
:1085B00002F28260264A1278002A35D01A7E012AF9
:1085C00039D0D3F8F4200132C3F8F420EFF311814D
:1085D000502282F3128858685C6C026822EA040216
:1085E0009C6C2243C9B2026081F31188D3E90C402C
:1085F0001A6999681D6C096814605061D3E90E40CE
:10860000546090600024B3F8A800D5604C62C86242
:1086100010680124204310601C7683F8F1408A8999
:108620009B8913439BB28B8130BC7047202404FA92
:1086300002F2C260BEE7002283F8F120D3F8F8000E
:108640000A68013022F00102C3F8F8000A60EBE783
:108650000400001010B40C4C6368002B11DD0020E6
:1086600004F1080C0146DCF8A03003F1C0025960A7
:108670000C339342FBD16368013083420CF5807C5C
:10868000F1DC5DF8044B704704000010F0B5414C7C
:1086900004EB401393F8243403B9F0BD3E4B93F838
:1086A0008D5093F88E2095424FEA401C0CD002EB7F
:1086B000420E03EBCE0E9EF89060771E012F4FEA1C
:1086C000420E58D9032E51D004EB0C00A0F8081428
:1086D000EFF31182902383F3128890F80A34B0F8F4
:1086E000081443EA41030021D2B29BB280F80A1475
:1086F00082F311882178D0F820441A0982EA1322E3
:108700005A40C9B1D0F80C14D4F8A040D2431B0190
:108710009BB202F00F0201208840134304F1C00114
:108720005A0013F4004F93B202D1626802436260B0
:108730000C34A142F4D1F0BDD0F80C14D4F8A04010
:108740001B0110319BB202F00F020120884013433D
:1087500004F1C0015A0013F4004F93B202D16268D1
:10876000024362600C34A142F4D1F0BD561C06F005
:108770000306AE42A8D0964403EBCE03184490F80B
:108780009D100029A0D004EB0C03012283F80A24D9
:108790009AE700BF04000010281C0020704700BFAB
:1087A000024B03EB401393F82504704704000010BC
:1087B0004368B0F8502010B41A83EFF311825023AD
:1087C00083F312884168446C0B6823EA0403C46C89
:1087D0002343D2B20B6082F31188D0E9074182684B
:1087E000036912681C605961D0E909415C60C46A80
:1087F0009960B0F86010DC600023D1625DF8044B32
:108800000376704710B4037D02681F2B09D95468A2
:10881000203B202101FA03F31C4215D15DF8044BE3
:1088200070471468202101FA03F31C42F6D00D4969
:108830004068002481F8F04001685DF8044B21F0A5
:10884000010101609360704706494068002481F887
:10885000F04001685DF8044B21F001010160D36034
:10886000704700BF281C00200C4B0D49DB68DB4320
:10887000C3F30223C3F104030122DBB202FA03F3C0
:1088800001EB000C1B0103F0F0038CF800334309EB
:1088900000F01F00824041F82320704700ED00E007
:1088A00000E100E010B4037D02681F2B09D9546871
:1088B000203B202101FA03F31C4215D15DF8044B43
:1088C00070471468202101FA03F31C42F6D00D49C9
:1088D0004068002481F8F14001685DF8044B21F004
:1088E000010101609360704706494068002481F8E7
:1088F000F14001685DF8044B21F001010160D36093
:10890000704700BF281C0020122301480B807047CD
:1089100088010020042301480B8070479C0100203F
:108920001C48D0F8103AD0F8182A10B59B184FF010
:108930001A040C8001D1184810BD174AD0F8140A47
:1089400002F1100411464FF0000E4FEA137CB3F110
:10895000204F34BF0CF1300C0CF1370C81F802C001
:1089600081F803E002318C424FEA0313EDD102F1AA
:1089700008040021030FB0F1204F34BF30333733E8
:108980009374D174023294424FEA0010F2D102483B
:1089900010BD00BF0070FF1FA0010020D0E909201A
:1089A000131A58425841704790F84F3830B53BB9C8
:1089B00090F84D1890F84E380124DAB2914200D860
:1089C00030BDB0F8565804FA03F22A43A0F85628EE
:1089D0000133F2E70379024613F0010006D0D2E931
:1089E0000731D2685B1A013A03EA0200704710B5FA
:1089F000037913F0010304460ED0FFF7EBFF0346A3
:108A000050B1226A6369E1689B5C0132B2FBF1F00C
:108A100001FB1022DBB22262184610BD03799B07CE
:108A20000AD5436A8269D154436A02690133B3FBB0
:108A3000F2F102FB113343627047704701717047D6
:108A40000379014613F0020007D00B69D1E909212F
:108A5000013B521A1A40D2B2981A704782B01D4B8D
:108A60001D49002201920193019B04330193019B54
:108A70001A688B6803F00C03042B02D0082B05D076
:108A8000164A174BC3F8F42002B0704748684B6889
:108A9000400203F03F0314D44A681049B1FBF3F3DA
:108AA000C2F3881203FB02F20B4B5B68C3F3014372
:108AB00001335B00B2FBF3F2094BC3F8F42002B0C0
:108AC00070474968B2FBF3F2C1F3881303FB02F26B
:108AD000EAE700BF50280040003802400024F400BC
:108AE000281C00204A484B494B4BDFF830C12DE988
:108AF000F04F4FF0010A4FF002094FF00408082729
:108B00001026202540244FF0800E30F8022B12F062
:108B1000010F03D01960A3F804A0083312F0020F6C
:108B200003D01960A3F80490083312F0040F03D0A7
:108B30001960A3F80480083312F0080F02D01960FE
:108B40009F80083312F0100F02D019609E80083306
:108B500012F0200F02D019609D80083312F0400FF0
:108B600002D019609C80083312F0800F03D0196086
:108B7000A3F804E0083312F4807F05D04FF4807B23
:108B80001960A3F804B0083312F4007F05D04FF445
:108B9000007B1960A3F804B0083312F4806F05D08D
:108BA0004FF4806B1960A3F804B0083312F4006F1F
:108BB00005D04FF4006B1960A3F804B0083312F429
:108BC000805F05D04FF4805B1960A3F804B00833D0
:108BD00012F4005F05D04FF4005B1960A3F804B0F5
:108BE000083312F4804F05D04FF4804B1960A3F87E
:108BF00004B00833D20B04D04FF4004219609A80BD
:108C0000083301F5806161457FF47FAFBDE8F08FE7
:108C10000C22070800000240201D0020001802401E
:108C200010B584464FEA810E102312F4004F14BF92
:108C30000E2407245200013BCCF8004092B2F444C9
:108C4000F3D100EB81128C01035142F82130122044
:108C500010BD00BF10B584464FEA810E0424130BEB
:108C600003EB430318331201013CCCF8003092B2FD
:108C7000F444F4D100EB01130A01845043F821407D
:108C8000062010BD704700BF704700BF034B00EBCC
:108C9000400003EBC00393F819057047040000106F
:108CA000064B93F8C825824283BF00EB400003EBDC
:108CB000C003D3F81C050020704700BF040000105B
:108CC0001D4B93F8CC25AAB3D3F8081509B10020A1
:108CD0000860012A2ED0D3F8201509B100200860C1
:108CE000022A27D0D3F8381509B100200860032ADA
:108CF00020D0D3F8501509B100200860042A19D0FB
:108D0000D3F8681509B100200860052A12D0D3F8FD
:108D1000801509B100200860062A0BD0D3F89815F9
:108D200009B100200860072A04D0D3F8B0350BB190
:108D300000221A60704700BF040000101D4B93F81A
:108D4000CC25AAB3D3F8081509B100200860012A80
:108D50002ED0D3F8201509B100200860022A27D0B0
:108D6000D3F8381509B100200860032A20D0D3F8C1
:108D7000501509B100200860042A19D0D3F86815ED
:108D800009B100200860052A12D0D3F8801509B176
:108D900000200860062A0BD0D3F8981509B10020EE
:108DA0000860072A04D0D3F8B0350BB100221A604E
:108DB000704700BF04000010C24B93F83230002B04
:108DC00040F05781C04B93F8CC25002A00F0518128
:108DD00093F8181530B500294ED1D3F808150020A6
:108DE000012A086047D993F83015002967D1D3F8D4
:108DF00020150020022A08603DD993F84815002963
:108E000040F0D080D3F838150020032A086032D90A
:108E100093F86015002940F0E880D3F85015002041
:108E2000042A086027D993F87815002940F0FF80BC
:108E3000D3F868150020052A08601CD993F890150E
:108E4000002940F01781D3F880150020062A086019
:108E500011D993F8A81500295BD1D3F898150020F3
:108E6000072A086007D993F8C025002A76D1D3F8DD
:108E7000B03500221A6030BDD3F80C158A0AA2F56D
:108E80008012522A40F218814FF0FE0CEFF311804D
:108E9000502282F312888D4C4D6A8A8A4FF02C0E34
:108EA0000EFB0C4C92B2013542F00102CCF820547A
:108EB000C0B28A8280F3118893F8CC258DE7D3F86D
:108EC00024158A0AA2F58012522A40F203814FF03B
:108ED000FE0CEFF31180502282F312887B4C4D6A16
:108EE0008A8A4FF02C0E0EFB0C4492B2013542F0F0
:108EF0000102C4F82054C0B28A8280F3118893F82A
:108F0000CC25D3F820150020022A08603FF675AF63
:108F1000B1E7D3F89C158A0AA2F58012522A00F212
:108F2000F2806B48024492F800C4EFF311805022A3
:108F300082F31288654C4D6A8A8A4FF02C0E0EFB24
:108F40000C4492B2013542F00102C4F82054C0B280
:108F50008A8280F3118893F8CC257EE7D3F8B41584
:108F60008A0AA2F58012522A9BBF594812184FF064
:108F7000FE0C92F800C4EFF31180502282F31288A5
:108F8000524C4D6A8A8A4FF02C0E0EFB0C4492B262
:108F9000013542F00102C4F82054C0B28A8280F345
:108FA000118864E7D3F83C158A0AA2F58012522A88
:108FB00040F295804FF0FE0EEFF31180502282F3C5
:108FC0001288424C4D6A8A8A4FF02C0C0CFB0E44DE
:108FD00092B2013542F00102C4F82054C0B28A8234
:108FE00080F3118893F8CC250CE7D3F854158A0A3E
:108FF000A2F58012522A77D94FF0FE0CEFF31180C0
:10900000502282F31288314C4D6A8A8A4FF02C0E1E
:109010000EFB0C4492B2013542F00102C4F8205418
:10902000C0B28A8280F3118893F8CC25F5E6D3F894
:109030006C158A0AA2F58012522A5AD94FF0FE0CFA
:10904000EFF31180502282F31288204C4D6A8A8AF5
:109050004FF02C0E0EFB0C4492B2013542F001028F
:10906000C4F82054C0B28A8280F3118893F8CC25CA
:10907000DEE67047D3F884158A0AA2F58012522AD8
:109080003CD94FF0FE0CEFF31180502282F312888E
:109090000E4C4D6A8A8A4FF02C0E0EFB0C4492B295
:1090A000013542F00102C4F82054C0B28A8280F334
:1090B000118893F8CC25C6E60548024492F800C40E
:1090C000E4E600BF8801002004000010281C0020F6
:1090D000181E07080D48024492F800C4F9E60B4830
:1090E000024492F800E467E70848024492F800C49A
:1090F00084E70648024492F800C4A1E7034802440A
:1091000092F800C4BFE74FF0FE0C0EE7181E0708E8
:1091100000EE100AB8EE400A704700BFBCEEC00A6D
:1091200010EE103A98B27047072809D8054B8C22E8
:1091300002FB0033B3F8D005B0FA80F04009704765
:109140000020704704000010072806D8034B8C222B
:1091500002FB0033012283F8D2257047040000107F
:1091600070B53F4C8C2303FB004393F8DF3503B904
:1091700070BD3C4B93F88DE093F88E2096450CD053
:1091800002EB420C03EBCC0C9CF890506E1E012EAF
:109190004FEA420C44D9032D3DD08C2202FB004201
:1091A000A2F8D015EFF31181902383F31288B2F85F
:1091B000D05592F8D23543EA45030025C9B29BB297
:1091C00082F8D25581F311881A09217882EA132294
:1091D0005A4001B1D2431B019BB294F8341AD4F81F
:1091E000305A02F00F021A438C2303FB004431BBB8
:1091F0000121D4F85806A847D4F85416B4F8DC5521
:109200008A8AD4F850362A438A8258601A6842F013
:1092100001021A6070BD551C05F003057545BCD0F0
:10922000944403EBCC03034493F89D100029B4D07D
:109230008C2303FB0043012283F8D225ADE7D4F849
:10924000D835D4F854165B79086903F0FC03184448
:109250000421A847D4F854368000988170BD00BF1F
:1092600004000010281C00207AE700BF072808D857
:10927000044B03EB401393F8242412B1012283F82A
:109280000A24704704000010072808D8054B03EB98
:109290004013B3F80804B0FA80F04009704700208A
:1092A000704700BF04000010054B93F8C8258242A8
:1092B00086BF03EB4013D3F814040020704700BFAF
:1092C00004000010012343770020704708B50346CF
:1092D0008269006BD96A02449A6101B18847002013
:1092E00008BD00BF436A1B681B6A5B685B78024667
:1092F00013F0010008BF5077704700BFF0B5224C53
:10930000224A234B95B0054604F13C00CDE900020A
:10931000049304F140000023CDE90503CDE90E33A9
:109320001C4A09920B9304F1340210931393119386
:109330006B6A2F7F0A921868012302228DF80C3085
:1093400007938DF820308DF834308DF848303B1D70
:1093500002920E460C9364F02BF997B1330E84F809
:1093600035303634320C330A22706370A670686A66
:10937000694657F00BFC6B6A186864F019F915B070
:10938000F0BD3534EEE700BF8801002088220020C0
:10939000E5920008C592000810B5044694B050222A
:1093A0000649684668F0A4FA606A694657F0EEFB21
:1093B000636A186864F0FCF814B010BD6C220708EA
:1093C000C2628161704700BF2DE9F0410446406AE6
:1093D00000681E460F46904664F0EAF8237FA069B5
:1093E000002B3DD0274D030E85F84530052205F1B1
:1093F00046039870EA67020C000A58701A703B68BE
:10940000C5F888300020D8F80030C5F89030012E1B
:109410002363C5F8A00028D0022E1FD1D8F804205D
:10942000C5F89800796885F89400C5F89C10134435
:109430001549C5F8A4200120236385F8A800C5F8C4
:10944000AC10124B627F606AA3F11401002A08BFBE
:10945000194657F09BFBE36A7BB1206BBDE8F081B6
:109460000B4B0422A3F14505C3E7074B85F8946035
:10947000C5E92630C5F8A400E3E7636A186864F01C
:1094800097F8EAE788010020CD920008E801002063
:10949000CD010020704700BF00B583B0816101920B
:1094A000049A0093C26201236A4601A9FFF78CFF68
:1094B00003B05DF804FB00BF043070470D4B93F818
:1094C0006826D3F864160244D2B283F8682693F86B
:1094D000682601441206C3F8641605D593F8682679
:1094E00082F0800283F86826034B012283F8C420AF
:1094F000704700BF281C0020880100202DE9F0479C
:10950000154FD7F86C56ED0A20D00026B14607F269
:10951000A4687419D7F870361048D3F828A0C7F893
:109520009C9604EBD474641010234246E102D047A9
:109530000F280BDD0A4B03F1100153F8042B013205
:1095400007D18B42F9D12546B542E2DCE802BDE8FD
:10955000F087661CF8E700BF281C00209822002036
:10956000CC220020194B1968D3F8B4268A1A322A63
:1095700005DCD3F8C8268A1A002A0FDC704793F856
:10958000B826D3F8BC1602F0010219B10868898820
:10959000B2B901830022C3F8C8267047D3F8BC26AD
:1095A00082B11068928810B444693231224218BFE7
:1095B00042835DF8044B08BF0283C3F8C8167047A6
:1095C0004183E7E73231C3F8C8167047281C0020F2
:1095D000064AD2F8BC363BB192F8B8169A881B6896
:1095E000C90754BF1A835A8300207047281C0020E3
:1095F0004FF40070034B1060D3F8D8360B60002096
:10960000704700BF281C00200020704701207047D1
:10961000012070470020704710B41C6994420CD39D
:1096200094460A4661448C42996938BFA4EB0C0207
:1096300061445DF8044B68F05BB95DF8044B70471A
:1096400030B585B068465BF091F80F480F4AD0F806
:10965000FC10009B0E4D41F08071C0F8FC100024FE
:1096600000F1C840C2F8B05FA0F565005460116811
:10967000084CA0F67D60A0FB030341F001019B0CA8
:10968000A360116005B030BD00ED00E0001000E007
:1096900055CEACC5281C00202DE9F84F01307E4C7A
:1096A0007E4D01F1FF385FFA80FB1026012761F043
:1096B0001DFD4FF4FA794FF0E0214FF47A7C6B688E
:1096C000C3F30803002B40F0C080EFF31183002B9D
:1096D00040F0BB802368886922689342FAD16268AF
:1096E0009042F7D8A2680CFB02FEAEEB000EBEFB68
:1096F000F2FE0CFB03EE6B68C3F30803002B40F093
:109700008680EFF31183002B40F081802368886905
:1097100022689342FAD162689042F7D8D4F808A040
:109720000CFB0AF2121AB2FBFAF20CFB0323A3EBB6
:109730000E03B3F57A7FDED3B9F10109BFD15846E4
:109740004FF47A7962F086F94FF0E021CC466B68ED
:10975000C3F30803002B40F08B80EFF31183002B41
:1097600040F086802368886922689342FAD1626853
:109770009042F7D8A2680CFB02FEAEEB000EBEFBD7
:10978000F2FE0CFB03EE6B68C3F308030BBBEFF3B5
:109790001183F3B92368886922689342FAD1626819
:1097A0009042F7D8D4F808A00CFB0AF2121AB2FBC8
:1097B000FAF20CFB0323A3EB0E03B3F57A7FE2D39B
:1097C000B9F10109C3D1B8F10108BFF470AFBDE828
:1097D000F88FEFF3118386F31288D1F818A00A6985
:1097E000D20344BFC4F80877D1F818A02068D4F891
:1097F0000827DBB283F311880244A0680CFB00F356
:10980000A3EB0A03B3FBF0F30CFB0233D3E7EFF354
:10981000118386F31288D1F818A00A69D20344BFD5
:10982000C4F80877D1F818A02068D4F80827DBB26C
:1098300083F311880244A0680CFB00F3A3EB0A0336
:10984000B3FBF0F30CFB023371E7EFF3118286F305
:10985000128888690B69DB0344BFC4F808778869FC
:109860002368D4F808E7D2B282F31188734439E749
:10987000EFF3118286F3128888690B69DB0344BF1A
:10988000C4F8087788692368D4F808E7D2B282F36D
:10989000118873446EE700BF281C002000ED00E033
:1098A0002DE9F0411D4CDFF87C801D4F82B004F59E
:1098B0004075012602E00834A54224D094F9063010
:1098C000002BF8D1206800F13F4303F57E0308EB3D
:1098D000932393F8A4345A09032A03F01F0306FACA
:1098E00003F317D0042A11D0022A02D17A6C134351
:1098F0007B640023A1881A46CDE90036083463F062
:10990000FDFDA542DAD102B0BDE8F0813A6B134308
:109910003B63EEE73A6C13433B64EAE7201D00200B
:1099200000380240181E070809494B6C10B5094C55
:1099300043F480434B644022002104F20C7068F031
:109940002FF84FF0FF33C4F84C37C4F84F3710BD31
:1099500000380240281C00202DE9F0411348144D26
:109960004FF41A72002168F01BF84FF00008A5F2BE
:10997000AC4705F6880440F2222655F8281000234B
:1099800054F8332091420BD001330E2BF8D1002034
:1099900008F1070862F0C4FBB045EED1BDE8F081E4
:1099A00007EBC30393F8380DF2E700BF2020002037
:1099B000C42207082DE9F843038AB0F80C801FFA87
:1099C00088F818EA030829D005460E464FF00047EC
:1099D000B8FA88F327FA03F2D24391B21B3B2982EB
:1099E00008EA0208042B16D8DFE803F0352C231A06
:1099F0000300B36A002B37D003F1FF3900231FFAAD
:109A000089F9B362746A34B123682046494698479D
:109A10006468002CF8D1B8F1000FD9D1BDE8F88303
:109A20007068696B036889B29847B8F1000FCFD1AD
:109A3000F4E7B068A96B036889B29847B8F1000FE2
:109A4000C6D1EBE7F068E96B036889B29847B8F1D3
:109A5000000FBDD1E2E73069296C036889B29847ED
:109A6000B8F1000FB4D1D9E7EB6A1FFA83F9C9E75F
:109A700070B50B4C05460726013E00D170BD94F928
:109A800000001AF075FC031E08DBEA18617891717A
:109A9000A178E954052BDCBFE37813730434EBE7BA
:109AA000BC2B070810B5274B93F88D2093F88E3008
:109AB0009A4242D1244A92F8F80AF8B192F8344A0C
:109AC00002F6382300EB4000D2F8382A03EBC0003E
:109AD000B4B140F20D3C00E01A6899689C894C6072
:109AE0000C6844F001040C60A2F848C09189183356
:109AF00089B241F4807183429181EDD110BD1A6821
:109B0000118821F0800109041833090C118033F801
:109B1000141CD162118889B241F080011180546215
:109B2000B2F80CC033F8041C41EA0C0189B283423C
:109B3000918123F8044CE2D110BD63F0B3FF0028FB
:109B4000B8D110BD281C00200400001010B5044638
:109B500066F096FE81B22046BDE81040FEF796BD45
:109B600010B5044666F08CFE81B22046BDE8104078
:109B7000FFF7F6BA38B50B4D00EB400005F5A163D1
:109B800003EBC00393ED027AD3ED037AE7EE007A9C
:109B9000C4002544B0EE670A66F072FED5F80835B9
:109BA000186038BD040000100A4608B5054920B900
:109BB00005485CF065FF034808BD04485CF060FFA1
:109BC000004808BD7C230020A8BF0708D0BF0708B5
:109BD00010B5044C04480A4621465CF051FF20466B
:109BE00010BD00BF7C230020F8BF070810B5044C4F
:109BF00004480A4621465CF043FF204610BD00BFE2
:109C00007C2300200CC0070810B5044C04480A4609
:109C100021465CF035FF204610BD00BF7C230020AC
:109C200018C00708F8B5A0F668042379DB0725D526
:109C3000657994F84C3805F001073D46FBB1D4F83E
:109C400048341A68D36A5B08536294F8503823B1D9
:109C5000B4F85A380133A4F85A38606C85F0010121
:109C600060F090FA012384F84F38002384F84D38CF
:109C700084F84E38A4F8563884F84C38F8BD94F877
:109C80004F68012E04BF94F84D3884F84E382046B2
:109C9000FEF78AFE4EB9012384F84F3887EA0301A4
:109CA000606CBDE8F84060F06DBA002384F84F386E
:109CB0003946F5E738B5A0F668040022606C344DEB
:109CC00003685A62A1F12903302B31D895F8533833
:109CD00095F854180133DBB2012B85F8533809D9B4
:109CE000B4F8563885F853285B08A4F856384B1C4E
:109CF00085F8543895F854280023082AA4F85838D1
:109D000015D185F85438B5F8563801339BB2032B7A
:109D1000A5F8563808D92379DB0705D5E36A94F806
:109D2000560843B3216B98470023A4F8563838BD32
:109D30005B396C290CD8B4F8563885F853285B0881
:109D400043F08003A4F8563895F854380133CFE730
:109D500094F85138002BCDD1012185F85338A5F85E
:109D60005638802384F85118A4F8563885F85418CA
:109D700060F008FABEE7E3696269D054E369E2681B
:109D80000133B3FBF2F102FB1133E361CCE700BF17
:109D9000281C00208069002836D003681A6A127BCC
:109DA0002ABBD3E904125B68496872B110B45468E5
:109DB00000220A6022609A885DF8044B22F00302B8
:109DC0001204120C9A8059F0D5B91A891206FCD4E3
:109DD0001A89D20709D400220A609A8822F0020266
:109DE0001204120C9A8059F0C5B99A89F0E782687A
:109DF000002AD6D0116892880A83D3E904125B68DE
:109E00004968002AD2D1E0E7704700BF806900B9F5
:109E10007047016830B4D1E904424B6864687AB194
:109E20005568002222602A609A8822F003021204F8
:109E3000120C9A800B6A1B7BA3B930BC59F09AB9FB
:109E40001A891506FCD41A89D20714D4002222607C
:109E50009A8822F002021204120C9A800B6A1B7B71
:109E6000002BEAD08368002BE7D01A689B88138305
:109E700030BC59F07FB99A89E5E700BF38B590F852
:109E80002830012B044606D0407F08B9012038BD98
:109E90000023637738BD406A03681A7B92B9637FF9
:109EA000002BF3D00A4D0B49022305F6580256F059
:109EB00027FE95F85938D84303F0010300F001005C
:109EC0006377E7E71B6A002BE9D0002038BD00BFAD
:109ED000281C00205002002038B5044694F8283091
:109EE000012B07D0637F0BB100236377012038BDBE
:109EF0001B6A23B1606A03681A7B002AF8D1637F6A
:109F0000002BF3D0074D0849022305F6580256F0FE
:109F1000F7FD95F8593803F00102DB076277E5D5C4
:109F2000DCE700BF281C0020500200202DE9F84388
:109F3000DDF820800F4615460021202204461E46EB
:109F400067F02EFDB8F1000F0CD0D8F80030E38197
:109F50001B0C2382D8F80430B8F80A20E3821B0CCB
:109F600062822383384664F0F9FCEB0619D4431E61
:109F7000B8B107EB000C01E0013B12D31CF801ED76
:109F8000BEF12E0FF8D1C01A421E032AA8BF032229
:109F9000082B03F10109A8BF08239046B9441A46CB
:109FA00006E008280246B946A8BF08224FF000087C
:109FB0004FF02033394623606360204667F098FCF9
:109FC00004F10800154B238142464946837067F02F
:109FD0008FFC611EE21D11F801CFACF16103192B5A
:109FE0009CBFACF1200C81F800C09142F3D104F188
:109FF0000A0011F8013FA3F16102192A9CBF203B1E
:10A000000B708142F5D118232373330CA382E572C0
:10A01000099B6683E361BDE8F88300BF2020200030
:10A020002DE9F04FDFF84CB4DBF8000085B0CBF839
:10A03000B406002B60D013440C46174601F5FE7A97
:10A0400099461FE0002F64D0DBF8E436BB4200F0F5
:10A05000C680DBF8E036BB4200F0F880DBF8E8367B
:10A06000DBF8EC16BB424BD8B94200F27081791A8A
:10A0700020465FF0B9FA01374F4504F500740AF540
:10A08000007A39D0DBF8F036BB42DBD8DBF800577A
:10A09000FB1A296BDA0802328A4203F0070602D360
:10A0A000AB6B9A420BD92946104602925FF06CFACC
:10A0B000029A0546002800F06A81CBF800072B7948
:10A0C000002B40F01E81D5F82880B8F1000F00F079
:10A0D00057812B6BD21AEB6806EBC20203EB4222CC
:10A0E00020462B464FF400710137C0474F4504F519
:10A0F00000740AF5007AC5D1002005B0BDE8F08FE4
:10A10000B942B4D94FF400720021204667F048FCF0
:10A11000B1E74FF400723946204667F041FC8023D6
:10A1200084F8BE310C2384F8C231DBF8E016C54A4E
:10A13000DBF8D836C4F8C6119142C4F8CA3100F32E
:10A140000B81C14AC14D82FB010285FB01050A4416
:10A15000C817C0EB6212C0EB2530BD4D84F8C101B9
:10A1600085FB0265C2EB82168010891B013120F04D
:10A170003F0015440843D117C1EBE5110A4484F8A8
:10A18000BF21B04A84F8C001013B934200F3F08044
:10A19000AD4AAE4882FB031280FB03101A44D91764
:10A1A000C1EB6212C1EB2031A94884F8C51180FBD4
:10A1B0000250C2EB821589105B1B013321F03F0175
:10A1C00010441943D317C3EBE0131A4484F8C411A5
:10A1D00084F8C3214AF65523A4F8FE314BE74FF02B
:10A1E000FF3384F8EC3184F8ED3184F8EE3184F8F3
:10A1F000EF315223237063706123A37084F8E73139
:10A200004123E37084F8E6317223002584F8E431B9
:10A2100084F8E531DBF8F836C4F8E8314FF4F07231
:10A220002946201D67F0BCFB552384F8FE316FF0F2
:10A230005503C4F8F051C4F8F451C4F8F85184F847
:10A24000FC5184F8FD5184F8FF3114E74FF400729B
:10A250000021204667F0A4FB7E4B03CB45F6EB03C1
:10A2600023809023C4F80710A37002220821F8234A
:10A27000C4F80300617322746375DBF8D836227367
:10A28000A27384F82C20DBF8E0269B1A2362DBF80B
:10A29000E826DBF8EC369B1A63620023E372E37373
:10A2A0006377A377E37784F82D3084F82E3084F831
:10A2B0002F3084F83130684BA361684BC4F84230CA
:10A2C0003E232377012384F83030654A802384F8C5
:10A2D000403084F846104AF65521A4F8FE1103CA0E
:10A2E000604BC4F84700C4F84B1003CB1388A4F8A4
:10A2F0004F309378C4F85200C4F8561084F85130A7
:10A30000B9E64FF400720021204667F049FB002EA9
:10A3100044D12B6C04F12008002B7BD02B6B5249CD
:10A320001122CDE900662046FFF700FE2B6C1A6C67
:10A33000002A7ED01B6B4D49CDE9006640461122B4
:10A34000FFF7F4FD04F140084FF4E0736DE0F91AF3
:10A3500020465FF049F98EE6FF2284F8C1214FF6CE
:10A36000FF72A4F8BF21374A013B93427FF710AF39
:10A37000FF2384F8C5314FF6FF73A4F8C33129E7F2
:10A3800041464FF40072204667F00AFB73E6384AF4
:10A39000231F43F8042F9A45FBD16CE6D5E910251D
:10A3A0003301002A43D0023B002D3FF464AE013B51
:10A3B000AD6CF9D1A0464FF40073002D3FF45BAEB5
:10A3C000CDE9027A08EB0306A24608E00024CDE9B5
:10A3D00000C4FFF7ABFDAD6CBDB1B04515D02C7915
:10A3E00029682B6B404605F11C0C112208F120084E
:10A3F000002CEBD16A792C6942F02102CDE900C42E
:10A40000FFF794FDAD6C002DE7D15446029FDDF8B7
:10A410000CA030E6CDE900663346DBF8DC160822F6
:10A420002046FFF783FD4FF4F0736D6CC5E7013BE9
:10A43000BAE7CDE900660D49334640461122FFF7E1
:10A4400075FD7FE7FF03FB00832008829755454198
:10A450008180808030C007083F00FF0029940E0DE6
:10A460003CC0070848C0070828C007082CC00708D8
:10A47000DEADBEEF281C002010B4EFF311821023D4
:10A4800083F31288084B19684FF0E02001311960FE
:10A49000816959600024C3F808470369D3B283F384
:10A4A00011885DF8044B7047281C002010B4EFF3AE
:10A4B0001181102383F312884FF0E022C9B294690E
:10A4C000136913F4803F0C4B1EBF0120C3F808072B
:10A4D00094691868D3F8082781F3118899680244B1
:10A4E0004FF47A7000FB01F31B1B5DF8044BB3FBC8
:10A4F000F1F300FB02307047281C0020234B5B68FF
:10A50000C3F3080310B4DBB9EFF31183C3B9204BD5
:10A510004FF0E02C1A68DCF8180019688A42F9D16B
:10A5200059688842F6D89C684FF47A7101FB04F3AD
:10A53000181AB0FBF4F05DF8044B01FB0200704701
:10A54000EFF31181102383F312884FF0E022C9B298
:10A550009469136913F4803F0D4B1EBF0120C3F8AB
:10A56000080794691868D3F8082781F31188996857
:10A570004FF47A73024403FB01F0001B5DF8044BB7
:10A58000B0FBF1F003FB0200704700BF00ED00E0FC
:10A59000281C00202DE9F04F037D02681F2B83B09B
:10A5A000044609D95068A3F120052021A9400142A1
:10A5B00007D103B0BDE8F08F106820219940014217
:10A5C000F7D04749474D4968A769C5F8FC1A8C215F
:10A5D00001FB075195F834CAD1F8D8050668BCF1DB
:10A5E000000F18D1D1F85006B1F8DCC5016821F090
:10A5F00001010160B18989B221EA0C01B181297898
:10A60000B9B91F2B60D9A3F1200120238B40D3605F
:10A6100003B0BDE8F08F0069016821F0010101601D
:10A62000B18921F480710904090CB18129780029CC
:10A63000E7D04FF08C0808FB07F805EB08030193FF
:10A64000D3F850A6DFF8A0B050465AF0DBF8019BD3
:10A65000012283F82426D5F8043B08F11809D944CF
:10A66000002B38D033889BB243F08003338008F14D
:10A6700074084FF0FF330BEB0801F36230465AF0D9
:10A6800007FB8C2303FB0757494600235046C7F8B6
:10A69000F43558F01BFCD7F8503616225A601A6869
:10A6A00042F001021A60D7F8D825B7F8DC351268F5
:10A6B00091890B439BB293810949237D49682268A4
:10A6C000C5F8001B1F2B9ED8202101FA03F39360CD
:10A6D00003B0BDE8F08FFFF711FFC5F8040BC1E729
:10A6E000001000E004000010D40500102DE9F8432C
:10A6F000FFF704FF204F214E7C6805464FF000080D
:10A70000002C2DDD00231A4607EB0321013391F8BD
:10A71000F9109C4242EA0102F6D142EA08095FFAC6
:10A7200089F990467368C3F30803B3B9EFF3118353
:10A730009BB9FDF765FC401BB0F5FA6F02DCB8F180
:10A74000000FDDD1B9F1000F04D00D4B93F85A285A
:10A75000542A09D04846BDE8F883FFF7A7FEEAE788
:10A76000C1464FF00008DDE7B3F860280132A3F8D6
:10A7700060284846BDE8F8830400001000ED00E0C2
:10A78000281C0020AD4B1B780BB9012070472DE928
:10A79000F04FDFF8BCB2AA49DBF80020A94BA1FBBF
:10A7A00002125209A3FB0213DB08A44987B003EB92
:10A7B0008303A2EB430391F8C825049201F6083401
:10A7C000DAB2059204EB8307002201F6E853019305
:10A7D00001F5816A9046049B984500F00D81DAF8F6
:10A7E0001820DAF80490D2F8E830D2F8EC6002933E
:10A7F000FFF784FE029B03904FEA890C9BF85A985E
:10A800009BF86C080CF1085C06F180610CEB431CB2
:10A810003939B9F1540F0CEB81110CEB801301D1D4
:10A82000ABF86208994240F27D811A68002A00F074
:10A8300071811A6C002A00F08381D3F88020002AED
:10A8400000F08081D3F8C02003F58073002AE9D19D
:10A85000A3EB0C0C99424FEAAC1240F26381B11A9F
:10A8600045294FF0000628BF45213046B64603EB88
:10A8700081111D4616460DE01A6C002A40F0EA8050
:10A88000D3F88020002A40F01581D3F8C02003F5CA
:10A8900080732AB9994206D91A68002AECD040334D
:10A8A000994200F2DB8032467646112E40F23E811C
:10A8B000DEF1150100F13A81634B1D46D3F8CC302F
:10A8C0009A4238BF2B46039D38BFC3F8CC20DBF833
:10A8D0007038EA1A002A18DB03F5F42303F59073A5
:10A8E0009D4284BF2B460533CBF87038564B564AF1
:10A8F000D3F8CC30052B86BF053BDBB200238BF8A9
:10A900006C384FF0FF33C2F8CC3031B100FA01F1AE
:10A91000C6F114060120B04008434C4EC0F3C433C6
:10A9200006EB8303D3F8BC1D00F01F0306EB830383
:10A93000D3F8BC2D42EA0132C0F3441106EB810189
:10A94000C0F3842306EB8303D1F8BC1DD3F8BC3DD0
:10A9500042EA011141EA032181EA112383EA131338
:10A9600003F00F02354BD3F8F03D0F2A03F101033A
:10A9700040F0BD80B1F5803F80F0B980B9F1540F4F
:10A980004FEA111140D02D4AB1F5606FC2F8F03D89
:10A9900045D0019B998194F85830059883420CD09A
:10A9A000BA6823689B1A23603A6B63689B1A6360DA
:10A9B0000023BB603B6384F85800236801332360A5
:10A9C000BB680133BB604FF6FF73994205D16368E2
:10A9D000013363603B6B01333B63019B08F101086A
:10A9E0001433B8F1080F04F15C0407F15C0701931C
:10A9F0000AF1200A7FF4EFAE104A0123012082F809
:10AA0000EC3E07B0BDE8F08FBBF85C280132ABF834
:10AA10005C280A4AB1F5606FC2F8F03DB9D19BF8E5
:10AA20008E3003EB43030BEBC303434493F89D3099
:10AA30000D2BAED1019A80239377ACE70400001070
:10AA40001F85EB51CDCCCCCC88010020181E070807
:10AA5000281C0020803399427FF625AFA3EB050C1C
:10AA60003C4A4FEAAC1C0CF1010C82FB0C52A2EBED
:10AA7000EC72012AB8BF012290404FF0010C9644BD
:10AA8000013A0CFA02F210439C46DCF800209AB11D
:10AA9000DCF84020002A57D0DCF88020002A56D06D
:10AAA000DCF8C0200CF5807C42B16145EDD81D4634
:10AAB0006346EFE6C033F3E60CF1400C6145F6D98E
:10AAC000ACEB03029211234B013283FB0253A3EB45
:10AAD000E273012BB8BF012398409E440122013B41
:10AAE00002FA03F3184363461D466346D2E6B9F102
:10AAF000540F04D1BBF85C280132ABF85C28164A2D
:10AB0000C2F8F03DD2F8EC3D0133C2F8EC3D4FF60F
:10AB1000FF7140E74033A3EB0C0C99424FEAAC12B3
:10AB20003FF69DAE10B101388BF86C08B9F1540FA7
:10AB30007FF453AFBBF85E380133ABF85E384CE7B7
:10AB4000803385E6C03383E60CF1800CB6E70CF168
:10AB5000C00CB3E75655555504000010F8B51D4B11
:10AB600093F88D2093F88E309A422ED11A4F7D683B
:10AB7000002D11DD3846002410F8086B16B1037E55
:10AB8000012B1CD002691368013443F00103A54274
:10AB900000F580701360F1D1FFF7B0FCD7F8F04EEC
:10ABA000002C0BDD0D4A02EBC404116893888889E0
:10ABB000083203439BB294428B81F6D1F8BD002347
:10ABC00080F8F030FDF7F4FDDCE762F06BFF002861
:10ABD000CCD1F8BD281C002004000010F80E001095
:10ABE000454B5B68C3F308032DE9F0430546002B92
:10ABF0005ED1EFF31183002B5AD1404B4FF0E0248C
:10AC00001A68A06919688A42FAD159688842F7D847
:10AC10009E684FF47A7101FB06F4241AB4FBF6F433
:10AC200001FB0244344E10274FF0E02C4FF47A7EA3
:10AC30004FF001087268C2F30802CAB9EFF311823B
:10AC4000B2B91A68DCF8180019688A42F9D1596853
:10AC50008842F6D8D3F808900EFB09F1091AB1FB27
:10AC6000F9F10EFB0212121BAA42E3D3BDE8F083F6
:10AC7000EFF3118287F31288DCF81800DCF810106B
:10AC8000C90344BFC3F80887DCF81800D3F8009064
:10AC9000D3F80817D2B282F311884944D3F8089048
:10ACA0000EFB09F2121AB2FBF9F20EFB0122DAE7EF
:10ACB000EFF31181102383F312884FF0E022C9B221
:10ACC0009669136913F4803F0C4B1EBF0120C3F833
:10ACD000080796691868D3F8082781F31188024499
:10ACE00098684FF47A7101FB00F4A41BB4FBF0F4F4
:10ACF00001FB024496E700BF00ED00E0281C0020A5
:10AD00002DE9F0473A4B3B4D471E10264FF0E0200F
:10AD10004FF47A7C4FF001086A68C2F30802002AF7
:10AD200052D1EFF31182002A4ED11A688469196852
:10AD30008A42FAD159688C42F7D899680CFB01FE17
:10AD4000AEEB040EBEFBF1FE0CFB02EE6A68C2F332
:10AD50000802E2B9EFF31182CAB91A688469196866
:10AD60008A42FAD159688C42F7D8D3F808900CFB84
:10AD700009F1091BB1FBF9F10CFB0212A2EB0E0267
:10AD8000B2F57A7FE2D3013FC6D2BDE8F087EFF398
:10AD9000118286F3128884690169C90344BFC3F82C
:10ADA00008878469D3F800A0D3F80817D2B282F3D9
:10ADB0001188D3F8089051440CFB09F2121BB2FB26
:10ADC000F9F20CFB0122D9E7EFF3118186F3128827
:10ADD00084690269D20344BFC3F808878469D3F841
:10ADE00000E0D3F80827C9B281F311887244A4E7C0
:10ADF000281C002000ED00E030B50C4683B005466D
:10AE0000D8B1036803F13F4303F57E039B0A0C4A64
:10AE1000134493F8A40461F083F9C4F34112C4F31A
:10AE20000013CDE90032C4F38103A988286804F037
:10AE3000030262F063FB03B030BD4FF0FF33E6E77F
:10AE4000181E070800B1D7E7704700BF70B50E4C59
:10AE500094F8C865B6B104F58164002504E00135B5
:10AE6000B54204F120040DD0237F002BF7D0E06819
:10AE70000028F4D0217D0135FFF7BEFFB54204F173
:10AE80002004F1D1012070BD0400001070B5002431
:10AE900086B0CDE90144CDE903440DF1040CC0E9CD
:10AEA0003D44C0E93F44C0F80441054600F5847EB6
:10AEB000BCE80F00AEE80F00CEF8004095F8213155
:10AEC000059444F23B36A5F84C610BB906B070BD51
:10AED0001C09013C052C03F00F0332D81F4E06EB72
:10AEE0004402B2F8F40340FA03F2D20729D5012252
:10AEF00002FA03F3013B1840264466F0E5FD96F89C
:10AF00003C3E174A034402EBC30452F83320A388A3
:10AF100012691340DAD12946124A2620E08041F80E
:10AF20000C2F20461A465FF06BFF0F49A288086875
:10AF3000B2FA82F24FF00043D34003430B6006B0F5
:10AF400070BD2946074B41F80C3F00231A461846AE
:10AF500006B0BDE870405FF053BF00BF181E070881
:10AF6000201D00204DB30008003C014048B18288FC
:10AF70000449B2FA82F208684FF00043D340034319
:10AF80000B607047003C014030B1036882881B6948
:10AF90001A4214BF01200020704700BF38B50409D1
:10AFA000013C052C1AD80F4D05EB440200F00F03AD
:10AFB000B2F8F40340FA03F212F0010210D00122B9
:10AFC00002FA03F3013B1840254466F07DFD95F835
:10AFD0003C3E054A034402EBC30038BD002038BDA7
:10AFE000104638BD181E0708201D002008B519F0AE
:10AFF000BFF9052807D8054BD3F874380344187BEC
:10B00000BDE80840CAE7002008BD00BF281C00209A
:10B0100008B51D20FFF7C2FF10B190F9063053B1FB
:10B020001E20FFF7BBFF10B190F9063003B108BD39
:10B030005523C38008BD5523C380F1E7F8B5037DD0
:10B04000856902681F2B04464BD95068203B20219C
:10B050009940084237D0D16010219940D1605168A1
:10B06000D940CE077FD4EFF31183502282F31288A8
:10B070002A6C1168C90757D4516889B291B9D5E9CA
:10B08000096086424DD0AF699CBF0E4629690744CE
:10B0900094BF081A301A80B20021D760AE6285F8DA
:10B0A00064105060116841F00101DBB2116083F35C
:10B0B000118895F86430002B3DD1237D22681F2B29
:10B0C000194614D9203B506808219940084200D005
:10B0D000D1605068042101FA03F3184200D0D36014
:10B0E000F8BD16682020984006420DD11946106818
:10B0F00008238B40184200D09360106804238B40D3
:10B100001842EDD09360F8BD102199409060916095
:10B110001168D940C807A6D5012101FA03F393604D
:10B12000A1E7012285F86420DBB283F3118895F84A
:10B130006430002BC1D095F87230002BBDD195F84A
:10B140007100FFF72BFF2A6E938923F008031B047D
:10B1500001211B0C938185F872100028ADD02021AD
:10B16000FFF74AFEA9E7012101FA03F3D3607AE76A
:10B1700008B55BF003FD1B20FFF710FF08B1292382
:10B18000C3801C20FFF70AFF08B12923C3800A4BA4
:10B1900093F87D28012A01D0012008BD0748C3F893
:10B1A000800800F120014C305EF06CFA044B002066
:10B1B00083F8230008BD00BF281C0020580200208F
:10B1C00000ED00E043680B4A23F0407323F48073E2
:10B1D00043F48073436083681A4042F00202826045
:10B1E000C36A0139C9B223F4700343EA0153C3624D
:10B1F000704700BFFDF7FFC0704700BF0020FCF79D
:10B200002DBF00BF0120FCF729BF00BF0220FCF7C3
:10B2100025BF00BF10B1036882881A83704700BF42
:10B2200010B1036882885A83704700BFF0B5056883
:10B2300090F888606B688488012285F824201A8839
:10B2400022F040021204120C1A802A89A24255D11F
:10B25000017BAA7A8A420BD01A8822F003021204D8
:10B26000120C1A801A8892B2002944D01A80A9724E
:10B270001A882F7B92B242F040021A802B6A9A6899
:10B2800092B34FF0000C2F4C1433E64653F8101CC9
:10B29000964401EA040221B1B2F1805F27D06A69C5
:10B2A0002AB353F8142C143302EA040112B1B1F199
:10B2B000805F1CD053F80C2C0CF1010C002AE5D156
:10B2C000AFB1A6B1BCF1010F0AD8BEF1070F07D884
:10B2D0000CEB8C0C4FEA8C022B6A13441B7B33B9AA
:10B2E000BDE8F04057F020BE0FB1002EF4D1BDE80C
:10B2F000F04058F097B842F00302B7E71A881249B5
:10B3000022F0380212048B424FEA124217D001F5A4
:10B3100080618B4213D02146B1F5807FA8BF4FF4E6
:10B3200080710229B8BF022191FAA1F1B1FA81F12D
:10B33000013942EAC10292B21A802C8188E7610881
:10B34000EAE700BF0000FFFF0038004038B52C4A94
:10B35000D0F8E0305268D0F8D810044673B1501AD3
:10B3600083420BDC94F8D030C4F8D820012B10D0E5
:10B37000D4F8D4300133C4F8D43038BDD4F8E43034
:10B38000C4F8D8200B44C4F8DC3094F8D030012B3A
:10B39000EED16168201D04F1E805EFF3118C102354
:10B3A00083F3128863681B6A0BB3D4F8F0302A4623
:10B3B0001BB1D3691432002BFBD10B6A6BB19968B6
:10B3C00039B9934209D0196829B15B689968002995
:10B3D000F7D01433F3E7C3E900055FFA8CFC8CF374
:10B3E0001188D4F8D4300133C4F8D43038BD0D629C
:10B3F0005FFA8CFC8CF31188FFF718FFB8E700BFE9
:10B40000001000E02DE9F041826992F8DC30012B58
:10B410008AB005464CD0023B012B54D892F84C31EF
:10B42000D2F89C202E4C63F07F0313708769D7F805
:10B43000A030D7F8108003F1010E0FCCEC46ACE839
:10B440000F00D7F89C30CDE9003E0FCCACE80F00E0
:10B4500094E8030007F110068CE80300EFF3118075
:10B46000102383F312883B691B6A002B2FD0029BA9
:10B470006A461BB1D3691432002BFBD1D8F82030B7
:10B4800073B1996839B99A420AD0196829B15B68D1
:10B4900099680029F7D01433F3E71E60C3F804D08D
:10B4A000C0B280F31188AA6911690B6A002BFCD124
:10B4B000D2F8A0305A8852BAEA819A8852BA2A82BF
:10B4C000DB885BBA6B8201200AB0BDE8F081C8F866
:10B4D00020D0C0B280F311883046FFF7A7FEE2E724
:10B4E0005C2C07082DE9F04190F8DC30D0F8A05032
:10B4F000012B8AB0044673D041D9023B012B6BD893
:10B5000090F84D31D0F89C205E4E63F07F031370AD
:10B51000D0F8A030D0F8108003F1010E00F1100730
:10B520000FCEEC46ACE80F00D4F89C30CDE9003EDD
:10B530000FCEACE80F0096E803008CE80300EFF3B1
:10B540001180102383F3128823691B6A002B00F0FB
:10B550008F80029B6A461BB1D3691432002BFBD14A
:10B56000D8F820302BB3996839B9934221D01968A3
:10B57000E1B15B6899680029F7D01433F3E7D0F89C
:10B580009C304FF0FF321A605A609A60DA60D0F84F
:10B59000E0300522B3F57A7FC0F8F0203BD80323D2
:10B5A00080F8DC3001200AB0BDE8F0811F60C3F8EC
:10B5B00004D0C0B280F311882269136A002BFCD139
:10B5C0006B885BBAA4F8D030AB885BBAA4F8D230F1
:10B5D000EB885BBAA4F8D43001200AB0BDE8F08152
:10B5E00090F84C2190F84D319B1A5B100133DBB27F
:10B5F00005EB430235F813305BBAA0F8D03053881E
:10B600005BBAA0F8D23093885BBAA0F8D43001209E
:10B610000AB0BDE8F08103691A7B2AB35B691BB3EA
:10B6200090F8983003B390F84C31D0F89C20C4F8CF
:10B63000A40063F07F03137090F84C1190F84D3123
:10B64000D0F8A0201048C4F804015B1A0733012188
:10B65000C4F8FC30D4F89C3084F800110A44C4E9E2
:10B660003D3284F8DC10B7E7022384F8DC30B3E71E
:10B67000C8F820D0C0B280F311883846FFF7D6FD55
:10B680009AE700BF5C2C070839800008D3B2012B71
:10B690001DD8104B02EB420210B54FEA820E0EF19C
:10B6A000080403F5137C02E01C3363450DD01A78BF
:10B6B0008242F9D15A788A42F6D11A59002AF3D037
:10B6C0000EF1040E03EB0E0010BD002010BD002093
:10B6D000704700BF842C070810B40C4C002304F6FC
:10B6E000840C01E0152B0CD003EB430201331CF852
:10B6F00002108142F6D1144494F986085DF8044B97
:10B7000070474FF0FF305DF8044B7047281C002055
:10B71000D3B2022B22D870B502EB4202104C4FEA92
:10B72000820E23460EF10C05002204E00132172A96
:10B7300003F12C0310D01E68B042F7D193F804C077
:10B740008C45F3D15E59002EF0D02C210EF1080368
:10B7500001FB0233E01870BD002070BD002070476F
:10B76000181E0708002839D030B51D4D90F804C0C8
:10B77000002305F6840401E0152B2DD003EB4302D2
:10B780000133A15C6145F7D11544046895F9863809
:10B7900090F805E0DAB2022A1ED803EB4303114801
:10B7A0004FEA830C0CF10C050346002204E0013241
:10B7B000172A03F12C030FD019688C42F7D119799D
:10B7C0007145F4D159590029F1D02C210CF108030D
:10B7D00001FB0233184430BD002030BD704700BF6C
:10B7E000281C0020181E07080348D0F8483113B160
:10B7F00000F59C7018477047880100200348D0F876
:10B800006C3113B100F5AE70184770478801002005
:10B810000348D0F8903113B100F5C0701847704755
:10B82000880100200348D0F8B43113B100F5D2707C
:10B8300018477047880100200348D0F8D83113B169
:10B8400000F5E47018477047880100200348D0F8DD
:10B85000FC3113B100F5F6701847704788010020DD
:10B860000348D0F8203213B100F504701847704730
:10B87000880100200348D0F8443213B100F50D7060
:10B8800018477047880100200348D0F8683213B188
:10B8900000F5167018477047880100200348D0F85B
:10B8A0008C3213B100F51F701847704788010020D3
:10B8B0000348D0F8B03213B100F52870184770472C
:10B8C000880100200348D0F8D43213B100F531705C
:10B8D00018477047880100200348D0F8F83213B1A8
:10B8E00000F53A7018477047880100200348D0F8E7
:10B8F0001C3313B100F543701847704788010020CE
:10B900000348D0F8403313B100F54C701847704726
:10B91000880100200348D0F8643313B100F5557056
:10B920001847704788010020094B0A4A013800EB8C
:10B93000C00003EB80030848D3F83831116B834211
:10B9400014BF4FF480034FF400130B43136370478D
:10B95000880100200038024000600240F0B4013845
:10B960003B4C3C4E3C4D00EBC00C04EB8C0CDCF82B
:10B970003871AF4214BF4FF480054FF40015376B98
:10B980003D433563354DCCF85031DCF83C31CCF8D3
:10B990004811AB424FEAC0013FD005F58065AB428C
:10B9A0003BD0A5F57A75AB4246D005F58065AB4234
:10B9B00042D0A5F57A75AB4240D005F58065AB4223
:10B9C0003CD0A5F57A75AB4234D005F58065AB4225
:10B9D00030D0A5F57A75AB4232D005F58065AB4223
:10B9E0002ED0A5F57A75AB422CD005F58065AB421B
:10B9F00028D0A5F57A75AB4226D005F58065AB4217
:10BA000022D0A5F57A75AB4220D0154D06F53256F9
:10BA10003836B34218BF002500E0124D0B1804EB76
:10BA20008304C2F3871194F84D01C4F85851F0BC57
:10BA300060F094BB0C4DF1E70C4DEFE70C4DEDE7DA
:10BA40000C4DEBE70C4DE9E70C4DE7E7044DE5E75E
:10BA5000880100200038024000600240106002406F
:10BA6000008000282080001000800018008800104E
:10BA700000802010208000200088002000802020EE
:10BA80002DE9F04F934A92F8D538012B85B021D09B
:10BA9000022B15D0002300938F4F4FF0000807F1C1
:10BAA000780A3B78022B17D008F10108B8F1030F90
:10BAB00007F128070AF1050AF3D105B0BDE8F08FB8
:10BAC00092F8CA3833B192F8C638083B18BF012340
:10BAD0000093E1E70093DFE79AF903307F4D029787
:10BAE000591C15BFDBB200239B464FF0010B1E46CD
:10BAF000DAB2012A00F2DB8006EB4601890073000E
:10BB0000774C019308315FFA88F703E01C34AC42AC
:10BB100000F0CD802378002BF8D16378BB42F5D1BB
:10BB200060580028F2D011F017F9009B814623B12C
:10BB3000A0F10901072940F2BF807A1CD2B214217A
:10BB4000484611F0F5F8002800F0B180DDE9013732
:10BB5000334404EB830409F1FF33E068614C59423C
:10BB600003EBC30201F0070103F0070358BF4B4288
:10BB700004EB820104F59C7404EB8202C1F84401D9
:10BB80003A61484681F84031FFF7CEFE9AF9043019
:10BB90005A1C00F09A80DEB23246CDE902974F4D32
:10BBA000F3B29346012B62D806EB4601890073007D
:10BBB0004B4C019308315FFA88F902E01C34AC4227
:10BBC00055D02378012BF9D163784B45F6D16058D5
:10BBD0000028F3D011F0C0F8009B07461BB1A0F17C
:10BBE0000901072947D909F10102D2B213213846C8
:10BBF00011F09EF800283AD0019ADDF808903244FE
:10BC0000BB4604EB82040BF1FF325142E068354C35
:10BC1000039F02EBC20501F0070102F0070258BFC3
:10BC20004A4204EB850104F59C7404EB8505C1F8D8
:10BC300044017D61584681F84021FFF775FEB9F156
:10BC4000000F3DD0BBF1000F1BD02846FCF71AFCBB
:10BC50003869FCF717FC3846FCF7E4FB00231A466A
:10BC600021495846FFF77AFE01233B731CE7013652
:10BC7000F3B29B4596D2DDE90297B9F1000F1FD0D0
:10BC80001A4C09F1FF33242202FB034000243861DF
:10BC90007C61FCF7F7FB3846FCF7C4FB23461449EC
:10BCA00022464846FFF75AFE01233B73FCE6013665
:10BCB000F2B25A457FF61DAF029F4FF0000965E7CB
:10BCC00000220023C7E90423EEE601231A460026DA
:10BCD00063E700BF281C002018250020D02E07088D
:10BCE000842C070888010020959D0008C0020020D0
:10BCF0000D9E00080C4A0D4903469342D1F8F4000A
:10BD000010D0A2F5806293420CD002F5804293429B
:10BD100008D002F58062934204D002F5806293421B
:10BD200018BF4008704700BF00040140281C0020D5
:10BD3000800AA0F58010522808D8054B034493F8D8
:10BD400000340D2B02D8034AD056704700207047AC
:10BD5000181E070828C10708064A136851690B40D6
:10BD600003F00103536123B1034BD3F80C070368BD
:10BD700018477047003C0140281C0020064A136801
:10BD800051690B4003F00203536123B1034BD3F815
:10BD90001007036818477047003C0140281C00202A
:10BDA000064A136851690B4003F00403536123B141
:10BDB000034BD3F81407036818477047003C014051
:10BDC000281C0020064A136851690B4003F0080341
:10BDD000536123B1034BD3F8180703681847704722
:10BDE000003C0140281C0020064A136851690B40A2
:10BDF00003F01003536123B1034BD3F81C0703680E
:10BE000018477047003C0140281C0020F8B50C4B37
:10BE10001D685A69154005F478755D617DB1094F5B
:10BE20000126B5FA85F4C4F11F0407EB840306FA72
:10BE300004F4D3F80C0703689847A543F1D1F8BD83
:10BE4000003C0140281C0020F8B50C4B1D685A69C5
:10BE5000154005F47C455D617DB1094F0126B5FAB9
:10BE600085F4C4F11F0407EB840306FA04F4D3F845
:10BE70000C0703689847A543F1D1F8BD003C014089
:10BE8000281C0020F0B5054683B0A0B307681D4B01
:10BE9000144607F13F4202F57E0203EB92230E4661
:10BEA00093F8A40460F03CF9A988B1FA81F3C3F1D6
:10BEB0001F03C3F3CC0207EB820203F00703156AEA
:10BEC0004FF00F0C9B009C400CFA03F325EA030390
:10BED0001362136A1C431462C6F30013C6F34112C3
:10BEE000CDE900323846C6F3810306F0030261F063
:10BEF00005FB03B0F0BD034B93F8A30460F010F909
:10BF00002B68FFDE181E070800B1BBE7704700BFB3
:10BF10002DE9F047684E06EB0013D3F87849002C62
:10BF200076D093F8807905464FEA0018384660F0DD
:10BF3000F7F807F01F027F090123032F03FA02F32A
:10BF400072D0042F6BD0022F64D006EB08030135AA
:10BF500093F87C09FFF722F8EDB2824610B1122364
:10BF6000C571837106EB080393F87D09FFF716F896
:10BF7000814610B11323C571837106EB080393F852
:10BF80007E09FFF70BF8074610B11423C5718371C2
:10BF900006EB0803504693F87F594A212A46FFF7DB
:10BFA000B3FF2A4648462A21FFF7AEFF2A460A2158
:10BFB0003846FFF7A9FF414B9C423AD0404B9C4288
:10BFC00042D0404B9C424AD03F4B9C4252D03F4BC8
:10BFD0009C425AD03E4B9C4262D0A38823F003037C
:10BFE0001B041B0CA380238803F4415343F44573C3
:10BFF00043F003032380A38B23F400631B041B0C77
:10C000000722A383228223889BB243F0400323802C
:10C01000BDE8F0872F4A516A0B43536295E72D4ADA
:10C0200011690B43136190E72A4A116A0B431362AB
:10C030008BE703F584335A6A42F480525A625A6A93
:10C0400022F480525A62C8E703F500331A6A42F4B8
:10C0500080421A621A6A22F480421A62BDE703F52E
:10C06000FE331A6A42F400421A621A6A22F400424B
:10C070001A62B2E703F582335A6A42F400525A62F6
:10C080005A6A22F400525A62A7E703F568435A6AD3
:10C0900042F480125A625A6A22F480125A629CE771
:10C0A00003F564435A6A42F400125A625A6A22F44F
:10C0B00000125A6291E700BF281C002000300140A6
:10C0C00000380040003C0040003401400050014076
:10C0D0000054014000380240431C00F057812DE914
:10C0E000F04FDFF880A400EB80030AEBC30287B0B7
:10C0F000D2F80C90810005460191DB00B9F1000FE8
:10C1000007D0D2E90548002C00F00C8194F90620F4
:10C1100012B107B0BDE8F08FB8F1000F00F06081F8
:10C1200098F90620002AF4D118330AF10C06F01809
:10C13000D9F80470F250691CC0E901221523C260CD
:10C14000C9B2A3711623E17188F8071088F8063088
:10C1500099F828005FF0E4FFBB882268A08823F4E8
:10C1600040731B041B0CBB80D8F800301083B8F858
:10C1700004201A8311212046FEF73EFE112140467D
:10C18000FEF73AFE09264FF0330B2CB9F5E0BBF170
:10C19000010B08D0FEF724FD2268A188136919421B
:10C1A0004FF00A00F3D051830520FEF719FD2368F4
:10C1B000A2881A830520FEF713FD013EE3D1002C6F
:10C1C00000F03081332603E0013E08D0FEF708FD81
:10C1D0002268A188136919424FF00A00F4D05183F4
:10C1E0000520FEF7FDFCB8F1000F00F04881D8F8FB
:10C1F0000030B8F804205A830520FEF7F1FC2368CC
:10C20000A2881A830520FEF7EBFCD8F80030B8F8B6
:10C2100004201A830520FEF7E3FC2368A2881B692B
:10C220001A4240F0B480019B2B440AEBC303997F70
:10C230001A7F002940F0B78020461221FFF722FE26
:10C240001221019B2B440AEBC3035A7F4046FFF7A0
:10C2500019FEBE4B9F4200F03081BD4B9F4200F063
:10C260003781BC4B9F4200F04481019B2B440AEB79
:10C27000C3034FF47A721C8CBB8823F440731B04F5
:10C280001B0CBB803B889BB243F001033B80BD8805
:10C2900002A802FB04F425F03F0558F067FA049960
:10C2A000AD4B2D04A3FB01232D0C45EA9345BD8026
:10C2B0003A8822F001021204120C3A80A74A980C24
:10C2C0009442034675DC6200B1FBF2F292B2013394
:10C2D000042A38BF04223B84BA833B889BB243F0D4
:10C2E00001033B803B8823F4816323F002031B049A
:10C2F0001B0C4FF4804243F480633B803A813B88BF
:10C3000023F080031B041B0C3B8099F82A000021BA
:10C310005FF024FF99F82900002107B0BDE8F04F35
:10C320005FF01CBFB8F1000F00F0F88098F906200C
:10C33000002A7FF4EEAE18330AF10C01CA18D9F8BE
:10C340000470CC50C2E901441623D46088F806304A
:10C350006B1C88F8073099F828005FF0E1FEBB8875
:10C36000B8F8042023F440731B041B0CBB80D8F8DE
:10C3700000301A8302E7FEF733FCBBF1010B4FF0EC
:10C380000A00F8D10520FEF72BFC13E77047019B4C
:10C39000D8F800202B440AEBC30312699A7F002AC5
:10C3A00000F0A1801A7F32212046FFF76BFD322179
:10C3B00047E704EB4404B1FBF4F18AB2C1F30B018B
:10C3C00009B942F0010266494FF4967300FB03F38A
:10C3D000A1FB03139B09013342F400423B847BE73A
:10C3E0000AF10C011833CA18D9F8047041F8038017
:10C3F000C2E901881523C2F80C80A371431CE371C4
:10C4000099F828005FF08CFEBB88A28823F4407363
:10C410001B041B0CBB80236811211A832046FEF7E6
:10C42000EBFCAFE6332401E0FEF7DAFB013C4FF012
:10C430000A00F9D10520FEF7D3FBB8F1000F63D055
:10C44000D8F80030B8F804205A830520FEF7C8FB5E
:10C450000520FEF7C5FBD8F80030B8F804201A8391
:10C460000520FEF7BDFB019B2B440AEBC3039A7F1B
:10C47000002A18BF32215A7F08BF1221E6E60520A4
:10C48000FEF7AEFB2368A2881A830520FEF7A8FBFF
:10C490000520FEF7A5FB2368A2881B691A4263D119
:10C4A000019B2B440AEBC303997F1A7F00296AD0B2
:10C4B00020463221FFF7E6FCCBE603F5F2331A6A99
:10C4C00042F400121A621A6A22F400121A62CCE6CE
:10C4D00003F5F0331A6A42F480021A621A6A22F4EF
:10C4E00080021A62C1E61A7F20461221FFF7CAFCB9
:10C4F000A6E603F5EE331A6A42F400021A621A6ADB
:10C5000022F400021A62B0E60520FEF769FB05205E
:10C51000FEF766FB0520FEF763FB9AE618330AF187
:10C520000C01CA18D9F8047041F80380C2E90188E7
:10C53000C2F80C8099F828005FF0F2FDBB8823F464
:10C5400040731B041B0CBB801CE600BF0054004062
:10C5500000580040005C004083DE1B43A0860100C1
:10C56000D34D6210281C0020019B2B440AEBC3030F
:10C5700020469A7F002A18BF32211A7F08BF122155
:10C58000FFF780FC65E620461221FFF77BFC60E6A2
:10C590002DE9F8430746FDF789FFDFF84C8007EBEC
:10C5A0008709044608EBC90542F20F7604E0FDF75F
:10C5B0007DFF001BB0420BDC95F82530002BF6D137
:10C5C00008EBC90898F8240080F00100BDE8F88362
:10C5D000B8F8A839013338469BB2A8F8A839FFF754
:10C5E0007BFD0020BDE8F883281C002010B582B038
:10C5F00004468DF807300DF107035EF083F808B9A3
:10C6000002B010BD2046FFF7C3FF02B010BD00BF4F
:10C61000B0F1FF3F6DD02DE9F04F022883B0044602
:10C6200014DC354E984600EB800306EBC305DB00B7
:10C63000D5F810A00093BAF1000F07D0894695F8FD
:10C640002510934601F0FF02019219B1002003B0BA
:10C65000BDE8F08FFDF72AFF009B019A20330746C3
:10C660004FEA490106F10C00C9B200EB030C85F852
:10C6700026104FF0010E0C9985F827B085F8292077
:10C6800085F82AE0C150CCF8041085F8288085F898
:10C6900025E085F82420BAF8043099051DD4BAF8AD
:10C6A0000030DA0512D442F20F7504E0FDF7FEFE09
:10C6B000C31BAB4213DCBAF800309B05F6D4BAF8C2
:10C6C00000309BB243F48073AAF80030BAF804300B
:10C6D0009BB243F44073AAF804300120B7E7B6F8E0
:10C6E000A83901339BB22046A6F8A839FFF7F4FC1D
:10C6F000ACE70020704700BF281C0020E0B5294EA1
:10C7000000EB800306EBC30384B0DA685568AA8A9D
:10C7100092B20392039A12F4706F1CBF012283F845
:10C720002420039B13F4E06F4FEA80070DD1AB8AFE
:10C73000074423F4706306EBC7061B041B0C00229E
:10C74000AB8286F8252004B0E0BD2B8BAB8823F4A8
:10C7500080631B041B0CAB80039B9A05E7D42B88DA
:10C760009B05E4D42B88D9050FD52B88DA05FCD49A
:10C770002B889BB243F400732B802B889B05FCD441
:10C780000190FFF7A9FC0198D1E72B889BB243F4F5
:10C7900000732B80AB8823F440731B041B0CAB800D
:10C7A000C5E700BF281C00200020A7E70120A5E75F
:10C7B0000220A3E770B590F871301C09013C052CEC
:10C7C0000FD81A4E06EB44020546B2F8F40303F004
:10C7D0000F0340FA03F2D20703D595F87220012A1D
:10C7E00001D0012070BD9A40013A1040264465F006
:10C7F0006BF996F83C3E0E4A034402EBC30452F830
:10C800003320A38810691840ECD0EB6E002285F825
:10C81000722093F8212002212046FFF733FB2A6E75
:10C8200093899BB243F008039381DAE7181E070847
:10C83000201D0020F8B50E4C94F8C8759FB104F582
:10C84000BA64C7F109070925013D0ED0A668307901
:10C85000FEF7A4FB217DF27908B1FFF713FBAF428D
:10C8600004F18C04F0D10120F8BDAB68FFDE00BFFD
:10C8700004000010094BD3F8AC29D3F8B01940F2EA
:10C880002A40002350604B620B889BB243F00103A7
:10C890000B80136843F0010313607047281C0020CD
:10C8A00010B41D4B1D48196C1D4A41F080510124E4
:10C8B00085B0196404625321FF24CA205462506277
:10C8C00051625B6FDB0017D41648042300210291EC
:10C8D0000290029A1A440292029A04331C2B1160AD
:10C8E000F5D103910390039B0393039B0E4A1A60B7
:10C8F00005B05DF8044B70470A4B0022019201938A
:10C90000019B0193019A084B12689A42DCD105B051
:10C910005DF8044B704700BF0038024000000E4233
:10C920000028004050280040316665422DE9F04162
:10C93000046ED0F80880A38923F400531B04074633
:10C940001B0C90B0A38143793D79C3F38000190398
:10C9500005F001061B0215F002054FEA00304FEA10
:10C96000860203F4806318BF42F0080203431A43AF
:10C97000238A9BB201F4005123F440530B432382DA
:10C98000A38923F4B05323F00C031B041B0C1A439C
:10C99000A281A38A23F440731B041B0CA38201A869
:10C9A00057F0E4FE6B4B9C4205D003F580639C423C
:10C9B00001D0039B00E0049BA2896749A08912046F
:10C9C00003EB83034CBF4FEA48084FEA880803EBA8
:10C9D0008303B3FBF8F3A1FB03C252094FF0640CCD
:10C9E00000040CFB12334FEA021200F19A801B0183
:10C9F0003233A1FB0313C3F3431313439BB22381CD
:10CA000097F9380097F80580FEF7F0FA30B103681F
:10CA1000828818F0010F14BF1A835A8318F0080F88
:10CA2000A38A78D09BB243F00803A382A3899BB268
:10CA300043F40053A381002E2FD0FE6B002E7DD037
:10CA40000023CDE90833CDE90C33CDE90E3304934F
:10CA500006937B6C0193FB6D0293FB6805937B69E6
:10CA600003934FF480714FF48033CDE90A133046BD
:10CA70004FF48063079357F0C5FE01A9304656F086
:10CA800025FA336843F001033360A38A9BB243F075
:10CA90004003A38273689BB27B65002D33D03E6C4C
:10CAA000002E46D0BB6C0193BB6D02933B6905938E
:10CAB000402304934FF48033002530460B934FF40A
:10CAC00080630793CDE90855CDE90C55CDE90E55A6
:10CAD000039506950A9557F095FE01A9304656F044
:10CAE000F5F9736943F080037361336843F016030B
:10CAF00033607560A38A9BB243F08003A382E3682E
:10CB000043F04003E360A3899BB243F40053A38145
:10CB100010B0BDE8F08123F008031B041B0CA382B6
:10CB200084E7DB003233A1FB0313C3F34213134347
:10CB300064E7E36843F08003E360E0E74FF6DF7308
:10CB40002380E36843F02003E360E36843F01003CD
:10CB5000E360A2E7001001401F85EB51BFF34F8F48
:10CB60000549064BCA6802F4E0621343CB60BFF389
:10CB70004F8F00BFFDE700BF00ED00E00400FA05A5
:10CB800008B50021032057F027FF72B6FFF7E6FF34
:10CB9000154C08B5D4F8B43994F8BA09ABB91420D7
:10CBA000FEF7AEF800BFD4F8B4395BB11A689B88C1
:10CBB000116994F8BA290B4012B91BB1FFF7E0FFD5
:10CBC000002BFBD0FCF7CEFCECE719689A880B69C8
:10CBD000134020B1002BE2D10B691340FAE7002B80
:10CBE000DDD00B691340FAE7281C002008B572B6A7
:10CBF000FFF7B4FF00B583B00D4900220092009109
:10CC0000009B0C330093009B1B68012B02D003B0E8
:10CC10005DF804FB01920191019B06490C330193DD
:10CC2000019B1A600B6883F308884B689847FEE7FE
:10CC3000502800400000FF1F38B5FFF731FEFFF716
:10CC4000D9FF012057F0D8FE6E4A936823F0030302
:10CC50009360936813F00C0FFBD113686949A0B976
:10CC600043F00103136041F2883302E0013B00F01E
:10CC7000C7800A689507F9D5634C00220823C4F8D9
:10CC8000BC29C4F8C03902251EE043F48033136088
:10CC900041F2883302E0013B00F0B2800A6894035D
:10CCA000F9D5594C594B5A4DB0FBF5F5B0FBF3F0A3
:10CCB000B5EB400F18BF28464FF48003C4F8BC39C9
:10CCC000C4F8C009B5FBF0F50220C4F8C45957F008
:10CCD00093FE03280DD84F4B03EBC0039988DA88E5
:10CCE000C4F8CC195B88C4F8D029B3FBF5F3C4F8B9
:10CCF000C839444B48491A6C42F080521A640A6899
:10CD000042F440420A609A689A609A6842F400428B
:10CD10009A609A6842F4A0529A60D4F8BC19D4F888
:10CD2000C0290A43D4F8C81942EA8112D4F8D019AC
:10CD300042EA0162D4F8CC194908013942EA0142B9
:10CD40005A601A6842F080721A601A689201FCD523
:10CD5000324A40F205711160996821F0030199602F
:10CD6000996841F00201A2F580629960936803F02E
:10CD70000C03082BFAD12A49D823B3FBF5F39B0106
:10CD800043F000530120C2F884308866FBF766FE4A
:10CD9000244D1C4B244AEA60596F244AC4F8D41924
:10CDA000AA605A6B224922F080025A635A6F42F0FD
:10CDB00080725A671A6B42F4CE021A635A6B5A6336
:10CDC0009A6B9A631A6C0A431A64596C194A0A439B
:10CDD0005A64FCF735FC184AD4F8F430A2FB03235C
:10CDE0009B09013BB3F1807F09D24FF0E022F02094
:10CDF00053610021072385F823009161136138BD39
:10CE0000014CC5E700380240281C002080841E0029
:10CE100040420F00D02E070800700040003C024046
:10CE20000000474200ED00E00005FA050000002088
:10CE3000FFC9FE36335F0700D34D621030B5154C85
:10CE4000154D85B00139002389B2A042ADF80C30F0
:10CE5000ADF806308DF80E300291D5F8F4300FD0D1
:10CE60000E4988420CD001F58041884208D001F576
:10CE70008061884204D001F58061884218BF5B0858
:10CE8000B3FBF2F301A9013BADF8043057F0A8FE63
:10CE900005B030BD00040140281C00200000014006
:10CEA00030B504682A482B4D85B00139002389B27A
:10CEB0008442ADF80C30ADF806308DF80E3002919A
:10CEC000D5F8F4300FD024498C420CD001F58041C4
:10CED0008C4208D001F580618C4204D001F580615C
:10CEE0008C4218BF5B08B3FBF2F301A9013B20465B
:10CEF000ADF8043057F074FE2288184892B242F020
:10CF00000102002300F63451228051F8332094426C
:10CF100008D001330E2BF8D1002005B0BDE8304019
:10CF2000FBF7A2BC00EBC30090F8394D2046FBF79D
:10CF30009BFC1B2C05D02E2C08BF2C20EDD005B05F
:10CF400030BD192005B0BDE83040FBF78DBC00BFF7
:10CF500000040140281C002000000140181E0708A2
:10CF600070B50468A30AA3F58013522B50D8364D30
:10CF70002B4493F800C4BCF10D0F49D8437902202B
:10CF800023FA00F50CEB8C03A8400CEB43031FFACB
:10CF900080FE2B44002949D0A5892C48ADB200EB76
:10CFA000830645EA0E05C6F8FC13C6F80C24A581D5
:10CFB000EFF31186502383F312882C2202FB0C031B
:10CFC000D3F8F81361B3C3F81C14214B04310CEBF4
:10CFD0008C02204D0CEB4202920005EB020E103247
:10CFE000134453F8042F0AB10A60111D7345F8D198
:10CFF0000022F3B20A6083F311882C2303FB0C0098
:10D00000D0F81C342BB1A3899BB243F00103A38158
:10D0100070BDA38923F001031B041B0CA38170BD09
:10D020000B4B02FB0C3202F12401D0E7A08980B245
:10D0300020EA0E00A081054800EB8305C5F8FC132B
:10D04000C5F80C24B4E700BF181E0708281C0020F0
:10D05000202000204020002001490248FCF7AABC03
:10D06000202000200000014010B5064C064804F5C1
:10D070007E71FCF79FFC04F284510448BDE8104027
:10D08000FCF798BC281C002000000140004401402F
:10D0900002494FF08040FCF78DBC00BF4C200020BF
:10D0A00001490248FCF786BC7820002000040040BB
:10D0B00001490248FCF77EBCA42000200008004083
:10D0C00001490248FCF776BCD0200020000C00404B
:10D0D00001490248FCF76EBC5421002000040140C5
:10D0E00010B5064C064804F22C51FCF763FC04F51D
:10D0F000C1610448BDE81040FCF75CBC281C00205E
:10D1000000040140001C004001490248FCF752BCE9
:10D11000802100200040014001490248FCF74ABC40
:10D12000D82100200048014001490248FCF742BCD8
:10D13000042200200018004001490248FCF73ABCD4
:10D140005C2200200020004010B50C2935D8DFE813
:10D1500001F09134343463343434073434343500DA
:10D16000038C5488B2F80CE023F480731B041B0C6E
:10D170000384038CB0F804C0818B21F073014EEA64
:10D18000040E0904148823F40073090C1B042143C2
:10D19000764C1B0C43EA0E23A0421FFA8CFC9BB278
:10D1A00000F0948004F58064A04200F08F809268C3
:10D1B000A0F804C08183C263038410BD038C54882B
:10D1C000B2F80CE023F480531B041B0C0384038C83
:10D1D000B0F804C0818B21F4E6414EEA040E090444
:10D1E000148823F40053090C41EA04211B045F4C0A
:10D1F0001B0C43EA0E33A0421FFA8CFC9BB289B28F
:10D200007ED004F58064A0427AD09268A0F804C071
:10D2100081830264038410BD038C5488B2F80CE04F
:10D2200023F010031B041B0C0384038CB0F804C010
:10D23000018B21F4E6414EEA040E0904148823F020
:10D240002003090C41EA04211B04484C1B0C43EA4F
:10D250000E13A0421FFA8CFC9BB289B26CD004F56D
:10D260008064A04268D09268A0F804C00183826301
:10D27000038410BD038C5488B2F80CE023F0010342
:10D280001B041B0C0384038CB0F804C0018B21F039
:10D2900073014EEA040E0904148823F00203090CFA
:10D2A0001B042143314C1B0C43EA0E03A0421FFA1E
:10D2B0008CFC9BB22CD004F58064A04228D09268EC
:10D2C000A0F804C001834263038410BDD489B2F87E
:10D2D00010E023F4006343EA0423548A2CF4405CF6
:10D2E0004EEA040E4CEA0E1C94884FF6FF3E03EA09
:10D2F0000E0E4EEA042E1FFA8CFC1FFA8EF356E730
:10D30000148A2CF4804C4CEA841C1FFA8CFC7CE7B9
:10D31000D489B2F810E023F008032343548A2CF494
:10D32000407C4EEA040E948823F004034CEA0E0C71
:10D330001FFA8CFC2343C2E7D489B2F810E023F033
:10D34000800343EA0413548A2CF4406C4EEA040E22
:10D350004CEA8E0C94884FF6BF7E03EA0E0E4EEA1E
:10D36000041E1FFA8CFC1FFA8EF37CE700000140BC
:10D370002DE9F04FB14BDFF8DC8293F8D6E8B04CE2
:10D38000B04D93B00EF1FF37FBB200930023CDE90F
:10D39000013EC246DFF8C0B2DBF80070BB0AA3F55D
:10D3A0008013522B00F20B81234493F800340D2B91
:10D3B00000F2058115F90390029B012B00F0068114
:10D3C000029B022B02D1B9F1080F33D1002631465E
:10D3D000484612F0B9FA12F043FB90F9003013B14D
:10D3E000542B40F0EB820436B6B2102EEFD1019BE5
:10D3F0000021002B00F0A38042460CE0234493F868
:10D4000000340D2B0ED8EB564B450ED002F5807232
:10D41000524500F09180906803689B0AA3F5801341
:10D42000522BEBD900234B45F0D143799BF80500F3
:10D430009842EBD1844B0BF11C0B9B45ACD1019B6B
:10D440000133042B01930AF5807AA3D1DFF80C9203
:10D4500099F8C835013309F5816A04934FF0010B3F
:10D46000049B5B4565D0DAF80C30744A9AF81010CA
:10D4700092F8D82901930291002B5AD01968D9F853
:10D4800004009B88039101F13F4505F57E050028C6
:10D490004FEA9525009340F3A780002303E0013372
:10D4A000834200F09E801C0258F80410A942F6D175
:10D4B0004444009A029B8AF81030B2FA82F6019B2B
:10D4C000CAF80C30C6F11F054FF00301CAF804502A
:10D4D000CAF81840997183F807B0E16C606C6B0072
:10D4E000012203279F4002FA03F3194399F8003001
:10D4F000E164384302FA05F56064276DD4F8A000B2
:10D50000A9B2002B00F060823D432565039D009B7E
:10D510002B83FBF707F820460BF1010BFBF748F9CB
:10D5200040F20113BBF1090FAAF81C300AF1200ADE
:10D5300096D113B0BDE8F08F00297FF47BAF584639
:10D54000FAF7B6FFC3B2022B9BF805E000F2778230
:10D5500000F1010C3A4A0CEB4C0C4FEA8C0C02F532
:10D560007D7003E02C32904200F0698213689F4284
:10D57000F8D113797345F5D152F80C30002BF1D066
:10D58000324842689A424FF0000108D00131102918
:10D5900000F124003FF44EAF42689A42F6D14B1C92
:10D5A000DBB22B4A013B03EBC30302EB830393F98A
:10D5B0005431002B7FF43EAFCAF808B03FE7009B20
:10D5C000012B7FF637AF4FF00009FFE6B9F1010FED
:10D5D0003FF4FCAE1C4B0BF11C0B9B457FF4DCAE07
:10D5E0002DE7042B00F0FC8109EB002301020591DB
:10D5F00019690691002900F016826C1C0792E4B2AA
:10D600004FF054029D6083F8042183F80541069B86
:10D6100001305E79C9F8040018461D680896FAF7CB
:10D6200047FFC3B2022B00F20A82471C07EB4707F1
:10D63000034B079ABF000021B44617E0281C0020C6
:10D64000181E070828C10708EC2F0708C002002091
:10D65000880100200C000010F02E070804000010C4
:10D660000131172903F12C0300F0E9811E68B5424E
:10D67000F6D11E796645F3D1DE59002EF0D02C2369
:10D6800000EB400001FB03F3BB49BC4F03EB8003FD
:10D690000B4438461969059B0A914B44C3E906615E
:10D6A0004368B3424FF0000108D00131102900F166
:10D6B00024003FF43EAF4368B342F6D14B1CDBB2CB
:10D6C000AF49013B03EBC30301EB830393F954110F
:10D6D00000297FF42EAF83F85541059CA948E1113C
:10D6E00001EB242101EB011100EB810C0599CDF830
:10D6F0001CC08C24091204FB01F100F54C7000EBF6
:10D7000041000599099049440998C1F8F440039CE7
:10D71000CC605424C1F8F00083F854419A48C1F811
:10D72000A8C03323C1F8AC30984B0599D3F8F43036
:10D73000854208EB01040FD095498D420CD001F5CC
:10D7400080418D4208D001F580618D4204D001F501
:10D7500080618D4218BF5B08062A00F06181072AAC
:10D760008C488D4A8D4918BF11468D4A18BF024614
:10D770000598B3FBF2F2B3FBF1F3013A09EB0001B8
:10D7800092B2013BA1F8B030A1F8682000F1540139
:10D790000023A4F85C30284648F80130A2654144D3
:10D7A00057F01EFA0023ADF838302B8808999BB249
:10D7B00043F080032B802B8823F001031B041B0CF8
:10D7C0002B80784B0D934FF0020E4FF48073CDE910
:10D7D00010E328460A230DAA0F93FFF7B5FC069B1A
:10D7E0001879002840F006812B889BB243F0010392
:10D7F0002B8000237A68964203F1010300F0F78042
:10D80000102B07F12407F5D14FF0FF3300205C4ABD
:10D810006549664F03EBC30302EB8303644AD3F805
:10D8200038318B4214BF4FF480034FF40013116B57
:10D830000B431363089A0C2A9BBF5E4B03EB420316
:10D840000021B3F8DC10059B4B449982002306E0CD
:10D85000954200F0EF800133042B00F0ED8057F883
:10D860003320002AF4D1D9F8F02E0132C9F8F02E75
:10D8700009EBC302DB00C2F8F45E3B4400259A8842
:10D880001143998090224C492346FEF767F833688C
:10D89000059A039843F010033360079BE3660A9BE5
:10D8A000636602F1640104234FF40032C4E92323C8
:10D8B00040233322C4E91C3200F118024FF4806780
:10D8C000A2664FF480504FF48042C4E920024144E4
:10D8D0003046C4E92555A567C4F88850C4F89C5063
:10D8E000E76755F0F3FA3068E061706920627068AC
:10D8F0000A9B6062B068A062F068C4F8AC30042390
:10D90000C4F8D830099BE062C4F8B4300398059A93
:10D91000C4F8C4704FF44033C4F8D4308C23C4F836
:10D92000BC3000F1100302F1AC01C4F8B0304FF488
:10D9300080424FF40063C4F8C830C4E9375541440D
:10D94000C4F8CC20C4F8B850C4F8C050C4F8D050C3
:10D95000C4F8E450304655F0B9FA3368236373696C
:10D9600063637368A363B368E363F3682364336832
:10D9700043F0100333609CE5181E0708C002002026
:10D98000880100200426002000040140281C0020FB
:10D9900000000140D0DD060044950800105522002B
:10D9A00040771B006000010000600240F80E00108C
:10D9B00000380240102F07086D850008019B0121E7
:10D9C000002B7FF419AD35E5C6F12F06B2403A437E
:10D9D0002265039A009D55831A46FAF7A3FD9AE53E
:10D9E000184A032382F8D93913B0BDE8F08FD8B2B2
:10D9F000431E0CE7FDF7D2FA0B9038B1069B0221CB
:10DA0000DA79FEF73FFA0B9B5422DA80B5F84430FE
:10DA10006FEA43436FEA53439BB2A5F84430E3E611
:10DA200009490A4AA4E6074A022382F8D93913B001
:10DA3000BDE8F08FDB0020E700239B88FFDE00239A
:10DA40005B68FFDE281C0020882A1100A0BB0D00A7
:10DA50000C2911D8DFE801F0231010101910101054
:10DA6000111010100700838B23F400631B041B0CA0
:10DA700043EA02239BB283837047838B23F008031E
:10DA80001B041B0C1A4382837047038B23F400632F
:10DA90001B041B0C43EA02239BB203837047038BD6
:10DAA00023F008031B041B0C1A430283704700BFBA
:10DAB0002DE9F04FDFF85CB39BF874709BB01FB991
:10DAC00000201BB0BDE8F08F00222F21384612F055
:10DAD0001BF880460028F3D0DFF83C930568C9F8AE
:10DAE000B059FDF73FFE0028EAD0D0E90143019389
:10DAF000C9F8AC49002CE3D0BA4E0022314601E00F
:10DB0000102ADDD04868844201F1240102F10102AB
:10DB1000F6D1D2B2DFF804A3013A02EBC2020AEB5B
:10DB2000820292F954110029CAD138462F27A2F84F
:10DB30005471FDF733FACBF8780028B1C78098F814
:10DB400007202A21FEF79EF9A74F002207F634503E
:10DB500050F832108D4200F0128101320E2AF7D1B6
:10DB600000205EF0DDFA2988D9F8F42021F00101C7
:10DB70000904090C29809D498D4200F0E880A1F537
:10DB800080618D4200F0E38001F580418D4200F01C
:10DB9000DE8001F580618D4200F0D98001F5806161
:10DBA0008D42934900F00A81B1EB520F4FEA5200C7
:10DBB00040F2F88001220021B0FBF2F2ADF80C1027
:10DBC0008C498D48120AA1FB02121109A0FB010128
:10DBD0004908ABF87E10490000271209ABF87C1009
:10DBE000284603A90492ADF81470ADF80E708DF8B4
:10DBF000167056F0F5FF98F80630ADF81C706022EC
:10DC000006929A07CDE908770A9798F8057040F1CF
:10DC1000A380DB0003F008034FF00408ADF82630C2
:10DC2000ADF81C8006AA39462846FFF78DFA08226F
:10DC30003946FFF70DFFB5F844206FEA42426FEA1C
:10DC4000524292B2A5F844202A8892B242F0800251
:10DC50002A802A8C08FA07F39BB292B222EA0302C6
:10DC60002A842A8C92B213432B842B889BB243F0D4
:10DC700001032B803246002351688C4202F12402BA
:10DC800003F1010376D0102BF6D14FF0FF3303EBF5
:10DC9000C3030AEB830A594ADAF8383158498B42F0
:10DCA00014BF4FF480034FF40013116B0B43136345
:10DCB00000237268944206F1240603F101035CD04C
:10DCC000102BF6D100204F4960220023FDF746FEBD
:10DCD000204656F097FD236823F001032360204679
:10DCE00056F090FD019B0B9305F134033B440C93DC
:10DCF00040F22A430F934FF480631193424B0D93EC
:10DD000040230E934FF480504FF480430026CDE91A
:10DD100012030BA94FF440332046CDE91666CDE936
:10DD2000186610961496159355F0D0F80C2F04D859
:10DD3000364B03EB4703B3F8DC60AB899BB233434C
:10DD4000AB81236843F0100301202360B9E6284922
:10DD50008A4219D2002131E75B0003F00203ADF8DB
:10DD600024304FF001084FF48073ADF81A80ADF8FD
:10DD7000283057E7DBB2013B89E7D8B2A3E707EBCE
:10DD8000C20797F8380DECE6214802F1B77101F5AA
:10DD90005851A0FB0101890D013989B2481CB2FB21
:10DDA000F0F20BE71A4900F1B77202F55852A1FBE5
:10DDB0000221890D013989B24A1CFDE68A4204D24A
:10DDC00001200021B2FBF0F2F8E6114802F1B77130
:10DDD00001F55851A0FB0101890D013989B2481C98
:10DDE000F0E700BFC0020020181E07080004014031
:10DDF000006CDC02598B4F01ABAAAAAA0038024082
:10DE0000006002400588000890930020102F07084A
:10DE1000819F5E16202D0020281C002088010020F4
:10DE20002DE9F04FDFF8709299F8003089B01BB9F6
:10DE3000012009B0BDE8F08F934B1C68FCF75EFB36
:10DE400099F8C8350393002B00F012828F4BA3FB87
:10DE500004328F4B5209A3FB0213DB0803EB83034D
:10DE6000A2EB4303D9F8042B821A049209F6083B6B
:10DE7000DAB207920BEB830309F5C66409F6E852A0
:10DE8000029200279846019432E0304656F0BAFCE0
:10DE90008C2303FB0793002583F824569AF805A0EA
:10DEA000204651462A46FFF7D3FD019C2246FFF744
:10DEB0004BF951460822FFF7CBFD402344F83C3C88
:10DEC000A4F14801304655F001F804F18C030193A8
:10DED000029B14330293336843F010033360039BB7
:10DEE00001379F420BF15C0B08F15C0800F0D68013
:10DEF000049A002A05DB019B53F8083C934200F387
:10DF0000A2818C23019A03FB079352F858AC93F833
:10DF10002436166ADAF80040002BB6D07568A3895B
:10DF2000ADB2114632F8542CC5F116059BB223EA66
:10DF30000203072DA381A8D9D9F8F03D8A6A0133DD
:10DF4000C9F8F03D0021CDE90572106896468C466F
:10DF5000012315E0BCF1140F1EDC12F1080748BFC5
:10DF600002F117073A110CEB271C571E01FA02F2B7
:10DF700001210B4401FA07F79D4247EA02010BD346
:10DF800002465EF8040F9D42A0EB0202E2D8CCF1FB
:10DF900015024FF0150CE8E7BCF1150FDDE905722D
:10DFA00066D13C4DC1F38423C1F3441005EB8303D8
:10DFB00005EB8000D3F8F830D0F8F8001B0243EAF4
:10DFC000001301F01F0005EB8000C1F3C43105EB25
:10DFD0008101D0F8F800D1F8F810034343EA013387
:10DFE00083EA132181EA111101F00F010F293FD1BA
:10DFF000C3F30F134FF6FF718B4239D0B3F5606F47
:10E0000000F02581029A93819BF85820079882425C
:10E0100014D0D8F80810DBF80020521ACBF80020F2
:10E02000D8F83010DBF80420521ACBF80420002274
:10E03000C8F80820C8F830208BF85800DBF800201A
:10E040000132CBF80020D8F808200132C8F80820A7
:10E050004FF6FF7293427FF418AFDBF804300133C0
:10E06000CBF80430D8F830300133C8F830300CE742
:10E07000D9F8EC3D0133C9F8EC3D002F00F0D98010
:10E080004FF6FF73C0E700BF281C00201F85EB512F
:10E09000CDCCCCCC102F070804000010D9F8D8152F
:10E0A000C9F8045B012389F8EC3E0A68487999F8BD
:10E0B000E015890748BF0423118C83409BB289B2C5
:10E0C00021EA03011184118C89B20B431384039B51
:10E0D000012B3FF4ADAED9F864261368517999F855
:10E0E0006C26970754BF012204228A40198C92B2F1
:10E0F00089B221EA02011984198C89B20A431A846F
:10E10000039B022B3FF494AED9F8F02613685179A3
:10E1100099F8F826960754BF012204228A40198CE8
:10E1200092B289B221EA02011984198C89B20A4398
:10E130001A84039B032B3FF47BAED9F87C2713682A
:10E14000517999F88427950754BF012204228A4007
:10E15000198C92B289B221EA02011984198C89B210
:10E160000A431A84039B042B3FF462AED9F80828B3
:10E170001368517999F81028940754BF012204229A
:10E180008A40198C92B289B221EA02011984198C51
:10E1900089B20A431A84039B052B3FF449AED9F890
:10E1A00094281368517999F89C28900754BF01224C
:10E1B00004228A40198C92B289B221EA02011984A0
:10E1C000198C89B20A431A84039B062B3FF430AEA4
:10E1D000D9F820291368517999F82829920754BF52
:10E1E000012204228A40198C92B289B221EA0201EA
:10E1F0001984198C89B20A431A84039B082B7FF473
:10E2000017AED9F8AC2999F8B4191368507911F000
:10E21000020F18BF0422198C08BF0122824092B25B
:10E2200089B221EA02011984198C89B20A431A843D
:10E23000FEE511461248582263F05AFBDAF8004016
:10E240004FF6FF73E0E6002009B0BDE8F08F0D49FE
:10E2500091F88E2002EB420201EBC2023A4492F89E
:10E260009D200D2A7FF4CEAE029980228A77CBE6DC
:10E27000012389F8EC3E039BC9F8043BD8E500BFB5
:10E28000980E0010281C00200E4A92F8F13003F07E
:10E29000FF01002BF9D10C4B4FF0010C82F8F1C0BB
:10E2A000D3F88000D3F8DC2BB3F89430436051628C
:10E2B00013889BB243EA0C031380036843EA0C0300
:10E2C00003607047281C0020202D002037B590F8EF
:10E2D0005F38032B04462FD10023204D8DF80730E3
:10E2E0009DF8073094F860289A4201D803B030BDF9
:10E2F0009DF8073005EBC30393F8E43B8BB181F045
:10E30000010383B19DF8073005EBC303D3F8E00B9D
:10E31000FCF780FF9DF807300133DBB28DF8073042
:10E32000DEE70B46EDE79DF8073005EBC303D3F8B6
:10E33000E00BFCF775FFEDE7D0E910039B7903F0E4
:10E340000103994204D003B0BDE83040FCF762BF3E
:10E3500003B0BDE83040FCF763BF00BF202D0020B4
:10E3600038B5044600790D4650B1FCF717FE08B1E8
:10E370000323C380E2792946BDE83840FDF7C4BDD8
:10E3800038BD10B504462221FFF7EAFF6379216802
:10E3900002229B0802FA03F3DB439BB20B826379F0
:10E3A0008889D3409A40024392B28A8110BD10B549
:10E3B00004460121FFF7D4FF206861798389890829
:10E3C00002229BB28A4023EA0203838110BD38B542
:10E3D00010F8133CA0F664041BBB94F850388BBBB8
:10E3E000D4E909239A421CD05A1CA169A262CB5CD1
:10E3F00021695B0043F40073A4F854380A2384F8BD
:10E400005238012384F8503894F85F388A4228BF84
:10E410000022012BA26201D0042B02D1606CFFF715
:10E42000C6FF94F84C38002B6DD194F84D38013369
:10E43000DBB2092B84F84D3825D12046BDE83840A1
:10E44000FAF7B2BA94F952586DB1B4F854184B08AF
:10E45000A4F8543801F001012046013DFFF736FFD2
:10E4600084F85258DDE7D4E909239A4284F85058D9
:10E47000D7D194F85F38012B01D0042BD1D1606C37
:10E48000FFF77FFFCDE70A2B3DD194F84F382BB92A
:10E49000B4F8563843F00103A4F856382379D90765
:10E4A0000AD5B4F85608820501D4C30718D4B4F8C5
:10E4B0005C380133A4F85C38012284F84C2894F8C5
:10E4C0004F280023012A84F84D381CD1617984F843
:10E4D0004F38606C01F00101BDE838405BF052BE7E
:10E4E000E36AC0F3470013B1216B9847E4E7E3699F
:10E4F0006269D054E369E2680133B3FBF2F102FBD5
:10E500001133E361D8E738BD2DE9F84310F8133C27
:10E51000A0F664047BB1B4F8583801339BB2082BE1
:10E52000A4F858381BD90021606C84F85118A4F85D
:10E5300058185BF027FE384F97F8208CB8F1000F81
:10E5400003D101212046FFF7C1FE94F8503853BB98
:10E55000D4E909239A4204D1002387F8203CBDE87E
:10E56000F883B8F1020F12D808F1010814BFFF2395
:10E570007F2387F8208CA4F85438082384F8523875
:10E58000012384F85038606CBDE8F8430FE75A1C4B
:10E59000A169A262CB5C21698A4228BF0022DBB25A
:10E5A00028BFA262E7E794F952685EB3B4F85498C2
:10E5B00097F8215C19F001010BD0012D01D8012140
:10E5C00003E0AB1E012B09D800212046FFF77EFE99
:10E5D00004E015F0FD03F2D0012BF6D00135EDB2C9
:10E5E000032D87F8215CBAD9013E4FEA590976B26A
:10E5F0000023A4F8549884F8526887F8213C002E30
:10E60000A6D0ACE7D4E909239A42A8D184F850688F
:10E61000606CBDE8F843B4E6202D00201648174A88
:10E62000174938B5174C184D121A63F061F9D4F830
:10E630008820164B164842F47002C4F888201A68E5
:10E64000002142F001021A6099601A6822F0847277
:10E6500022F480321A6058601A6822F480221A600C
:10E660000C4AD960521B28460B4963F041F9A5605A
:10E67000BDE83840FAF7F2B90000001004000010BD
:10E68000A584080800ED00E00000002000380240EA
:10E69000103000248801002000000008144BD3F83B
:10E6A000F430B0EB930F14D2B0EBD30F13D2B0EB26
:10E6B000131F12D2B0EB531F11D2B0EB931F10D225
:10E6C000B0EBD31F0FD2B0EB132F0ED24FF48070EC
:10E6D00070470220704704207047082070471020C0
:10E6E000704720207047402070478020704700BF4F
:10E6F000281C002011F001020ED170B590F82810EE
:10E70000C568012982B0044607D0B5F1807F01D9E0
:10E710000123037702B070BD70470A4B466AD3F8F5
:10E72000240CFFF7BBFFB5F1807FB080F2D9B7258D
:10E7300021770B46304601A98DF8045052F0E0F9DC
:10E74000E8E700BF202D00202DE9F0410546406A92
:10E7500094B0144600681F460E465EF029FF0B94E5
:10E76000264C0C9704F560730093254B019302230C
:10E77000002202930123CDE90922CDE90E22CDE941
:10E7800010228DF80C308DF834308DF84830069218
:10E790002B7F8DF8202013921A4A049204F55E72A2
:10E7A00005921A1D079223B3330E84F8793304F2CD
:10E7B0007A34330CDFF850802370330A6370A6700C
:10E7C000D8F8240C6A6AFFF769FF6B7F90809BB1D1
:10E7D0006946104652F0DAF96C6A20685EF0E8FE8D
:10E7E000D8F82C0CFFF75AFFA080384614B0BDE8CB
:10E7F000F08104F27934DCE705A9EAE7880100201A
:10E8000048390020E5920008202D00202DE9F04F26
:10E81000013B9FB2B44BDFF8D8C2D3F8F4400B6889
:10E8200083B06345BDF830609DF834503AD0DFF8CE
:10E83000BCC2634536D00CF5804C634500F0428184
:10E840000CF5806C634500F03D810CF5806C6345F0
:10E8500000F038816408B4FBF2F41A88013CB3F18B
:10E86000804FA4B292B200F03781DFF888C26345CE
:10E8700000F032810CF5806C634500F02D810CF5C1
:10E88000806C634500F02881DFF86CC2634500F0BE
:10E890006481DFF868C2634540F01A811A80DF6244
:10E8A0001C850DE0B4FBF2F41A8822F45C721204A9
:10E8B000120C013C1A80A4B20022DF621C851A8669
:10E8C00001229A824C798A790DB182F0010212F00C
:10E8D000020C62D0D2004FF0000E02F008074FF495
:10E8E000806201924FF0400CF346CDF800E0F24612
:10E8F00072464FF0040975460C2C35D8DFE804F059
:10E90000B73434348B343434073434345E001C8CE4
:10E91000DFF8D8C124F480742404240C1C841C8CDB
:10E9200024F4007424042A43240C9D8844EA02241D
:10E930009A8B22F073021204120C6345ADB242F0BE
:10E94000600200F0EB800CF5806C634500F0E6801F
:10E950009D809A83DE631C849A8B22F00802120445
:10E96000120C42F008029A83B3F844206FEA424244
:10E970006FEA524292B2A3F844201A881C4692B21F
:10E9800042F0010224F8342B4A794360A118002395
:10E990000160A35003B0BDE8F08F4FF480655200D2
:10E9A000CDE9005C02F002024FF4805E4FF4804B30
:10E9B0004FF4807A6746E14601259DE715431A8C9E
:10E9C0004A4F22F480521204120C1A841A8C22F438
:10E9D00000521204120C42EA05329D889C8B24F4EA
:10E9E000E6442404240CBB42ADB244F4C04400F01D
:10E9F000AF8007F58067BB4200F0AA809D809C83B2
:10EA00001E641A849A8B22F400621204120C42F4DF
:10EA100000629A83A8E71C8CDFF8D0E024F0100491
:10EA20002404240C1C841C8C24F0200424042A4379
:10EA3000240C9D8844EA02141A8B22F4E642120444
:10EA4000120C7345ADB242F4C04259D00EF5806E3F
:10EA5000734555D09D801A839E631C841A8B22F4C3
:10EA600000621204120C42F400621A837CE71C8CD0
:10EA7000DFF878C024F001042404240C1C841C8CCE
:10EA800024F0020424042A43240C9D8814431A8B86
:10EA900022F073021204120C6345ADB242F0600220
:10EAA00049D00CF5806C634545D09D801A835E6328
:10EAB0001C841A8B22F008021204120C42F0080285
:10EAC0001A8351E7B4FBF2F2541E1A88A4B292B230
:10EAD00022F4407292B2E1E622F45C7292B21A80A1
:10EAE000DF621C85ECE600BF281C0020000001400E
:10EAF00000040140000400400010004000140040E9
:10EB000024F0800444EA0714009F25F4406524F0B3
:10EB100040042F434CEA04043D469BE724F4006480
:10EB200044EA0724019F24F4806425F440553C43C3
:10EB30004EEA05050CE74FF6F37C04EA0C0C25F4CD
:10EB400040754CEA070C45EA0A054CEA0904ACE7B3
:10EB500025F480454BEA050550E7ACF80020CCF8D9
:10EB60002C70ACF82840ABE6274A92F8F83A7BB311
:10EB7000D2F8381A884237D0012B29D0D2F8501A4F
:10EB8000814235D0022B23D0D2F8681A884231D086
:10EB9000032B1DD0D2F8801A88422DD0042B17D019
:10EBA000D2F8981A884229D0052B11D0D2F8B01A81
:10EBB000884225D0062B0BD0D2F8C81A884221D023
:10EBC000072B05D0D2F8E01A814208BF07230CD0EA
:10EBD00003EB430102EBC10103F1010CC1F8380A58
:10EBE00082F8F8CA184670470023DBB2184670470F
:10EBF0000123FAE70223F8E70323F6E70423F4E707
:10EC00000523F2E70623F0E7040000100548D0F8DA
:10EC1000703623B1DB6A13B100F5CE6018470248A5
:10EC2000704700BF281C00208830070838B51D4CED
:10EC3000D4F8303C1B8843B91B4D002384F83F3C7B
:10EC400085F86836C5F8643638BDD4F8342C002A07
:10EC5000F2DDD4F8381C012A488806D00123124D71
:10EC6000A4F83C0C84F83E3CE7E78A880132121A8B
:10EC70009A42F3D10C4DD5F8703600221B69C5F8C5
:10EC80009C2605F5CE609847D5F870369B68002B1A
:10EC9000D3D005F5CE6098470028CED15CF0F0FBCC
:10ECA000CBE700BF202D0020281C00200748D0F80B
:10ECB0006C361BB1064B93F83E3C0BB100207047FD
:10ECC000D0F8703600F5CE605B681847281C00202D
:10ECD000202D002030B4174A174B92F868C603F570
:10ECE000446505EB0C04C0E9004593F83F3C92F8FD
:10ECF0006806834292F8680614D8834206D300233C
:10ED00001A46184630BCC1E90032704792F86806CE
:10ED10001A1EC0F1800330BC0CBF01200220C1E9E3
:10ED2000003270471B1A0022012030BCC1E90032BA
:10ED3000704700BF281C0020202D00200E4B0F4ADA
:10ED400093F8681692F83F0C93F86826904293F86F
:10ED500068260CD8904238BF93F86826D3F86436FA
:10ED60003ABFC2F180028018002018447047D3F8DF
:10ED70006436801A18447047281C0020202D00207B
:10ED800038B5194D194CD5F8302C937B012B08D090
:10ED9000D4F8643603F2FF736FF30A03C4F86436E1
:10EDA00038BDD4F870365B6A63B104F5CE6098471D
:10EDB000D4F870369B681BB104F5CE60984778B1E3
:10EDC000D5F8302CD4F864365288013B13445242B3
:10EDD000134003F2FF736FF30A03C4F8643638BDBF
:10EDE0005CF04EFBECE700BF202D0020281C00202B
:10EDF00070B51E4C1E4D94F8683694F8681684B0B1
:10EE000005F544621344029395F83F3C03928B420C
:10EE100020D894F86826934214D294F868161E46B7
:10EE2000C1F18001F3B98C460122CDE9001610B979
:10EE3000BCF13F0F06D90023694602A85FF0F4FC3D
:10EE400095F83F3C94F86806C01AB0FA80F0400983
:10EE500004B070BD94F868C6A3EB0C0C61460026A4
:10EE60000122E2E701EB030C0222DEE7281C00206E
:10EE7000202D00202DE9F043164685B0002936D01C
:10EE8000441E254D254F04EB01084FF0000901E019
:10EE9000A0452CD095F83F0C14F8013F411C2844A4
:10EEA000C9B280F8403C0B0648BF002097F868368E
:10EEB00085F83F1C4ABF0146084685F83F9C9942A9
:10EEC00097F8683636BFC3F18003C01AC0183F28D0
:10EED000DED997F868369942DAD0114B93F8C430EE
:10EEE000002BD5D00020FFF783FFA045D2D1694683
:10EEF00002A8FFF7EFFE20B1DDE9003213443F2BFB
:10EF000002D805B0BDE8F0830246334602A85FF0A0
:10EF10008BFC05B0BDE8F083202D0020281C0020CC
:10EF20008801002030B585B0694602A8FFF7D2FEFF
:10EF300058B9094C04F5CE65D4F8703628465B689C
:10EF400098470028F8D005B030BD0246012302A83A
:10EF50005FF06AFCEDE700BF281C002070B5134D80
:10EF6000134C0023C5F86C365AF0C8FDC4F8380CB1
:10EF7000FFF74CFED4F8383CC4F8300CA3B19A88A3
:10EF80005B88D21A436802FB0333C5F86C36FAF784
:10EF9000B5FA95F8683694F83F2C9A42064601D0A7
:10EFA000FFF7C0FFC5F8646670BD00BF281C0020D5
:10EFB000202D00202DE9F041104ED6F86C36154674
:10EFC00082189A420E4A88BF1D1A92F83F2C96F872
:10EFD00068369A4204460F4601D0FFF7A3FFD6F8E1
:10EFE000702608480023C6F89C362B46956A2146B1
:10EFF0003A46AC46BDE8F041604700BF281C0020FF
:10F00000202D0020982200208C461346014662469F
:10F010001846CFE72DE9F04F41F62C728BB0002156
:10F02000C44862F0BDFC042055F0E6FC044605200F
:10F0300055F0E2FC50EA040340F02A81BE4B0393F2
:10F04000039BBE49BB48D3F8B443E42262F050FCB2
:10F05000B84BC3E90744C3E91A445C621C67C3F8B0
:10F06000B4401F46C3F8B840C3F8BC405DF094F804
:10F07000FFF774FF002108460DF080FEFAF73EFA14
:10F08000B0F1000840F3A481AD4DDFF8DCC2AD4E15
:10F09000CDF808C0002407F1E40901942746A246F0
:10F0A00005F54C6B04E00AF5006AD04540F3AF80EB
:10F0B000029A1368C2F8B436FAF754FA2022594675
:10F0C0005046FFF777FFA0491222584662F0A5FC90
:10F0D0000028E8D1BA4525D001999C4B01EB4102AB
:10F0E00003EB820301934A1C184699490592AAEB47
:10F0F0000703049301F04CFC4946019B41F84C3B4B
:10F10000049B059AC9F80C70C9E90433D9F81C307E
:10F110000192C9E908338F4BC9F828300123C9F897
:10F1200008308946039BD3F8B433C9F81C305746DE
:10F130001222A918335D91F8C01C994202F1010214
:10F140000BD00024202AF4D12037B8455946384640
:10F1500053DBFFF72FFF0022EBE70134152CF1D131
:10F16000D0197D492022FFF725FF00230A2209A993
:10F170007948CDF824B001F03DFD074609980023F9
:10F1800001300A2209A9099001F034FD079009987D
:10F19000002301300A2209A9099001F02BFD0690F5
:10F1A0000998002301300A2209A9099001F022FDE3
:10F1B0000590099809A9013000230A22099001F05D
:10F1C00019FD04900998002301300A22194601F024
:10F1D00011FD97B1DDE9063243EA4212049B05991D
:10F1E0005B0143EAC123A7F2BC7143EA600342EA30
:10F1F000412243EA0243C9F81C30019B642B00F012
:10F20000B58057460AF5006AD0453FF751AF019BDC
:10F21000642B00F0AB80BA451DD0019B4B4C4C4990
:10F220000C2202FB034401331A462046019301F0ED
:10F23000AFFBD9F81C20C9F80040AAEB0705C9E9C3
:10F240000822C9E90375434AC9F828200122C9F8F0
:10F250001450C9F80820019B002B03F1030100F3AF
:10F2600088804FEA4803B3F1805FC0F2B280314B2F
:10F27000986830B91A461B791BB11368002B40F00F
:10F28000DE80002108460BB0BDE8F04F0DF076BDE2
:10F290004FF47A72002321465FF0BEFF2F4BA3FB91
:10F2A00000231B0C40F2B27240F26D1401E05B1AB5
:10F2B000013212F0030514BF21464FF4B7718B429F
:10F2C000F5DA1D49002D00F0B48003910399D1F8BF
:10F2D0008413994200F35781214D01245B1A55F89C
:10F2E000041F994204F10104F8DD013343EA441399
:10F2F000A2F2BC7243EA42231A4A039DB0FBF2F128
:10F3000002FB11024FF461603C24B2FBF0F100FB00
:10F3100011221C20C5F88803B2FBF4F004FB102274
:10F32000521042EA401242EAC12242EA0343C5F8BF
:10F33000B43385E6706E0020880100209C300708F9
:10F34000202D002078C0070854C00708003A00208C
:10F3500068C0070809F00008E039002007452EC200
:10F360000C05002080510100281C0020642301931B
:10F3700067214C268548DFF82892854F06FB01F46B
:10F38000051932460021284662F00AFB3246002168
:10F39000284662F005FB7D487E4E40F8049004F15B
:10F3A00010034FF0010AC5F808A02F62AE6240F8C2
:10F3B00003800344021DC3F804801834039B0199A1
:10F3C000D3F8B4331351A018043143606B6248E79B
:10F3D00003216E4BDFF8CC914C2606FB01F41D197E
:10F3E00032460021284662F0DBFA324600212846E8
:10F3F00062F0D6FA654B664E43F80490039A2E628B
:10F40000654ED2F8B40304F1100104F1180201278B
:10F41000341FC8F10063BB404FF0020A85F805A015
:10F42000AF60635021444B60B0503244506068621A
:10F430001DE70C4603911D21C4F8881346E7534984
:10F4400000220023C1E9102388640A46C8630546E8
:10F450000146D46C02F14C03B4B19C689D644E1E0D
:10F46000B442C2E92355DD6300F086804E1CB442ED
:10F4700074D113F8481C00293FF403AF1A6443F811
:10F48000083C21461A46E4E7404A0226254615E094
:10F49000D36B16635B0118BF03F6FF73C2E9045513
:10F4A00014BF01EB1333334653631946916352F88B
:10F4B0004C7FCB1A1C444E1C0130CFB11379711E06
:10F4C000002BE5D1136916635BB103F6FF7357692F
:10F4D00001EB133353634FB107F6FF7701EB17319D
:10F4E000E4E7576933465363002FF5D13146DDE732
:10F4F000DFF8B4C0294BCCF8F84601390CF5DA62D4
:10F50000CCF8DC363E2440233F25CCF80407CCF869
:10F51000E836C2E90445CCF8F416880F8B00D9B15F
:10F5200040F2FF141B1940F100005B0A43EAC0538C
:10F530001648C2E90B0003F14000034403EBC1018C
:10F54000CCF8F036CB0D53604B02CCF8EC06CCF87F
:10F55000D816CCF8D03694E60123E9E78C427FF444
:10F5600090AE00293FF48DAE146CE66B0136E66375
:10F570001C6493641A466CE700293FF482AE53F88A
:10F580000C2C2146EDE70124AFE600BF706E002091
:10F590000068214C09F00008746E0020ACC0070818
:10F5A00090C00708A0C00708281C00202DE9F043E0
:10F5B000DFF82881474D93B0FFF738FB98F868369D
:10F5C00095F83F2C9A4201D0FFF7ACFCD8F86C7646
:10F5D0000024C8F86446002F6DD03F4E0AE098F82A
:10F5E000683695F83F2C9A4201D0FFF79BFC2034F7
:10F5F000A7421BD922463146684601F0C9F9684640
:10F600005FF0ACF9012201466846FFF733FCA3B274
:10F61000002BE4D1D8F8BC36002BE0D09A881B68C8
:10F6200059690A4214BF5A831A83D8E7FFF7A8FB27
:10F6300098F8683695F83F2C9A4201D0FFF772FC93
:10F640000023DFF89490C8F864361E461C4602E09A
:10F650002034A74229D92246494609A801F098F941
:10F6600021220021684662F09BF92022694620464B
:10F67000FFF7A0FC2022054609A9684662F0CDF9F3
:10F6800008B9202D00D00136A3B2002BE0D1D8F864
:10F69000BC36002BDCD01A689B88516920340B42A1
:10F6A00014BF53831383A742D5D8B6FA86F0400916
:10F6B00013B0BDE8F083FFF763FB98F8683695F860
:10F6C0003F2C9A4201D0FFF72DFC0023C8F8643686
:10F6D0000120EDE7202D0020B4C00708281C0020E1
:10F6E00000B585B0184A002301930192019A0C32AB
:10F6F0000192019A0321116072B6144AD2E92612CE
:10F7000051EA020412D11A460F48002402940290D2
:10F7100002991031029102990A6003940390039AAE
:10F7200014320392039A1360FDF760FA084B1B68CA
:10F730004EF6602404FB00F05B1842F10002C3188F
:10F7400042EBE072E0E700BF50280040183E002086
:10F75000281C0020704700BFD0ED007AD0ED016A70
:10F7600030EE677AE6EE877AB0EE670AC0ED007A8F
:10F77000704700BFD0ED017AD0ED026A30EE677AB3
:10F7800090ED000AE6EE877A37EEC07AC0ED017A96
:10F79000A6EE870A80ED000A704700BF90ED017A5F
:10F7A000D0ED036AD0ED027A30EE470AA6EE807AF9
:10F7B00090ED000A80ED017A37EE676AE6EE867A10
:10F7C00037EEC07AC0ED027AA6EE870A80ED000A15
:10F7D000704700BFD0ED056AD0ED017A90ED066A62
:10F7E000D0ED025A90ED035AC0ED066AB0EE407AB1
:10F7F00026EEA70AD0ED007A80ED057AA7EE870AFB
:10F80000D0ED077AA5EE860A90ED086AD0ED045A8D
:10F81000C0ED087AA5EE670AA5EEC60A80ED070AD4
:10F82000704700BFF0EE406AD0ED007A90ED050A17
:10F8300090ED067A90ED016AD0ED035AA7EEA60A84
:10F84000A6EE267AD0ED047A90ED026A67EEC07AD1
:10F85000A5EEC07AE6EE267A80ED057AC0ED067A4E
:10F86000704700BF2DE9F047DDF820A055460F4650
:10F8700015F8011B002B064614460CBF4FF020095B
:10F880004FF0300939B3002A2BDD2B4600E09CB144
:10F8900013F8012BA046013C002AF8D1A8F1020878
:10F8A00054B1444649463046B847013CFAD29AF82A
:10F8B000001008F1010459B13046B8472B4615F83D
:10F8C000011B0029F8D1A4EB0A041819BDE8F08740
:10F8D0002046BDE8F087002A02F1FF38E1DC084647
:10F8E000F4E70024E8E700BF03685A1C02601970BF
:10F8F000704700BF10B500F100440246013C04E02F
:10F90000B3EB0E0015D1A24214D012F8013BA3F1C3
:10F910004100192811F8010BA0F1410C98BF2033C8
:10F92000BCF1190F00F1200EEAD91B1A04D10028EE
:10F93000E9D110BD002010BD184610BD884210B599
:10F940004FF001043ED301FB04F4B0FBF4FC8C4502
:10F95000F9D2CCB122BB08E0A14203F801EBB4FB21
:10F96000F1F211D8B0FBF2FC1446BCF1090F0CF116
:10F97000570E0CF1300204FB1C00EDDCA14203F831
:10F98000012BB4FBF1F2EDD900221A7010BDA14297
:10F9900003F801EBB4FBF1F2F6D8B0FBF2FC14462D
:10F9A000BCF1090F0CF1370E0CF1300204FB1C0006
:10F9B000EDDCA14203F8012BB4FBF1F2EDD90022FA
:10F9C0001A7010BD8446002AEAD1CEE7002870B52F
:10F9D00003DA2D2301F8013B4042092886464FF007
:10F9E000010307DD03EB83035B00B0FBF3F2092A9D
:10F9F000F8D8E3B10F4CA4FB0320BEFBF3F2092AB5
:10FA000002F1570602F130054FEAD00007DD092B5D
:10FA100001F8016B03FB12EE09D90346EBE7092B52
:10FA200001F8015B03FB12EE01D90346E3E7002373
:10FA30000B7070BDCDCCCCCC0378202B024600F1EE
:10FA40000100F9D0092BF7D02D2B28D02B2B03BF89
:10FA50005378B7EE000A0246B7EE000AA3F1300170
:10FA6000C8B209289FED567A10D8F2EE046A07EE64
:10FA7000901AF8EEE77A12F8013FE7EE267AA3F142
:10FA80003001C8B20928B0EE677AF0D92E2B5ED0CB
:10FA900003F0DF03452B07D020EE070A70475378A9
:10FAA000BFEE000A0246D9E710B451782D2978D06C
:10FAB0002B296AD0A1F13003092B02F101026BD886
:10FAC0000024002303EB830301EB430312F8011F1F
:10FAD000A1F130000928A3F13003F3D9B3F59A7FDF
:10FAE0001A4628BF4FF49A72072B66D9DFED356AA4
:10FAF0001346F7EE007A083B072B67EEA67AFAD892
:10FB000002F00702DAB1F2EE046A012A67EEA67A81
:10FB100015D0022A67EEA67A11D0032A67EEA67ADC
:10FB20000DD0042A67EEA67A09D0052A67EEA67AD8
:10FB300005D067EEA67A062A18BF67EEA67A6CB3E0
:10FB400087EE277A5DF8044B20EE070A704753785A
:10FB5000A3F13001C8B2092802F1010298D8F2EEEF
:10FB6000046AF0EE665A07EE901AF8EEE77A12F899
:10FB7000013F87EEA66AA3F13001C8B2092866EEFC
:10FB8000A56A37EE067AEED982E79178A1F13003C3
:10FB9000092B02F1020293D9F7EE007A27EE277AB9
:10FBA000D0E79178A1F13003092B02F1020288BF5E
:10FBB000F7EE007AC4D8012483E7F7EE007AA1E7D4
:10FBC0000000000020BCBE4CF0B5067906F0E00352
:10FBD000402B03D145794FF0FF3406E0602B4FF006
:10FBE0000105F8D1447905FA04F40023012006F058
:10FBF0000706AB4200D1F0BD052E0FD8DFE806F0B6
:10FC00000308101D242448B1C85CD75C78400FE07D
:10FC100020B1C856D756C71B784278410133E8E770
:10FC20000028FBD031F8130032F81370784080B20E
:10FC300020420CBF01200020F0E70028EED031F96F
:10FC4000130032F91370E6E70028E7D051F82300DB
:10FC500052F82370DAE7F8B50C4E337805468BB9C5
:10FC6000F8BD25B12388C3F30B039D4204D0D4E92A
:10FC70000201A28861F03CFE1C34BC42F1D3002397
:10FC80003370EDE7024C034FF7E700BF38A40020C4
:10FC9000F05D0808C8670808037903F01803102B03
:10FCA0001CD003D833B9B0F80B007047182BFAD02A
:10FCB00000207047104BB0F80B0093F90030591C2E
:10FCC00006BF0E4B1B78DBB203EB430203EB820350
:10FCD00003EBC30300EB430080B27047064BB0F860
:10FCE0000B0093F901305A1C06BF044B5B78DBB262
:10FCF00000EB4310F0E700BF34060020B83E0020C0
:10FD0000032870B516D80C4BC60003EBC000C943DE
:10FD1000057A427A01F0010181EA0504A24209D084
:10FD200042682AB190881268A94214BF1083508398
:10FD300033445C7270BD00BF38A400200379062BE9
:10FD40000FD1C9B20D2998BF074BC26894BF59564D
:10FD5000002101238B40134214BF08464FF0FF30AF
:10FD60007047481C704700BF28C10708092900D008
:10FD700001B9704701394A0002F00802930001F00E
:10FD80000301A3EB9203C1EB0111C3EB0313C1EB1E
:10FD9000011100229B00890002608180438070472E
:10FDA000B5EEC00ADFED347AF1EE10FACCBF30EEDA
:10FDB000270A30EE670ADFED317A20EE270A30B5E8
:10FDC000FDEEC07A87B017EE904A054684EAE470EB
:10FDD000002303A9A0EBE470CDE90033029357F0B0
:10FDE0000BFE002CB4BF2D23202303A88DF8003078
:10FDF0005EF0B4FD012829D0022833D003281DD09D
:10FE000003A9684661F0D4FD68465EF0A7FDC41EF4
:10FE1000E4B222466946284661F06AFD00232B556C
:10FE200028465EF09BFD2E232B5401300DEB040180
:10FE3000284461F0EAFD284607B030BD302303A90D
:10FE400068468DF8013061F0B3FDDDE743F2300222
:10FE5000302303A96846ADF801208DF8033061F026
:10FE6000A7FDD1E743F2300303A96846ADF801309E
:10FE700061F09EFDC8E700BF6F12033A00007A44AC
:10FE80000CF09EBD38B5054658B14C1E14F8011F44
:10FE9000284619B9BDE838400CF0A6BD0CF090FD1D
:10FEA000F4E738BD70B50546B0F8090054F0F0FB32
:10FEB000054B1E7804462846FFF7EEFE16B1E368B0
:10FEC000184470BDA368FBE738A4002038B5054688
:10FED0000C46FFF7E7FF2A7902F0070302F0E00281
:10FEE000602A29D1052B0CD8DFE803F0030B0F0B98
:10FEF0001B1B6A7901239340DBB2027814B11343D0
:10FF0000037038BD22EA0303FAE76A7901239340BC
:10FF10009BB2028814B113430380F2E722EA030381
:10FF2000FAE76B7901229A40036814B11343036026
:10FF3000E7E723EA0203FAE7052BE2D8DFE803F05C
:10FF40000303050507070470DBE70480D9E70460B5
:10FF5000D7E708B5202161F03AFD0346184623B1E2
:10FF60000278202A03F10103F8D008BD08B5CB07B9
:10FF700001D4FCF73BFE08BD2DE9F341124D134FB0
:10FF8000002305F8243F044600EB8106B44203D168
:10FF90000F4802B0BDE8F0813946284661F008FDFF
:10FFA0002146684661F031FD4FF000082021684687
:10FFB00061F00DFD28B96946284661F0F9FC04346A
:10FFC000E4E780F80080F1E738A40020FF4108084A
:10FFD0005CA400202DE9FF47914604468A461E4650
:10FFE000FFF7ACFE421CBDF83070DDF834800546EA
:10FFF0001FD0B9F1FF3F1FD0CDE90009144A236893
:020000040801F1
:1000000031463846C0474A4620795FFA8AF1FBF705
:100010003DFB024600B10288D3B20393C2F303232F
:10002000120BCDE90052029323680A4A3146384642
:10003000C04704B0BDE8F0877B06FAD40C90236873
:10004000054A31463846C44604B0BDE8F04760472B
:100050001A360808273608084B3608082DE9F043F9
:10006000154685B06A1C8946BDF830600D9F19465B
:1000700025D04FEA101800F00F0408F14008CDE930
:100080000045164A43463046B847A8B199F80510CE
:10009000D9F800002A46FBF73BFB68B103880278D9
:1000A0000392C3F303221B0BCDE9004302924346A4
:1000B0000B4A00213046B84705B0BDE8F08373060F
:1000C000FAD40309074A00F00F000C904033304681
:1000D000BC4605B0BDE8F043604700BF5A3608088B
:1000E0006C360808953608082DE9F04387B00709F3
:1000F000DDF8388091461E46403700F00F0439B3D2
:100100000FF0C0FBC379174ACDE9004305463B46D3
:1001100049463046C047C0B12868FBF709FEAA79B6
:100120006B79114912F0020F4FEA93030F4A18BF7F
:100130000A46E97900940133CDE90321CDE90103B1
:100140000B4A3B4600213046C04707B0BDE8F0836C
:10015000084A0E943B4649463046C44607B0BDE8BF
:10016000F0436047A9360808A03A0808294C080857
:10017000BB360808DD36080800B501EB020E7145F4
:1001800016D001390EF1FF3E41F2210C11F8013F6A
:10019000082280EA032003B2002B4FEA4000B6BFDA
:1001A0008CEA430380B298B2013AF4D18E45EDD186
:1001B0005DF804FB4840082341B240000029C0B26A
:1001C000B8BF5040013BF7D1704700BF30B505685C
:1001D0008D42044618D901F1FF3E681E00231EF827
:1001E00001CF082183EA0C034FFA83FC5B00BCF1CA
:1001F000000FDBB2B8BF53400139F5D17045EED1E5
:100200006A1C22602B7030BD00236A1C22602B7098
:1002100030BD00BF10B52DED028B08EE101AB8EE00
:10022000488ADFED7E7ADFED7E0A28EE008A0446FA
:1002300028EE278AB0EE480A60F0B0FA9FED797A8E
:10024000B4EEC70AF1EE10FAF0EE407A40F3BD804A
:100250009FED736ADFED746AB0EE677AB4EEE67A0A
:10026000F1EE10FA77EEC67AF6DC9FED707AF4EED6
:10027000C77AF1EE10FA40F3C5809FED6A7A77EE07
:10028000677A27EEA76ADFED6A5ADFED6A6A9FEDAB
:100290006A7A9FED660ADFED620AE6EE256A67EE8E
:1002A000865AA6EE267A38EE000AE5EE877AB0EE98
:1002B000678A60F073FADFED5B7AB4EEE70AF1EE7D
:1002C00010FA5BDDDFED566A9FED577AF0EE407A6B
:1002D000F4EEC77AF1EE10FA30EE660AF6DCDFEDE6
:1002E000537AB4EEE70AF1EE10FA62DDDFED4D7AF3
:1002F00037EEC00AF7EE007ADFED504ADFED4C5AD8
:100300009FED4C7AC4ED097AB0EE675AA8EE245AF4
:100310000023A36160EE006A87EE856A6361236251
:10032000E361A6EEA57A9FED445AA6EE875A20EE29
:10033000264AF0EE675AA4EE050AE8EE645ABDECD0
:10034000028BB6EE007AF8EE006A77EEC07A26EEFF
:10035000077A66EE266A27EE277A66EE806A67EEEF
:10036000867A25EE866A84ED007AC4ED017A84ED02
:10037000027AC4ED036A84ED046A10BDDFED307AC1
:10038000B4EEE70AF1EE10FAA9D5DFED256A9FED8C
:100390002D7AF0EE407AF4EEC77AF1EE10FA30EEF4
:1003A000260AF6D4DFED217AB4EEE70AF1EE10FA70
:1003B0009CDCDFED257AB4EEE70AF1EE10FA44BFDB
:1003C000DFED1F7A37EEC00A94E79FED1D7AB4EE99
:1003D000C70AF1EE10FA7FF548AF9FED116ADFED25
:1003E000196AB0EE677AB4EEE67AF1EE10FA77EEBB
:1003F000867AF6D49FED0D7AF4EEC77AF1EE10FA14
:100400003FF73BAF9FED107AF4EEC77AF1EE10FAAA
:1004100044BF9FED0B7A77EE677A32E727D4D23666
:10042000DB0FC940DB0F4940E4CB1641DB0FC93F6E
:1004300092E741B99730083C15A82ABEF304353F2E
:10044000DB0F49C0E4CB16C1DB0FC9BF08B5DFED38
:100450002D0A60F0A3F9DFED2C7AB4EEE70AF1EE95
:1004600010FA28DDDFED276A9FED287AF0EE407A5A
:10047000F4EEC77AF1EE10FA30EE660AF6DCDFED44
:10048000247AB4EEE70AF1EE10FA2FDDDFED1E7AE2
:1004900037EEC00A20EE007A9FED1E6ADFED1E6A7D
:1004A000DFED1E7AE7EE066A20EE076AE6EE877A4F
:1004B000A6EE270A08BDDFED1A7AB4EEE70AF1EEE0
:1004C00010FADCD5DFED0F6A9FED167AF0EE407A78
:1004D000F4EEC77AF1EE10FA30EE260AF6D4DFED2C
:1004E0000C7AB4EEE70AF1EE10FACFDCDFED0E7A0B
:1004F000B4EEE70AF1EE10FA44BFDFED097A37EE09
:10050000C00AC7E7DB0FC940DB0F4940E4CB164107
:10051000DB0FC93F92E741B99730083C15A82ABEC6
:10052000DB0F49C0E4CB16C1DB0FC9BFDFED2F7A6B
:10053000DFED2F0A30EE270A08B560F02FF9DFED66
:100540002D7AB4EEE70AF1EE10FA28DDDFED286A25
:100550009FED297AF0EE407AF4EEC77AF1EE10FAC8
:1005600030EE660AF6DCDFED217AB4EEE70AF1EE52
:1005700010FA2FDDDFED1F7A37EEC00A60EE006A59
:100580009FED1E6A9FED1E7ADFED1E7AA6EE867A3B
:1005900020EE266AE6EE877AA6EE270A08BDDFED92
:1005A0001A7AB4EEE70AF1EE10FADCD5DFED106A44
:1005B0009FED167AF0EE407AF4EEC77AF1EE10FA7B
:1005C00030EE260AF6D4DFED097AB4EEE70AF1EE52
:1005D00010FACFDCDFED0E7AB4EEE70AF1EE10FA96
:1005E00044BFDFED097A37EEC00AC7E7DB0FC93F2A
:1005F000DB0FC940DB0F4940E4CB164192E741B91C
:100600009730083C15A82ABEDB0F49C0E4CB16C1C1
:10061000DB0FC9BFB0EEC07AF0EEE06AF4EEC76A55
:10062000F1EE10FAB4BFF0EE475AF0EE665AF5EE6E
:10063000405AF1EE10FAF0EE407A44D0F4EEC76A78
:10064000F1EE10FA8CBFB0EE475AB0EE665A85EE66
:10065000256A9FED1E2A9FED1E3A9FED1E4ADFED93
:100660001E4ADFED1E2ADFED1E3A9FED1E5AA6EE52
:10067000423AE6EE223AA6EE034AF7EE005AE6EEDA
:10068000044AE6EE235AA6EE245A85EE250AF4EE35
:10069000C76AF1EE10FA48BF9FED137AF5EEC00A73
:1006A00048BF37EE400AF1EE10FA48BF9FED0F7ACF
:1006B000F5EEC07A48BF37EE400AF1EE10FA48BFB7
:1006C000B1EE400A70479FED070AE0E739094E3D59
:1006D000E3B59E3E88FA163E45FE7F3F99FB243FD8
:1006E00069A2163EA7DFA834DB0FC93FDB0F4940E4
:1006F0002DE9F04F144689B08846217801320392E3
:10070000002900F01681002507461E46A94609E08B
:100710003846C047039C01352178631C03930029A8
:1007200000F08F802529F3D16078A31C3028CDE913
:10073000033923D0A0F13003DBB2092B4FF0000ABC
:1007400026D96C282AD078287FD8572878D9A0F1C4
:100750005803202B79D8DFE803F0BD7878787878D3
:10076000787878787882AF787878787878787878C8
:10077000AA787878789E788A7878BD00A078E31C8B
:100780000393A0F13003DBB2092B4FF0010AD8D854
:1007900004AA03A959F08CF96C28D4D1039C2278BF
:1007A0000134782A0394B7D8572A40F28E80A2F1F8
:1007B0005803202BB0D801A151F823F0F308010809
:1007C0001907010819070108190701081907010885
:1007D0001907010819070108190701081907010875
:1007E0001907010819070108610801080F09010824
:1007F0001907010819070108190701081907010855
:100800001907010819070108190701081907010844
:1008100019070108B108010819070108190701089B
:1008200019070108190701089908010819070108A3
:100830001F0901081907010819070108F308010831
:1008400028B9284609B0BDE8F08F039C64E7252845
:10085000FBD1039C25213846C04701355CE7039C4A
:1008600056F8041B3846C9B2C047013554E70DF1AC
:10087000140B56F8040B039C5B4600220A21FFF779
:100880005DF8049ACDF800B0534641463846FEF76D
:10089000E9FF054440E7039C56F8043B0093049AA3
:1008A000002341463846FEF7DDFF054434E7039C4C
:1008B00056F8043B1D602FE70DF1140B56F8040B9E
:1008C000039C5946FFF782F8DBE7002AB9D0252AB6
:1008D000C0D021E7A0F15802B2FA82F20DF1140B58
:1008E00056F8040B52095B461021FFF727F8039CCA
:1008F000C7E7A2F158020DF1140BB2FA82F256F8D2
:10090000040B52095B461021FFF718F8B9E70DF107
:10091000140B56F8040B5946FFF758F8B1E70DF1E0
:10092000140B56F8040B5B4600220A21FFF706F869
:10093000A7E70D4685E7F8B5104C0746A06C0D46B5
:100940001646A0B10E49FFF79DFAA06C3946FFF795
:1009500099FA0C49A06CFFF795FA0B49A06C334645
:100960002A46FFF7C5FE0949A06CFFF78BFA94F8F9
:100970004C3013B1012384F84D30F8BD38A4002069
:10098000EF3608082A51080881FE0008FC360808DE
:100990000EB400B584B005AB019053F8042B0649A2
:1009A000039301A8FFF7A4FE019B00221A7004B074
:1009B0005DF804EB03B07047E9F80008F7B5114E95
:1009C00007463046002300F84E3F0C460E4B0F49B9
:1009D000002F18BF1946154660F0EAFF0C4F04EBD4
:1009E00045054E36AC4202D10A4803B0F0BD394647
:1009F00034F8022B6846FFF7CBFF6946304660F0BB
:100A0000D7FFEFE738A400200037080809370808A7
:100A10001237080886A40020F7B50C4E0C4F0023AF
:100A200006F87F3F044600EB4105AC4202D109487D
:100A300003B0F0BD394634F8022B6846FFF7A8FF33
:100A40006946304660F0B4FFEFE700BF38A40020ED
:100A500082580808B7A40020F8B5084F4E1E054676
:100A600001F11F0416F8012F28463946FFF790FFC1
:100A7000A64205F10205F5D1F8BD00BF17370808F9
:100A80000246531C084605D1034B1A681B790A60BD
:100A90000B71704701497BE75536080883580808F1
:100AA00010B5013114460EF0EDFE28B9054B1A6859
:100AB0001B792260237110BDC27903492046BDE82D
:100AC000104065E755360808B636080803685A1C12
:100AD000026019700368090A5A1C02601970704795
:100AE00010B402681346511C016013F8021B036026
:100AF000D31C5478036093781B0443EA0423141D29
:100B00000460D0785DF8044B0B4343EA0060704703
:100B1000A0F13003092B07D920F020004138192813
:100B20008CBF002001207047012070473038092811
:100B30008CBF002001207047413819288CBF00204D
:100B400001207047613819288CBF002001207047B0
:100B5000202805D0093804288CBF002001207047C8
:100B600001207047A0F14103192B98BF2030704736
:100B7000A0F16103192B98BF2038704702B310B55C
:100B80008446841803E0981A15D1A44514D01CF8A3
:100B9000013BA3F14100192811F8010BA0F1410E0E
:100BA00098BF2033BEF1190F00F12002EBD91B1AB8
:100BB00004D10028E9D110BD002010BD184610BD99
:100BC0001046704770B5044608460D465DF0C6FEF7
:100BD000064602E014F8013F43B13246294620465A
:100BE000FFF7CCFF0028F5D1204670BD1C462046FB
:100BF00070BD00BF2DE9F043064686469EF800C052
:100C0000BCF1200F7446ACF109050EF1010EF5D0D0
:100C1000042DF3D9BCF12B0F64D0BCF12D0F26D1DC
:100C20000127102A94F801C004F1010423D04FF0E9
:100C3000FF35B5FBF2F502FB05FE6FEA0E0E5FFA1B
:100C40008EFE9046002014F801CBBCF1390F4CF019
:100C50002009ACF1300C29D85FFA8CFC944528DAD5
:100C6000A84226461ED81BD000FB08C0EBE7102A7E
:100C70004FF00007DBD1BCF1300F0AD16078A0F152
:100C80004105192D98BF2030661C78280CBF02340E
:100C900034466FF070454FF00F0E4FF01008D1E75B
:100CA000F445E1D94FF0FF301F40CCE7B9F1600FB8
:100CB0000AD801B10E6067B923B16FF000439842C2
:100CC00028BF1846BDE8F083A9F157095FFA89FCEF
:100CD000C4E723B1B0F1004F28BF4FF000404042BD
:100CE000BDE8F08300279CE773B50E461049054622
:100CF000FEF700FE18B93070012002B070BD2C78EC
:100D0000602C8CBF613C413C082C0FD8013501237D
:100D10000A2201A92846FFF76DFF019BAB4205D0CF
:100D20000F2803D8013440EA0410E4E70020E4E788
:100D30005536080801230A2200215BE770B50D46ED
:100D40001446FFF706F90646A0B1FFF7F3FF40F699
:100D500034039842A8BF1846B0F5617FB8BF4FF47E
:100D60006170A0F561731922B3FBF2F32B70237845
:100D7000013323703046FFF7ECF80646A0B1FFF7C9
:100D8000D9FF40F634039842A8BF1846B0F5617FFA
:100D9000B8BF4FF46170A0F561731922B3FBF2F391
:100DA0006B70237801332370304670BD2DE9F0411C
:100DB00016461F460446394630464FF47A720023E1
:100DC0005EF02AFA3C4D3D4B054483FB0560284408
:100DD000E917C1EB601183FB01030B44384EC817C0
:100DE000C0EB631086FB003CC317364EC3EBAC036D
:100DF00086FB03764FEAE37ECEEBE61EC1EB0116DF
:100E0000A5EB860CC0EB0015A1EB8501617103EB2E
:100E10004301A0EBC10040F2B55101FB1E33B3F515
:100E2000896F84F806C020714FEA8E0633DA40F2EB
:100E3000DA218B4237DCB3F5B77FB4BF4FF0000E39
:100E40004FF0010E204F0EEB4E0107EBC10175462E
:100E5000C88A4FEA4E0808EB0E0C07EBCC0C0CF1DD
:100E6000160C0B2101E03CF8020D984210DD01390F
:100E7000F9D1F044012137F83800A170013306F5AB
:100E8000FA6E1B1A7544E37022812580BDE8F0815B
:100E90000131C9B2F1E703250B4F40F29650AE463F
:100EA0004FF00608D7E70225074F40F22940AE462B
:100EB0004FF00408CFE700BF80BC92C789888888BC
:100EC000ABAAAA2A73B06D16184507080C4B10B5CB
:100ED000D3E9004354EA030209D1014640F2011369
:100EE0000020C1F8023088710880088110BD054AD1
:100EF0001268121943F10003FFF758FF012010BDDB
:100F0000B03E0020281C00202DE9F0410446944208
:100F10001546084609D2B4FBF2F6154B05FB1644FC
:100F20001B5D00F8013BBDE8F081B4FBF2F6964290
:100F3000B6FBF2F70CD20E4B05FB176705FB164408
:100F4000DA5D00F8012B1B5D00F8013BBDE8F08184
:100F5000BA42B7FBF2F807D9054B05FB187813F82E
:100F6000082000F8012BE7E74046FFF7CDFFF3E745
:100F700038C1070870B5884CB4F8D434B4F8D82414
:100F8000B4F8DC14B4F8DE04B3F57A7F88BF4FF40C
:100F90007A7382B088BFA4F8D434B4F8D634B3F5E9
:100FA0007A7F84BF4FF47A73A4F8D634B4F8DA3475
:100FB000B2F57A7F84BF4FF47A72A4F8D824B3F5DF
:100FC0007A7F84BF0023A4F8DA34B1F57A7F50D950
:100FD0004FF47A718842A4F8DC145CD89A429CBF22
:100FE0000023A4F8D83481429CBF0023A4F8DC3449
:100FF000B4F8EC34B4F8EA24684D9A4284BF002374
:10100000A4F8EA34664B1B8803B36979654E01295D
:10101000B27848D9062A55D93179002940F096800E
:101020009FED617A61490A7807EE903A06EE902AC0
:10103000F8EEE77AB8EEE66AB379C6EE276A002BD7
:101040007CD1B4EEE67AF1EE10FA49DC6A78032A34
:101050001DD8574B03EB42132A78C4F8F434032A03
:101060000ED8544BEA2102FB0133534A136002B0FD
:1010700070BDB0F57A7F84BF0020A4F8DE04ADE730
:1010800000224C4B2A704C4A136002B070BD002203
:10109000474B6A70E0E700219A42A4F8DE14A7D813
:1010A000A4F8D814A4E7B1790029B3D0072A61D0F5
:1010B000B3F57A6FAED93D4908780228B8BF02204F
:1010C0000870A7E73D4901EB820191ED187A31796B
:1010D0000029A7D0531F032BB8D9002AB6D03BE074
:1010E00027EE277AFCEEC77ACDED017A9DF8043021
:1010F00007EE903AF8EEE77AB4EEE77AF1EE10FAFE
:10110000C4BF0133DBB29BB3102BA8BF1023DBB2EB
:10111000934238BF13460B7098E73279002A95D175
:1011200022499FED277A0A7807EE903A06EE902A38
:10113000F8EEE77AB8EEE66AC6EE276A37EE077A87
:10114000B4EEE67AF1EE10FA80DDC9E7053A032A3B
:101150007FF67CAF9FED147AB7EE000A80EE070AA7
:101160005FF08EFB3388834228BF034633806DE7F0
:101170000123CCE70622B3F57A6FB270CDD90B49C3
:1011800030790A78022AB8BF02220A7000287FF458
:101190005DAF9FED0B7A46E738A40020B83E0020F3
:1011A00054130010EC2400206F120338FC40002080
:1011B000E0A4002060A50020044100201845070895
:1011C00017B7D1382DE9F04FA74B83B01B78A3F1A7
:1011D0001702022A00AF13D9A44A12F833100029CB
:1011E00040F0AF82DB001A4452784AB1A04A3A601C
:1011F000134493F87C302BB99B4A1823137001E0F9
:101200009B4B3B609B4B9C4E93F808809B4B4FF055
:10121000000A03F154059B461FE09BF90430142B90
:1012200000F00683204660F04FFCA20323D501287E
:1012300000F0FE82082800F3FB82B9F1000F01D014
:10124000344206D1414620465CF0EEF9002800F019
:10125000EF820BF10C0B5D4513D0DBF8004014F06E
:101260000109DAD0204660F02FFC0AF1010AA2033E
:101270005FFA8AFADBD40128DCDC0BF10C0B5D454C
:10128000EBD10AF1FF33022B00F2D2827C4DDFF862
:101290000C920023022085F8503512F075FF95F866
:1012A0005435D9F80040022B00F0CC82002800F021
:1012B0002A83DFF8ECA1734B95F8ADC5C7F804C0DD
:1012C00003F56A7B4FF47A784FF0000E64222646CD
:1012D00033F8081CB1F57A7FB3F8461088BF23F8BD
:1012E000088CB1F57A7F33F8061C88BFA3F84680D6
:1012F000B1F57A7F33F8041C88BF23F8068C33F8E5
:10130000060CB1F57A7F84BF002123F804EC8842F3
:10131000B3F85A00B3F85C1098BF23F806EC884283
:1013200093F86B1088BFA3F85AE00139632993F84A
:101330006C1088BF83F86B200131C9B2092988BFBE
:1013400083F86CE003F16500002113F8314010F8D8
:1013500001CF0131A44538BF80F800E00329F4D162
:101360007968012918BF83F886E0EA339B45AFD13D
:101370003446454EB378042B00F09F8233B933884E
:10138000B3F5F07F84BF4FF4F0733380FFF7F2FDC5
:101390003E4895F8C015FEF7E9FC95F8DF151030CA
:1013A000FEF7E4FCB5F8EE15B5F8EC350B43B5F8EF
:1013B000F0150B431BB213B10123A5F8F235344BE2
:1013C0002340002B00F0AC82E30700F1718260043F
:1013D00000F1C281210740F130822E49DAF8003055
:1013E0000C400B40C9F80040CAF80030230440F11B
:1013F000B981204A0023D373D377E00440F1BD8143
:1014000095F8FF35DFF89080022B04BF012385F8A3
:10141000FF3508F17804434602E006339C420CD0C5
:101420001A780A2AF9D19978DA78914202D35A794E
:10143000002AF2D00A2027F0BBF900234FF4806085
:1014400085F8503512F0A0FE002800F049821249BC
:10145000C7F804A08B468A469AF8050070B39AF83C
:10146000001041B3434620E0703F0020903307084E
:1014700018450708D03E0020BC02020030A9002019
:1014800038A400206AA50020EC24002008AA00202F
:1014900009600002FE9FFFFD3CAA00209445002049
:1014A000CC3E002006339C4208D01A788242F9D103
:1014B0005A79002AF6D0084627F07AF90AF1060A86
:1014C0005445C9D196F80280D7F804A0B8F1080FA6
:1014D000594600F0C78195F8AD35DAF800C0A3F1A0
:1014E0000103B3FA83F35B0985F87C3695F8AE35D2
:1014F000A3F10103B3FA83F35B0985F8823695F80B
:10150000D134032B84BF002385F8D134B04BCCF306
:10151000C0309A7B85F87F06D9F80030AD4803408B
:101520000CEA0000C9F80030CAF80000002A00F0F8
:10153000B781DFF8D892B9F80430002B40F0A481CD
:10154000A54A1368B3F5000F24BF00231360936806
:1015500023F4007323F0020313B140F202239360DB
:101560001379013B042B84BF01231371A8F10508F3
:101570009A4BB8F1030F93F800B040F20F814FF08F
:101580000008BBF1000F25D0DFF884927C605C4638
:10159000CB46894606E0AAF1060AAAEB060A54459C
:1015A00040F2DC80DA461BF8010F0028F3D00EF081
:1015B00091F90028EFD082799307ECD57C684946F1
:1015C0000122B8F1000F05D0737C3BB97379012B70
:1015D00000D01AB1B3790BB10023B371804BDA8814
:1015E00002F00F00042803D8C2F30312022A02D922
:1015F0004FF42062DA801A8902F00F00042803D821
:10160000C2F30312022A02D940F601221A8195F888
:10161000950695F8A12695F89436904205D90022B2
:1016200085F8952653B1A5F8982695F8A0269A42F4
:1016300004D2002385F89436A5F8983695F88A37B1
:1016400095F89626674ED7F800809A4284BF00230B
:1016500085F8963606F18009334613F8032D02EB20
:101660004202424492F854E192F855C192F8560170
:1016700013F801AF9A79F245A8BFF2466245A8BFB8
:1016800062469A71DA7883F800A08242A8BF0246C7
:10169000B342DA70ECD103F120064E45DCD1524B57
:1016A000DA6A002A00F0E880002601200B782B2B54
:1016B00007D14B78043300FA03F313421CBF9A435B
:1016C000012606318C42F1D10EB1474BDA62474C0C
:1016D0006E4604F10808234601E098456FD013F8E0
:1016E000012F072AF9D9002304F8013F0133082B01
:1016F000FAD1B5F8A625B5F8A4359A42B54602D375
:101700003B4BC5F8A4353B4B3B4CFF2285F8BC272F
:1017100003F1540013F9082C142A05D053F80C1CBB
:1017200034EA010100F0C6800C339842F2D1334B09
:101730005A79022A01D100225A710C37BD46BDE800
:10174000F08F02EBC301DB00496800297FF44BAD49
:101750002B481721017046E52A493FE67C68494637
:1017600000222EE7204BDB7B002B00F0C6801E4AB8
:101770000023E004D3773FF543AE21067FF540AE6A
:101780001F4B1978182904D81F4BCB40DA073FF5B7
:1017900037AEDFF8808008F178044EE6002333711D
:1017A0004FF00108BBF1000F7FF4EEAE737C002B0D
:1017B0007FF414AF7379012B7FF410AF0AE788B080
:1017C000E9462022FF21484660F0EAF8074A28E06F
:1017D000B83E0020BDD777180C410020D011001072
:1017E00068440020E5A40020D03E0020FE24002014
:1017F000AE014A013CA9002001000200A024002003
:10180000703F0020F6DFFFFD004100010440002092
:10181000F32400203CAA0020424549F823303FF43D
:1018200068AF12F8013F59F823100131F4D05AE79C
:101830004049414852F042FF28E5A2047FF5D6AD69
:101840003E49CBE500283FF434AD90F904604FF0F9
:10185000FF0801E080F8088030460FF033FF0028D1
:10186000F8D126E5B379002B3FF435AE737C012B1C
:1018700004BF022373742EE62B20796026F098FFB4
:101880002F4B7968DA6A0FE799F8000079600EF05B
:1018900021F8796800287FF453AEA9F804004FE6D8
:1018A000284A13431043C9F80030CAF8000040E644
:1018B000254993E585F8BC2739E7DAF8003023F4A9
:1018C0008053CAF80030338C24F48054B3F57A7F07
:1018D000C9F80040BFF45AAD4FF47A73338455E52C
:1018E000D9F8003023F00063C9F80030DAF800308E
:1018F00023F00063CAF80030A9E542F201031C425C
:101900007FF435AF79E5DFF844A0DAF8003024F051
:10191000800423F08003C9F80040CAF80030CAE40C
:10192000DAF8003043F0080344F00804CAF8003045
:1019300053E500BF30A90020E4600808F6BFFFFDB2
:10194000D03E002000040500F79FFFFDCC3E0020A4
:101950002DE9F04F804B93F8C037013B012B83B04A
:1019600040F2E280DFF81C827C4ED8F80C30DFF8C1
:10197000189203F2DC534E45C8F80C3080F0E98031
:1019800001230193764BDFF804B206F11C059F1C7E
:10199000734B5988002900F0B2807A185A4580F0BC
:1019A000AE803C4608E0118814460A44002900F045
:1019B000A6805A4580F0A380052940F2A08035F822
:1019C0001C3C6188C3F30B039942ECD163799B07FC
:1019D000E9D1238855F8141C94F804A000933046EC
:1019E00052F06CFE35F81C1CBAEB113F00F08D80F4
:1019F0000023019335F8181C55F8140C55F8044CC5
:101A0000C1F30B0157F04CF91C364E45206005F12F
:101A10001C05BDD3534A544B544E1268544C1A60A3
:101A2000FFF7D0FB3178534D7278EA2301FB034373
:101A30002B60A4F1800303EB4213C4F8CC3326F0EF
:101A400089F828684C4D4FF0FF336B6031F008FF88
:101A500026F0F6FE04F2DC4304F2545102E00633B1
:101A600099425CD01A78002AF9D19C78D8788442BF
:101A700002D358790028F2D0374C2A7294F8FC35FA
:101A8000B4F8002603EB830303EB83039B00642B72
:101A9000B8BF6423C8F80430642303FB02F2642A4D
:101AA000B8BF64220023C8E90223C8F82020334AC3
:101AB000A8F82430C8E90433C8E9063388F826308A
:101AC00004F2EC53936234F0A9FC94F8E617B4F8EE
:101AD000E40727F0C3FC43F0F3FC18F01BF894F87C
:101AE000C037013B012B2CD9254A01981268C8F850
:101AF0000C20012388F8253003B0BDE8F08F55F89D
:101B0000141C304652F0DAFD72E7009BA11D9A1FAB
:101B1000304652F009FE00287FF46CAF68E7F27B94
:101B2000003A18BF0122A7E7F8F7E8FC0A4B00F5D6
:101B3000B71000F558700222C3F8DC0783F8E027DD
:101B400010E7F8F7DBFC0223C4F8DC0784F8E03781
:101B5000CAE7012301935DE738A40020F05D08087F
:101B60000040000894450020CC3E0020B83E0020F4
:101B700060A5002004410020340600204817001012
:101B8000281C00201C410020C867080800800008AD
:101B90000121194A10B5032800EB01040346117016
:101BA000E4B218D9FF2825D0144A002341F202419B
:101BB00000E034B10233402B22F8021B04F1FF3461
:101BC000F7D10F4A1344FF2183F8E817BDE810400E
:101BD0000E2012F057BC0B480B49EA2203FB02000F
:101BE0000A4A0B70106031F03BFE28F011F828F023
:101BF000F3F8D9E70023E4E78417001020AC0020B5
:101C000038A4002060A50020B83E00200441002038
:101C1000054BD3F82C28012142F4001283F829182F
:101C2000C3F82C28704700BF38A400207047F8B5CF
:101C3000164D6B78BE2B26D1022229464FF6FF7037
:101C4000FEF79AFA124FAC1C22884AB1A618BE427F
:101C500019D2052A17D92146FEF78EFA3446F3E742
:101C600021460222FEF788FA0222A118FEF784FA22
:101C70000634084B641BA3F8304841F60F53C31ACF
:101C800058425841F8BD0020FCE700BF0040000862
:101C90000080000838A400202DE9F0410768C7F350
:101CA0000D04064688460CB3D8F8005052F040FEAA
:101CB000092840F08680454C236923F44073236152
:101CC000236943F400732361236943F00103236113
:101CD0003D6052F02DFE2369092823F001032361A2
:101CE0006FD133680433336000206CE0384B394ADD
:101CF00093422BD302F58042934226D302F58042D1
:101D000093424CD3344A93424BD902F580329342EA
:101D100049D902F50032934247D902F50032934285
:101D200045D902F50032934243D902F5003293427D
:101D300041D902F5802293423FD9B3F1016F3ED3DE
:101D400005205AF057F859F0C9F9082452F0F0FD6F
:101D5000092821D11D4D2B6923F440732B612B6978
:101D600043F400732B612B6923F0F8032B612B697B
:101D70001C4344F002042C612B6943F480332B6133
:101D800052F0D6FD2B6923F002032B612B69092841
:101D900023F0F8032B6187D04FF0FF3013E01024BD
:101DA000D4E71824D2E72024D0E72824CEE7302433
:101DB000CCE73824CAE74024C8E74824C6E75824BB
:101DC000C4E76FF00200BDE8F08100BF003C0240B4
:101DD0000040000800400008FFFF00082DE9F04126
:101DE000594E3378B12B8AB073D1FFF720FF80F0C2
:101DF0000104E4B2554B564DB3F86331554FADF87D
:101E0000043004F00104BD4265D3002C00F0998039
:101E10000023CDE9073309934F4B05969B1B06938F
:101E20004E4B1A69002A04DA4D4A5A6002F1883290
:101E30005A6001228DF82520F322DA6001A90222DE
:101E400005A84FF000088DF824805BF0ADFE02225B
:101E500001A94FF6FF70FEF78FF93D4D0446BD42D4
:101E600047D3022202A905A80025ADF808505BF06F
:101E70009BFE022202A92046FEF77EF940BAC0432B
:101E8000ADF80C00022205A803A95BF08DFE0898AE
:101E900078B107ABC0F10402294618445FF080FD19
:101EA0009DF9240018B907A905A8FFF7F5FE8DF8DC
:101EB00024009DF8253023B1284A136943F00043DC
:101EC00013619DF92400B0FA80F040090AB0BDE822
:101ED000F08101248EE7A988AB69A868D3F8008057
:101EE000C1F30B0156F0DCFE1C35804518BF012400
:101EF00089E7AE888DF81180C6F30B06B31DADF8E7
:101F00000C302B88C3F30B02ADF80E201B0B0622FE
:101F100003A905A88DF810305BF046FE062203A940
:101F20002046FEF729F9A9680446324605A85BF069
:101F30003BFEA96820463246FEF71EF91C350446D2
:101F40008DE70120C2E700BF0040000818450708E0
:101F5000F05D0808C867080800800008003C0240DF
:101F600023016745F8B5284DFFF72CF995F8C037E0
:101F7000013B012B33D9254E254FF368012203F293
:101F8000DC53F36085F832280324FFF727FF58B1AC
:101F90003B78B12B08D1FFF74AFE013C0BD060B96A
:101FA000FFF71CFF0028F3D1013CEED1052059F0CA
:101FB00021FF59F093F80028F8D095F8C037013B7D
:101FC0000022012B85F8322815D9124B01221968FD
:101FD00086F825200023F16085F83338F8BDF8F73E
:101FE0008DFA00F5B71000F558700223C5F8DC072C
:101FF00085F8E037BFE7F8F781FA0223C5F8DC0778
:1020000085F8E037E1E700BF38A400201C4100203C
:1020100000400008281C002008B50B490B4A01238A
:102020000B709373FFF79EFFFFF792FC084B41F292
:102030000241FF22A3F8E81783F8EA27BDE8084029
:102040000E2012F01FBA00BF84170010B83E002007
:1020500038A4002090F89230DFED6B6A6B4A07EEEF
:10206000903A90F8963005EE103A90F8943004EEDD
:10207000903A90F8953005EE903A90F89830F8EE56
:10208000E77AB8EEC55A04EE103A67EEA67A25EE66
:10209000265AF8EEE44AF8EEE55AB8EEC44A25EEC0
:1020A000275A64EEA64A65EEA65A24EE264AF0B5F3
:1020B000B7EE007A90F8917064EE854A65EEA75A03
:1020C00024EE274A00F16F06014602F11A050024AA
:1020D000B0EE476AB0EE473A137807EE903AF8EE62
:1020E000E77A67EE857A67EE867AFDEEE77A17EE95
:1020F000903AFA2BA8BFFA2323EAE3730B725378C2
:1021000007EE903AF8EEE77A67EEA47A67EE867A01
:10211000FDEEE77A17EE903AFA2BA8BFFA2323EAEE
:10212000E3734B72937803EE903AF8EEE33A63EE82
:10213000A57A67EE877AFDEEE77A17EE903AFA2BEA
:10214000A8BFFA2323EAE3738B72938807EE903AD1
:10215000F8EEE77A67EE847A67EE867AFDEEE77A44
:1021600017EE903AB3F57A7FA8BF4FF47A7323EA5B
:10217000E3738B812B68D5ED007A002BF8EEE77ABC
:102180003FDD90F8973002EE903AF8EEE22AB0EE9A
:10219000436AA2EEE66A63EE863A83EEA76AA2EE8F
:1021A000A66A013465EEA77A67EE877A67EE867ACB
:1021B000FDEEE77A17EE903AFA2BA8BFFA2323EA4E
:1021C000E373BC4206F8013F00DDF0BD012C13D1E2
:1021D00090F8933007EE103A90F89B3006EE103AE4
:1021E000B8EEC77AB8EEC66A27EE267A26EE266AD9
:1021F0000435083208316FE7B7EE007AB0EE476A6F
:10220000F6E7B7EE006ACCE70AD7233C7E4607081C
:1022100090F899306BB3B0F864308BB190F89A2095
:1022200002EB82036421C3EB0313B3FBF1F3A0F8C9
:102230006430962312FB03F3B3FBF1F3A0F866308E
:1022400043884BB190F89A3003EB8303C3EB03133D
:102250006422B3FBF2F34380B0F850304BB190F8F6
:102260009A30962213FB02F36422B3FBF2F3A0F838
:102270005030704790F821304BB3438B83B190F8C6
:102280002230FA2213FB02F203EB8303B3F57A7FC9
:10229000A8BF4FF47A7364218383B2FBF1F24283C7
:1022A000838843B190F82230FA2213FB02F36422B0
:1022B000B3FBF2F38380C3884BB190F8223003EB79
:1022C0008303B3F57A7FA8BF4FF47A73C380704756
:1022D00070B50B4C002504F56A7694F8913013B173
:1022E0002046FFF7B7FE2046FFF792FF0135304644
:1022F000FFF7C0FF042D04F1EA04EED170BD00BF6A
:1023000060A5002010B5064C4FF48072002104F641
:1023100034005FF045FB0023C4F8343910BD00BF22
:1023200038A40020034BD3F8380908B10AF05CBB8D
:10233000704700BF38A4002008B50B460549024687
:10234000D1F8380928B10449FEF7D2F9BDE80840B0
:10235000E8E708BD38A4002081FE0008024B0146D2
:10236000D3F83809FDF78EBD38A400200048F5E702
:10237000274C08080CB4C30607B500D561B904980A
:1023800005A90191FFF7D8FFFFF7F0FF012003B087
:102390005DF804EB02B070470020F8E70FB407B512
:1023A00004A951F8040B0191FFF7C6FFFFF7DEFF08
:1023B00003B05DF804EB04B070470349034801F52E
:1023C00021610EC9EAE700BF0070FF1F1C37080833
:1023D00070B5134C134D144E002294F8F33403F0EF
:1023E000010302B170BD002BFCD001212846FFF78C
:1023F000D5FF752034F056FC01463046FFF7CEFF7E
:102400001A2034F04FFC01460848FFF7C7FF1B2095
:1024100034F048FC01460648FFF7C0FF0122DCE724
:1024200038A40020303708083C3708084F37080820
:102430006237080808B5FFF791FFBDE8084095E747
:102440002DE9F04385B0FCF7E1FB0269838901883F
:102450000292826801924288009242681B4EDFF825
:102460008080DFF880901A4F04461A48FFF796FFE5
:10247000002515B91848FFF7DDFFD8F800309D4258
:1024800013DA3378052B96BF09EB83030022D3F8C8
:102490008C21B38800937388294638460135FFF7AD
:1024A0007DFF062D06F10606E3D157F027FB428893
:1024B000838864689B1A03FB0444FCF73FFC0246D4
:1024C0000648214605B0BDE8F04367E774AD00203B
:1024D000DF37080875370808D3370808EE370808CB
:1024E000543900201845070810B504460348FFF783
:1024F00035FF2046BDE810409CE700BF0B380808B8
:1025000008B5034610460AB9002008BDDB0601D510
:102510000029FAD0FFF7E8FFF6E72DE9F04F0A4669
:102520008DB000218346FFF7EBFF714CDFF8CC91B3
:10253000039004F1800A0025A37A99F80060AB4269
:1025400000F3938010345445F5D140F2162052F038
:102550009FF8D0E902450DF1180A002E4FF0150240
:102560004FF00001504604BF254634465FF018FA8C
:1025700000272E78002E3ED06978059130460DF068
:1025800081F995F90290049009F1010253425341F7
:10259000002C00F0A98005990022A05CB04240F018
:1025A0009F80224492F90280C14540F09780527882
:1025B0008A4208BF012301220AF8072003F0010321
:1025C00083F00101039A05935846FFF799FF059B95
:1025D000039044B1474A0499CDE900B230464246DF
:1025E000FDF73CFD059B444A0499CDE900B2304615
:1025F0004A46FDF733FD0137152F05F10305B8D124
:1026000084B3DFF8F080DFF8F090564604F13F071E
:1026100016F801ABBAF1000F21D12078F8B194F986
:10262000023001331BD061780DF02CF9039A054676
:1026300001215846FFF764FF94F9022003905346A6
:1026400020782946CDE900B8FDF708FD20785346EB
:10265000CDE900B94FF0FF322946FDF7FFFC033406
:10266000BC42D5D10DB0BDE8F08FE08852F010F833
:10267000D0E90231627A207A002E08BF194605FBA4
:10268000002208BF33468F562BB39E56039A0493FD
:10269000B74214BF0121002158460CBF4FF001087A
:1026A0004FF00008FFF72CFF049B039043B1114B40
:1026B0003246CDE900B3294643462046FDF78AFC61
:1026C0000D4B2946CDE900B33A4643462046FDF777
:1026D00081FC013530E74FF0FF36D7E700236AE78A
:1026E00003323F2A7FF459AF4FF0FF3868E700BF4D
:1026F00040060020792801087523010838A400202D
:1027000010B508460749FDF7F5F8002815BF012464
:10271000002405480548FFF7E7FE2046BDE81040C5
:1027200009F036BF1038080819380808403808087A
:102730002DE9F04F07468BB040F216200C4651F0C1
:10274000A7FF2246054600213846FFF7D9FE424B37
:10275000D5E902451B78002B08BF254606464FF0F9
:1027600015024FF0000104A808BF1C465FF018F9DD
:1027700005F13F03039395F80090B9F1000F31D0B4
:1027800095F801A0002C65D0224600231178494518
:1027900058D128336B4492F80180012203F8182C99
:1027A000D045324614BF0121002138460CBF4FF0FE
:1027B000010B4FF0000BFFF7A3FE064654B1B8F132
:1027C000000F07D0254B00935A463B4641464846EA
:1027D000FDF78AFC224B00935A463B465146484639
:1027E000FDF782FC039B03359D42C4D13CB3DFF867
:1027F0006C90DFF86CA0651C0DF11008403418F8DF
:10280000013BCBB915F8013CB3B116B13046FFF727
:102810006BFE297815F8010CCDF800903B4600229C
:10282000FDF762FC002215F8010CCDF800A03B4634
:102830001146FDF759FC00260335A542DFD10BB048
:10284000BDE8F08F0133152B02F103029ED14FF04A
:102850000008A5E7A046A3E738A4002079280108CE
:1028600075230108034B0146D3F8380908B10AF073
:10287000A7B8704738A400200CB407B510F02000AA
:102880000BD079B92320FFF7EDFF049805A901913A
:10289000FFF752FDFFF76AFD012003B05DF804EB7E
:1028A00002B070470020F8E72DE9F04F914687B05D
:1028B0000C461A4600218046FFF722FE4D4606468A
:1028C0000027B9F1000F66D02946062220465FF0A6
:1028D000EBF80028324614BF0121002140460CBF0E
:1028E0004FF0010A4FF0000AFFF70AFE064628786B
:1028F00017F0D8F88346F8B1687917F0D3F8AB78B9
:10290000EA789BF805E095F801B04FF461714FF05B
:10291000190C1CFB03131CFB0212297900B140792E
:10292000CDE90410CDE90232CDE900EB1B4A3B466C
:1029300051464046FFF7A0FF207817F0B3F88346D2
:10294000F8B1607917F0AEF8A378E2789BF805E06B
:1029500094F801B04FF461714FF0190C1CFB031394
:102960001CFB0212217900B14079CDE90410CDE9B8
:102970000232CDE900EB094A3B4651464046FFF79B
:10298000F9FC0137142F04F1060405F1060598D16E
:1029900007B0BDE8F08FCA46CEE700BF5C38080834
:1029A0002DE9F04F904689B01A460C460021814629
:1029B000FFF7A6FD3B4EDFF8F0B008F154030746E1
:1029C0004546079394F904000EF07CFE00285DD084
:1029D000B8F1000F63D029460C2220465FF064F85E
:1029E00000283A4614BF0121002148460CBF4FF091
:1029F000010A4FF0000AFFF783FD074695F904002E
:102A000054F0E4FFEA7906EB82020346D2F8A421EF
:102A100004922A7A06EB82025146D2F8A42103924C
:102A2000AA7906EB82024846D2F8A42102926A797A
:102A300006EB8202D2F8A42101922A6800925A463B
:102A4000FFF71AFF94F9040054F0C0FFE27906EB97
:102A500082020346D2F8A4210492227A06EB820273
:102A60005146D2F8A4210392A27906EB820248468D
:102A7000D2F8A4210292627906EB8202D2F8A42154
:102A80000192226800925A46FFF774FC079B0C35AE
:102A9000AB4204F10C0495D109B0BDE8F08FC246F9
:102AA000D0E700BF18450708753808082DE9F04F32
:102AB00090468BB00C461A4600210746FFF720FDD2
:102AC0004546099000264FF0190A4FF46179B8F194
:102AD000000F4BD029460A2220465EF0E5FF002871
:102AE000099A14BF0121002138460CBF4FF0010B99
:102AF0004FF0000BFFF704FD2A890692EA88059241
:102B00002A790492EA780392AA7809901AFB029231
:102B100002926A781AFB029201922A780092334656
:102B2000134A59463846FFF7A7FE22890692E288E3
:102B3000059222790492E2780392A2781AFB02921B
:102B4000029262781AFB0292019214F80A2B009208
:102B50003346074A594638460136FFF70BFC1E2E0E
:102B600005F10A05B3D10BB0BDE8F08FC346DCE731
:102B7000923808082DE9F04F2DED088BDFF828A1D9
:102B800095B0804691461E460C461546002794EDAA
:102B9000008AB5EE408AF1EE10FA7DD0D4ED019AAC
:102BA00094ED029AD4ED038AB9F1000F49D0D5ED26
:102BB00000BA95ED01BAD5ED02AA95ED03AAB4EEDF
:102BC0006B8AF1EE10FA6CD1F4EE4B9AF1EE10FA3A
:102BD00067D1B4EE6A9AF1EE10FA62D1F4EE4A8A45
:102BE000F1EE10FA0CBF0121002132468B4640461F
:102BF00081F00101FFF784FCB0EE6B0A064611A8D4
:102C0000FDF7CEF8B0EE4B0A07900EA8FDF7C8F816
:102C1000B0EE6A0A06900BA8FDF7C2F8B0EE4A0AB9
:102C2000059008A8FDF7BCF80599069A079B039044
:102C300002910192009352463B4659464046FFF7A7
:102C40001BFEB0EE480A11A8FDF7AAF8B0EE690A1B
:102C500083460EA8FDF7A4F8B0EE490A06900BA82B
:102C6000FDF79EF8B0EE680A059008A8FDF798F801
:102C7000069B059A0390CDE900B302923B4652466B
:102C8000002140460137FFF775FB082F04F11004BF
:102C900005F110057FF47BAF15B0BDEC088BBDE8E6
:102CA000F08F0021A1E700BFB53808082DE9F74FE4
:102CB00092460C461A4600218146FFF721FCDFF8B8
:102CC00070B0804656460025BAF1000F2ED031462E
:102CD000042220465EF0E8FE0028424614BF01218F
:102CE000002148460CBF01270027FFF709FC738825
:102CF00001933AF82530009380462B465A463946D0
:102D00004846FFF7B9FD6388019334F8043B00930C
:102D10005A462B46394648460135FFF72BFB042D12
:102D200006F10406D0D103B0BDE8F08F5746EAE7BC
:102D3000C93808082DE9F04F89468FB017460021A1
:102D40001A460646FFF7DCFBDFF874A005460024B0
:102D50000DF1240B59F82480CDF80880594602A8BB
:102D600054F0E2FD57B357F82430039398452A46B0
:102D700014BF0121002130460CBF4FF001084FF075
:102D80000008FFF7BDFB04A9054603A854F0CCFDDD
:102D900004A900912346524641463046FFF76CFD98
:102DA0002346CDF800B05246414630460134FFF785
:102DB000E1FA202CCED10FB0BDE8F08FB846EFE796
:102DC000DA3808082DE9F04F924685B00C461A46CD
:102DD00000218146FFF794FBDFF874B0804655462A
:102DE0000026BAF1000F31D02946042220465EF0B9
:102DF0005BFE0028424614BF0121002148460CBF5B
:102E000001270027FFF77CFBEB780293AB78019357
:102E10002B880093804633465A4639464846FFF78A
:102E20002BFDE3780293A378019334F8043B0093DD
:102E30005A463346394648460136FFF79BFA102E6C
:102E400005F10405CDD105B0BDE8F08F5746E8E7A0
:102E5000E43808082DE9F04F85B0144602911A466F
:102E600000210546FFF74CFB4FF0000806460623FD
:102E700003FB08F7C0374FF00009029B13F807B0B7
:102E8000002C7ED0E35D03939B45324614BF0121A5
:102E9000002128460CBF4FF0010A4FF0000AFFF74F
:102EA0002FFB039B394ACDE9009306464346514622
:102EB0002846FFF7E1FCCDE9009B344A43465146E2
:102EC000284609F10109FFF755FAB9F1060F07F194
:102ED0000107D2D108F10108B8F1060FC7D1E427E4
:102EE000029BA7F1E40913F807A0002C4BD014F8BB
:102EF00007B0DA45324614BF0121002128460CBF35
:102F00004FF001084FF00008FFF7FAFACDE9009BF7
:102F100006461E4A062341462846FFF7ADFCCDE98A
:102F2000009A1A4A0623414628460137FFF722FA3B
:102F3000EF2FD5D1029B93F8EF70B4B194F8EF80E6
:102F40004745324614BF0121002128460CBF012409
:102F50000024FFF7D5FA002300930C4ACDF8048033
:102F6000072321462846FFF787FC00230093074AE2
:102F70000197072321462846FFF7FCF905B0BDE875
:102F8000F08FA24697E7A046C9E700BFF6380808C9
:102F90002DE9F04F0E46154689B01A460021044629
:102FA000FFF7AEFAB04681462F464FF0000B002DDA
:102FB0007CD039460C2240465EF076FD00284A4619
:102FC00014BF0121002120460CBF4FF0010A4FF031
:102FD000000AFFF795FA97F90B20049297F90A2057
:102FE0000392B7F908200292B7F906200192B7F9C7
:102FF000042000928146384A5B4651462046FFF73E
:103000003BFC98F90B20049298F90A200392B8F936
:1030100008200292B8F906200192B8F90420009223
:103020005B462D4A514620460BF1010BFFF7A2F9F2
:10303000BBF1080F08F10C0807F10C07B7D1DFF856
:103040009C804FF0000B0C2303FB0BF985B300278A
:1030500055F8090056F80920012303FA07FA4240FF
:103060003AEA020214BF1946002110EA0A0F07D0FB
:1030700000975B46424620460791FFF7FDFB079904
:1030800056F809201AEA020F05D000975B4642461F
:103090002046FFF76FF901370E2FD9D10BF1010B45
:1030A000BBF1080FCFD109B0BDE8F08FAA46A8E761
:1030B0002F4656F80910012303FA07F20A4206D0F8
:1030C00000975B46424601212046FFF753F901373E
:1030D0000E2FEED1E2E700BF0A39080822390808AE
:1030E0002DE9F04F89468DB0164600211A46074655
:1030F000FFF706FADFF8DCA005460024C4EBC403A2
:1031000009EB030259F8030091889279089040F383
:103110000748ADF824108DF82620B8F1000F54D0E0
:10312000002E55D0F218F058918893790A90ADF896
:103130002C1007220AA908A88DF82E305EF0B4FCE6
:1031400000282A4614BF0121002138460CBF4FF049
:10315000010B4FF0000BFFF7D3F99DF82E300693CB
:103160009DF92D3005939DF92C3004939DF82B305B
:1031700003939DF92A3002939DF8293001939DF81D
:103180002830009305462346524659463846FFF7F5
:1031900073FB9DF8263006939DF9253005939DF924
:1031A000243004939DF82330CDE902839DF821302B
:1031B00001939DF8203000935246234659463846E5
:1031C0000134FFF7D7F8102C98D10DB0BDE8F08F7F
:1031D000B346DEE7373908082DE9F04F924689B04B
:1031E0000C461A4600210746FFF78AF90026079089
:1031F0005546B3464FF019094FF46178BAF1000F04
:1032000028D02946062220465EF04EFC0028079A68
:1032100014BF0121002138460CBF4FF0010B4FF0C5
:10322000000BFFF76DF96A79079019FB028205928E
:103230002A7919FB02820492EA780392AA78029210
:103240006A7801922A7800923346124A59463846E3
:10325000FFF712FB627919FB02820592227919FBB2
:1032600002820492E2780392A2780292627801923A
:1032700014F8062B00923346064A59463846013662
:10328000FFF778F80A2E05F10605B7D109B0BDE8B9
:10329000F08F00BF543908082DE9F04F0F468BB06E
:1032A000144600211A460646FFF72AF90546002C67
:1032B00000F0DD8022783B789A4218BF0121024657
:1032C00008BF002130460CBF4FF001084FF0000846
:1032D000FFF716F923789E4A054641463046FFF728
:1032E000CBFA3B789A4A41463046FFF743F8002C28
:1032F00000F0BF8062787B789A4218BF01212A468D
:1033000008BF002130460CBF4FF001084FF0000805
:10331000FFF7F6F863788F4A054641463046FFF7D7
:10332000ABFA7B788B4A41463046FFF723F807F12A
:10333000C9030593A31C0693822307F1020A04F133
:10334000CA0B07934FF000093B784B4500F393807D
:10335000002C00F0F68097F8EA3094F8EA209A42C0
:1033600018BF01212A4608BF002130460CBF4FF08C
:1033700001084FF00008FFF7C3F894F8EA30764AE6
:10338000054641463046FFF777FA97F8EA30724A29
:1033900041463046FEF7EEFF002C00F0D48004F1E9
:1033A000EA0307F1EA0204F1FA014FF0010833F8E9
:1033B00002CF32F8020F844518BF4FF0000899423F
:1033C000F5D188F001012A46C9B23046FFF798F8D6
:1033D0000821054604F1EC00FDF71EFB5F4A034699
:1033E00041463046FFF748FA97F8EA1007F1EC003B
:1033F000FDF712FB594A034641463046FEF7BAFF35
:10340000002C00F0A2804FF0FC094FF0010807EB00
:10341000090104EB0900FCF76DFA09F10409002821
:1034200018BF4FF00008B9F58E7FF0D188F0010188
:103430002A46C9B23046FFF763F8082104F1FC00C0
:10344000FCF79AFD464A034641463046FFF714FA18
:1034500097F8EA1007F1FC00FCF78EFD404A03469E
:10346000414630460BB0BDE8F04FFEF783BFA046A3
:1034700037E7A04655E7079BFB180993002C5ED061
:10348000079B0998E31819460893FCF733FA059B44
:103490005A789BF800309A42069A06BFB0FA80F834
:1034A0004FEA58184FF00008AAF10203023A0AF155
:1034B0000E0133F802CF32F8020F844518BF4FF0E7
:1034C00000088B42F5D188F001012A46C9B2304686
:1034D000FFF716F86278069905469BF81800FDF785
:1034E0006DFA02909BF800300193089B00931D4AEF
:1034F00009F1010341463046FFF7BEF9059B7A7892
:10350000587E5146FDF75AFA059A029012F8013F8B
:10351000019309F10109099B05920093114A4B4659
:1035200041463046FEF726FF069B10330693079B65
:1035300009330AF1100A0BF1010B079304E7A046C7
:10354000DCE7A04621E7A0464EE7A04680E700BFA3
:103550006D3908087F390808AD390808C5390808E9
:10356000DC390808943908082DE9F04F89B00F4676
:1035700090460021139A03930646FEF7C1FF87EA9F
:1035800008086FEA0803DFF88490069304460025D4
:1035900028460EF035F8129B184230D0069BDFF813
:1035A00070B0034014BF4FF0010A4FF0000A0493BB
:1035B00010EA07030CBF4A465A462846059307926D
:1035C0000EF030F8039B079A009080465146304633
:1035D000FFF752F9049BB3FA83F1224649093046BA
:1035E000FEF78EFF059A039BCDF800800446002A63
:1035F0000CBF5A464A4651463046FEF7BBFE0135DF
:10360000172DC5D109B0BDE8F08F00BFF339080808
:10361000C33808082DE9F04F0A4689B00021054655
:10362000FEF76EFF384C059094F9000009F088FE13
:103630008146608851F02CF8344BD0F808B01F78E0
:1036400017B15F46D0F80CB0A379012B38BF012326
:10365000069300262279637906FB02331BF8038068
:10366000002F3BD0FB5C059A0793434514BF012113
:10367000002128460CBF4FF0010A4FF0000AFEF768
:103680003FFF079B0590013653B303F00F021B0960
:103690004033CDE9006302924B461D4A514628460D
:1036A000FFF7EAF8B8F1000F24D008F00F034FEA53
:1036B0001818029308F14003CDE90063144A4B4601
:1036C00051462846FEF756FE069BB342C2DC114B1C
:1036D0000834A342A8D109B0BDE8F08F3B46C2E749
:1036E000002FDFD00C4A00964B4651462846FFF784
:1036F000C3F8D7E76B06E7D4074A00964B46514616
:103700002846FEF737FEDFE7FC46070838A400200E
:10371000FA39080854480708103A08080FB407B5E2
:1037200004A951F8040B0191FEF706FE03B05DF801
:1037300004EB04B070472DE9F041037903F0E00297
:10374000402A4DD009D83ABB03F00703052B1ED8F9
:10375000DFE803F0181D181D0910602A47D0802AE1
:1037600041D0BDE8F081D0F805102348BDE8F04114
:10377000FEF714BED0F8052051422048BDE8F041C4
:10378000FEF70CBEB0F80720B0F80510F5E7B0F969
:103790000720B0F90510F0E74679194D194805EBF7
:1037A000C605FEF7DBFD95F8407300240123A74210
:1037B00003D8BDE8F041FEF7D9BDD5F83C6356F813
:1037C00024204FEA84084AB113B90F48FEF7C6FD1A
:1037D00056F808100D48FFF7A1FF00230134E6E773
:1037E00041790B48C2E7827941790A48C6E7BDE8CA
:1037F000F0410948FEF7D2BD243A08083A3A0808D1
:1038000018450708513A0808E83B0808E750080837
:10381000623A0808733A08088A3A0808194B1B6884
:103820002DE9F04163B31848184FDFF86880FEF7C0
:1038300001FEFEF777FDFBF7F9F90025FBF736FAF5
:10384000044648B1132010F01DFEFEF78FFDBDE8C1
:10385000F0410F48FEF7EEBD3B78012BF2D0404619
:10386000FFF75CFF792D05F1010602D1FEF77EFD21
:103870002646FEF757FD6420F7F742FA3546DDE7A6
:10388000BDE8F08194220020A23A08085E390020A9
:10389000BC3A0808B15108082DE9F047B74BB849C0
:1038A0001A68B848B84BB2FBF3F296B0FFF736FF90
:1038B000B64BDFF8A0C30FCBDCF808700AAD85E883
:1038C0000F00390748BFDCF80440B14B05934FEABD
:1038D000970EB04B069348BFC4F3805416AB1EF04E
:1038E000020F18BF03EB8404C7F3810603EB8606BF
:1038F00018BF54F8442CA84C08BFA84A56F8301CEE
:10390000A748A84DA84FFFF709FFB4F860294FF466
:103910007A73B2FBF3F103FB11220A20B4F9623986
:1039200092B2B2FBF0F2A148FEF738FDA04AA149DD
:10393000A148FFF7F3FEFEF719FDA04BA04A997BC3
:10394000A04BA14805EB8101D31AD1F81C15B4F89E
:103950003028FEF723FDFEF709FD9C48FEF7FEFC2C
:1039600094F864199A48FFF7D9FE9A48FEF7F6FCD6
:10397000994B94F865191A88984892B2FFF7CEFED1
:10398000FEF7F4FC96499748FFF7C8FE4FF0000891
:103990004646DFF8C49294F8EF3403F00103B8F11F
:1039A000000F00F05D81002E40F08E818E48FEF702
:1039B00041FD8E4FD4F86C89DFF8A092012607F103
:1039C000180A0123B34013EA080F15D019F806208E
:1039D00057F826305AF8261053F822208448FFF76B
:1039E0009DFE012E06D1834B93F8211011B1824820
:1039F000FFF794FEFEF7BAFC0136062EE1D17F48B0
:103A0000FEF7ACFC7E4B1B681B0640F1918194F8DD
:103A10008C39032B8CBF7B487B48FEF79FFC94F8C6
:103A20005435022B40F053817848FEF797FC94F808
:103A30008C39042B00F273817548FEF78FFC94F8E3
:103A40009C39002B00F0728105EBC303D3F8B81545
:103A50007048FFF763FEFEF789FC6F4B6F481E68E6
:103A60006F4B1B7805EB8303D3F8EC15FFF756FE7D
:103A700026B1327A717A6B48FFF750FEFEF776FC7A
:103A8000FBF7C4F8016921B182686748120DFEF79F
:103A900085FCFEF76BFC654B654819684FF47A733B
:103AA000B1FBF3F1FFF73AFE07A8FDF70FFA38B1C3
:103AB00007A90EA85AF0E6FD5E480EA9FFF72EFEF4
:103AC000FEF754FCD4F8288AB8F1000F00F03481D6
:103AD00007EE908ADFED586AB8EEE77AC6EE877A8D
:103AE000FDEEE77A17EE903A544F97F8A80130B1FF
:103AF000534A039392ED250A5CF0C2FE039BD4F86F
:103B0000A8695EB107EE906ADFED4B6AF8EEE77ADE
:103B100086EEA77AFDEEC77A17EE906A354AB2F8BC
:103B200070106429A8BF6421CDE9000642464548CB
:103B3000454EFEF733FCB7F8AC2144486423B2FB92
:103B4000F3F103FB112297F8BD3105EB830592B227
:103B5000D5F80036009397F8BC31FEF71FFC3C48BF
:103B6000FEF7FCFBD4F82C480125002C40F0E68041
:103B7000FEF7FCFB16B0BDE8F08700BF1C1D00205F
:103B8000CA3A0808D43A080840420F00244A0708F5
:103B9000E63A0808EB3A080838A40020294C08083F
:103BA000F03A08081845070854130010F83A0808B6
:103BB000F0FF0010000800001A3B0808B83E002083
:103BC00000800008004000082C3B0808433B080820
:103BD000553B08085D3B0808D02500205F3B0808DE
:103BE000733B0808783B0808973B08089C4A07087D
:103BF00002490808841700109C3B0808A03B0808ED
:103C0000CC3E0020A63B0808B23B0808C23B08088F
:103C100031540808063C0808E4440020223C080807
:103C2000E04400202B3C0808353C0808281C0020F4
:103C3000503C08086A3C08080024744930B500204C
:103C4000340600207D3C0808123C0808C33C0808E4
:103C5000E83C080800380240E83B0808C00600209D
:103C6000002B3FF4A0AE16B14846FEF777FB3B4869
:103C70000121FFF753FD94F86839394805EB8303B8
:103C8000D3F82415FFF74AFD97F8CE33DA0702D5AB
:103C90003448FFF743FD97F81831032B09D0324819
:103CA000FFF73CFD97F81831012B02D12F48FFF7A1
:103CB00035FDFB6C5B7B0126B342B0467FF66BAEF5
:103CC0002B48FFF72BFD64E6FEF750FB71E6022060
:103CD00010F07AFA064608B92648A6E690F90400DC
:103CE00053F074FE074641F0D5FB05EB80003946E2
:103CF000D0F8A4212048FFF711FD94F85735012B87
:103D000004D11E48FEF72AFB1D488EE6B3791D48F4
:103D100005EB8303D3F8A411FFF700FDF4E794F853
:103D200056350BB9184888E6184886E618498FE6D4
:103D30001848FEF713FB8EE64346D5E694FAA4F046
:103D4000B0FA80F005FA00F024EA00040DF03EFC21
:103D500001463046FFF7E2FC07E700BF7D3B08085D
:103D6000123C0808DB400808823B08088A3B080828
:103D70008F3B0808C83B0808D23B0808E23B08080C
:103D8000E73B08088E380808EB3B0808FB3B0808AF
:103D9000C23A0808163C08082DE9F04FDFF8708198
:103DA00098F8033099B0002B00F094804F48504EA3
:103DB000DFF860B1DFF86091DFF860A1FEF73AFB51
:103DC00000252F460BA9E8B216F022F99DF83430F1
:103DD000002B53D0139C54B107EE904A9FED450A37
:103DE000F8EE677A80EE270A5CF04AFD04460B9AEB
:103DF00029465846FFF792FC109A002A6CD002FB25
:103E000004F04FF47A73B0FBF3F30993DDF848C084
:103E1000BCF1000F62D00CFB04F142F21073B1FB55
:103E2000F3F198F80330082D18BF7F18002B57D0F6
:103E30001798079015980690169805900A231198E0
:103E40004FF47A7EB0FBFEFE0998CDF810E0B1FB8E
:103E5000F3FE03FB1E11CDE902E10999B1FBF3F179
:103E600003FB1100CDE90010BCFBF3F321465046E3
:103E7000FEF794FA0023C6E90D33B3620135242D11
:103E800006F140069ED198F8033003B31A4C1B4844
:103E9000D4E970124FF47A73D208B1FBF3F3D4F87B
:103EA000C811FEF77BFA0A22154897FBF2F102FBD4
:103EB0001172FEF773FA134B1B78432B04D1D4E92C
:103EC00073211148FEF76AFA0023C4F8C83119B00B
:103ED000BDE8F08F0D486AE7099297E76146A0E7D1
:103EE00021464846FEF75AFAC4E700BFFE3C0808E0
:103EF000D8AD00208096184B30B50020A53D0808AD
:103F0000C53D080882240020E93D08085C3D0808FA
:103F1000B83E0020663D080889400808753D08083D
:103F200010B586B0104B0493104B0393104B0293C3
:103F3000104B0193104B1149114A00930446114B49
:103F40001148FFF7EBFBFEF711FA10491048FEF796
:103F500025FA3CB10F4A1049104806B0BDE81040A0
:103F6000FEF71CBA06B010BD533E0808583E0808BC
:103F7000623E08086B3E0808773E08081D3E0808A8
:103F8000133E0808BF3E0020283E0808813E08086E
:103F9000893E08089A3E0808A23E0808A63E08087E
:103FA0000120BDE770B52348FEF7D8F9224B93F8FE
:103FB000A831002B38D0214B93ED250A5CF060FC32
:103FC00001461F48FEF7EAF91E4C1F48FEF7C6F9E6
:103FD0001E4B94F821001E4A00280CBF10461846BC
:103FE000FEF728FA94F8213013B31A4C1A48B4F8A3
:103FF00006111A4E1A4DFFF791FB94F804010028A0
:104000000CBF30462846FEF715FAB4F808111548DB
:10401000FFF784FB94F8050100280CBF30462846C2
:10402000BDE87040FEF706BA0F48FEF703FACBE78B
:1040300070BD00BFE33E080830B500203406002004
:10404000FD3E0808D03E00200C3F08089F3A0808B3
:1040500093590808841700101D3F0808DC3E080823
:10406000D33E0808443F0808023F080838B50B4D06
:1040700005EBC0050C4695F9E40109F061F901462C
:104080000748FFF74BFB95F8EA3133B1611C05484F
:10409000BDE83840C9B2FFF741BB38BD1845070835
:1040A000E7500808825808082DE9F04F6B4B1B7841
:1040B00087B0002B00F0CB80694D6A48A968FEF7F5
:1040C0006DF969686848FEF769F9684B6848D3E993
:1040D0000031C91A674B1A68B1FBF2F2FEF75EF9BC
:1040E000FEF744F96448FEF7A5F96448FEF7A2F923
:1040F0004FF00008624B1B785FFA88F4A34222D885
:10410000FEF734F95F4D604E002455F8041F304629
:104110000134FFF703FB162CF7D1FEF727F95B4DAF
:10412000594E01242B4669681B683046C91A013470
:10413000FFF7F4FA162C05F10405F3D107B0BDE83A
:10414000F04FFEF713B9524B142603EB840306FB22
:10415000045693ED450AB6F80E905CF091FB96F884
:104160001EA01AF0010F0CBF2D2252221AF0020FCE
:104170000CBF2D2354231AF0040F0CBF4FF02D0C4D
:104180004FF0560C1AF0080F0CBF4FF02D0E4FF0E9
:10419000430E81B21AF0800F4FF03C0BB1FBFBF1E4
:1041A00005914FF064010CBF4FF02D0A4FF0530AF8
:1041B00080B201FB09F1671CCDE902A10490CDE9B1
:1041C00000CE34483946FFF7A9FAB37FDB073AD56A
:1041D0005C23314A6343D118D05891ED010A70B184
:1041E000DFED2E7AB8EE400A20EE270A07EE900A9D
:1041F000F8EE677A80EE270A5CF042FB00B2642298
:1042000090FBF2F102FB11022548FFF787FA142117
:1042100001FB075701FB0454F988628A0491218B42
:104220000391E18A0291A18B0191A18A009102F090
:10423000030319214B431B48218A9208FEF7AEF86D
:1042400008F1010856E71848FEF788F8DFE7174835
:1042500007B0BDE8F04FFEF7EDB800BF0400001056
:10426000EC0D0010643F0808743F0808000B0010B4
:104270008B3F0808301C0020B83F0808144008088D
:10428000D0110010940E0010C4400808980E0010C1
:1042900084170010704008080C0B001000401C46EA
:1042A0008D400808A240080899400808C84008083E
:1042B0000EB403B503AA52F8041B0192FCF73BFBB2
:1042C000064BD3F838291AB90549986CFBF7DAFD83
:1042D00002B05DF804EB03B0704700BF38A40020C3
:1042E000274C08082DE9F04798460B7903F0E005C4
:1042F000402D81460F46164632D1644DDFF8A88125
:10430000DFF8B091002416E03B7903F00703013B8E
:10431000042B04D8DFE803F014171A1D2100315DC7
:104320005A48FFF7FBF97B79013BA34202DD48467F
:10433000FEF714F801347B79A342E5DCBDE8F08791
:1043400031572846EDE736F81410FAE736F914101D
:10435000F7E756F824104046E3E756F82410F0E754
:1043600003F00703052B57D8DFE803F0031F2729C5
:104370002C3E3478602D55D02CD8002D75D1B7F84F
:104380000550B7F8076041482146FFF7C7F9AC422E
:1043900039DBB44237DCB8F1000FCFD032462946C2
:1043A0003B48BDE8F047FFF7B9B996F90040602DEA
:1043B00038D00FD8002D58D151E03488DAE7B6F95B
:1043C0000040F4E7D6F800A0202D54464DD034D953
:1043D000602D27D0802DB1D132782E4B2E48002A67
:1043E00014BF3146194635E0202D34683DD0EFD852
:1043F00021462648FFF792F9D7F80510A14202DBC3
:104400004B42A34221DDFDF7B1FF3A682349234621
:104410004846BDE8F0474BE7202D25D01ED9602D3A
:10442000D8D100247B7944FA03F3DB07BDE8F047D9
:104430004CBF1B481B48FFF771B951461A48FFF79C
:104440006DF9D7F805108A45DDD8B8F1000F3FF4B3
:1044500075AF1648BDE8F047FFF760B90024B7F91B
:104460000550B7F907608EE700247A79104B03EB0B
:10447000C20393F84023A242C5DDD3F83C3353F87E
:104480002400BDE8F047FDF769BF00BF8358080866
:104490004D3908089A520808E7500808EA40080809
:1044A0009F3A080893590808373A0808E440080872
:1044B000184507085D3B08082DE9F04F164685B002
:1044C000CDE901011A4600213046FEF719F8314CBA
:1044D000009006F010034FF00009A2460393FDF789
:1044E00021FF2379029A03F01803934203D0002A94
:1044F00044D1182B42D14FF00D0B0BFB09A3B3F89D
:10450000090050F0C5F880462046FBF7C5FBD8E906
:1045100002210746024401442046FBF755FB80F088
:104520000101009A0546C9B23046FDF7E9FF039B39
:10453000009003B115BB0BFB09FBB3065AF80BB097
:104540000ED56DB914485946FFF7E8F8D8F8082099
:1045500001982B463A442146FFF7C4FEFDF706FFBB
:104560000E485946FFF7DAF8D8F80C2001980023D6
:104570003A442146FFF7B6FEFDF7F8FE09F10109BE
:1045800040F28723994504F10D04A8D105B0BDE898
:10459000F08F00BF6054070804410808054108086F
:1045A00070B50546084616460C46FBF77BFC3346BD
:1045B000024621462846BDE8704093E60EB403B596
:1045C00003AA52F8041B0192FCF7B5F9044B054904
:1045D000986CFBF757FC02B05DF804EB03B0704732
:1045E00038A40020274C08080049E7E70F410808D5
:1045F00038B50C46054615492046FBF77BF930B91E
:10460000FDF766FE1248BDE83840FDF713BF1149BB
:104610002046FBF76FF9A0B90F4B83F8B90183F877
:10462000C10183F8A30283F8AB0283F88D0383F8FA
:10463000950383F8770483F87F0483F8F10407482F
:10464000E1E72846BDE83840CEE700BF1E41080834
:10465000244108083F41080838A4002047410808C1
:104660000049ABE763410808F8B5064608460C4622
:10467000FCF760FB2021054620465DF0A8F90446C2
:1046800018B93046BDE8F840EAE7124F124E3B78C1
:1046900032789A4204F1010401D0FAF743FC0F4B3F
:1046A00020461D605AF05AF9012201462046FAF7C9
:1046B000E1FB3B7832789A4201D0FAF733FC20468E
:1046C0005AF04CF92A460146BDE8F8400448FDF787
:1046D00065BE00BF902200205F3900208C220020A0
:1046E0007A4108082DE9F041064688B008460D4693
:1046F000FCF720FB2021044628465DF068F920B92C
:10470000304608B0BDE8F041AAE7FCF713FB2246AB
:10471000054601460F48FDF741FE85B1202D2A468A
:10472000694628BF20222046FAF744FCE8460646A0
:104730000027B74208DBAD1B3444002EEDD1FDF756
:1047400015FE08B0BDE8F08118F8010BFEF78AF8F5
:104750000137EEE7904108082DE9FF470746084674
:104760000D465AF0FBF8082845D105F1FF3801AE97
:10477000073531464246B14612F8010FFCF7F8F909
:10478000AA4201F8010BF7D10023DFF87CA08DF8D5
:104790000C30A84517D11B49484630F01FFE194878
:1047A0001949082310F8012B11F8014B10326A4403
:1047B000013B02F80C4CF5D114488DF80C3001A9DE
:1047C000FDF7ECFD14E018F8010FFCF7D1F906F83D
:1047D000010B0446014650465DF0F9F828B1214628
:1047E00030465DF0F4F80028D3D03846FFF7FCFEE1
:1047F00004B0BDE8F0870028D1D0384604B0BDE849
:10480000F0472DE7D03E00203CD00708A84108081B
:1048100007B5009313460A460249FFF7CFFE03B0DF
:104820005DF804FBAF4108082DE9F04FDFF8A482E2
:104830008BB006460D4628465AF090F8034638B924
:104840009649024601200BB0BDE8F04FFEF748BC88
:10485000934905222846FCF791F90446C8B9914DC1
:104860000146702205F5EA705DF09AF8C5F84442F9
:10487000C5F85042C5F85C42C5F86842C5F87442B4
:10488000C5F88042C5F88C42C5F898420BB0BDE827
:10489000F08F042241462846FCF770F9044628BBF5
:1048A0002846FBF756FB81460028EFD05AF056F811
:1048B000DFF824B282465BF8047B37B97A492A468E
:1048C00030460BB0BDE8F04F78E6524639464846D0
:1048D000FCF754F940B920462FF0ECF87348744DBA
:1048E0003946FDF75BFDA6E70134E4E7714907228D
:1048F0002846FCF743F9074600287AD120212846AC
:104900005DF065F8044670BB6B486C4DFEF706FF22
:10491000214628460134FEF701FF0E2CF8D1FDF7A1
:1049200025FDDFF8B891664FDFF8B48100252946F0
:104930004846FEF7F3FE0C26DFF8A8A16E430024DC
:10494000F25960480123A34013420CBF414651462F
:104950000134FEF7E3FE0E2CF2D10135FDF706FD22
:10496000082DE4D192E75849574D01AA5CF0FBFFAE
:1049700002AC002848D0022F11D1029A072A07D88A
:10498000039C0D2C04D80378722B13D06E2B25D0EA
:104990004E49082300223046FFF73AFF76E7FCF73E
:1049A000C9F901AA44F8040B2946002001375CF03C
:1049B000DAFFDEE73B490C2303FB02110123D1F8A8
:1049C0004412A3400B4337490C2000FB0212394923
:1049D000C2F844323046FFF727FF57E7314B0C202F
:1049E00000FB02330121D3F84432A14023EA010342
:1049F000E9E728463449344F01AA5CF0B4FF02AD20
:104A0000002480B1082C03D13046FFF729FE3DE792
:104A1000FCF790F901AA45F8040B3946002001344F
:104A20005CF0A1FFEDE7082CEED1029B0F2B30D8F4
:104A3000DDF80CE0BEF1070F2BD8DDF810C0BCF19B
:104A40000D0F26D8059F07F16402C82A21D8069DBC
:104A5000FF2D1ED8079864281BD80899642918D8F8
:104A6000884216DA099C032C13D8C3EBC3020D4B02
:104A7000134483F8D91183F8D4E10D4983F8D5C1E3
:104A800083F8D67183F8D75183F8D80183F8DA41D7
:104A9000A0E70F493046FFF791FDF7E604B7002085
:104AA000C841080830B50020D3410808E44108088F
:104AB000294C0808EE410808E8500808F6410808A3
:104AC00074B70020FB410808FF41080801420808AC
:104AD00007420808CE4108082C4B070883580808ED
:104AE000C05008083539080810B504460748FDF7D6
:104AF000A1FCFAF75BFD20B1BDE810400448FDF7CA
:104B000099BC20460349BDE8104057E51D420808FE
:104B1000274208082F4208082DE9F04F8FB00446BD
:104B200002AA0846B1495CF01EFF054640B903469B
:104B30000246AF494120FEF7AFFB0FB0BDE8F08F52
:104B4000AC49FAF7D7FE064628BBA84902AA5CF092
:104B50000AFFFCF7EFF80828054606D9A6490823FE
:104B600032462046FFF754FEE7E7A44C94F8A036FF
:104B700083420CDC84F8A056DFE73146384639F032
:104B800067F9013694F8A036B342F6DCF2E7064640
:104B900004F5D467F6E79A492846FAF7ABFE0646CD
:104BA000E0B9924902AA5CF0DEFEFCF7C3F80828DF
:104BB000054603D9934908233246D2E78F4C94F82F
:104BC000A136834202DC84F8A156B6E73046294676
:104BD000013652F0CDFD082EF8D1F4E78A49284677
:104BE000FAF788FE064600BB804902AA5CF0BBFECD
:104BF0000028A2D0FCF79EF80828054603D983496F
:104C000008233246ADE77D4C94F88A37834209DDAC
:104C1000014604F5D46039F05FF9294604F5D46003
:104C200039F068F984F88A5787E779492846FAF70E
:104C300061FE064618BB714BDFF8B09193F88A7796
:104C400006AD0146102228465CF0AAFEA846BE42E8
:104C500002AA80F20A81494600205CF084FE10B965
:104C60006C493A460AE1FCF765F8013628F8020B70
:104C7000EDE795E80F00684C84E80F005DE76749B1
:104C80002846FAF737FE0646C0BB5C4BDFF85C915E
:104C900093F88A7706ADBE4202AA80F2F3804946B5
:104CA00000205CF060FE014610B95D493A46E5E03F
:104CB000032228465CF0C3FEAA464FF000082846AF
:104CC00059F04CFE404502D801360435E3E79AF826
:104CD0000000FBF74DFF08F101080AF8010BEEE7B1
:104CE000504DB6000446B4423FF427AF06AB191945
:104CF0002819032239F096F80434F4E74A49284683
:104D0000FAF7F8FD0746002840F0AC80DFF8EC80A9
:104D1000364998F8A06602AA5CF025FE00283FF408
:104D20000CAFFCF707F8451E01D4AE4203DC3F4947
:104D30003346012215E72D4902AA00205CF013FE3C
:104D4000014600283FF4F9AE0026082203A88DF89A
:104D500014605CF074FE0DF10C0903A859F0FEFD1F
:104D6000B0421BD8214902AA00205CF0FCFD0028BB
:104D70003FF4E3AE037898F8A1A601930026B1466C
:104D800056451A4902AA4FF0000080F285805CF077
:104D9000EAFD834650B9264952466FE099F8000073
:104DA000FBF7E6FE013609F8010BD6E7A6B99BF83A
:104DB0000030303B092B0FD91E49FAF79BFD38B163
:104DC0001D495846FAF796FD70B11C495A4655E000
:104DD0004FF001094FF0FF365846FBF7ABFF0028B4
:104DE00030DA17495A4649E0B146F3E7FF4108086F
:104DF000D8AA0020364208083C42080838A40020FF
:104E000047420808504208085E4208086A420808FB
:104E10007C4208086B430808C4AB0020A64208087F
:104E20008B430808D4AB0020D0420808D5420808BC
:104E3000AB43080801370808E1420808E8420808BF
:104E40001D4308080EAB03EB4603013623F8200C84
:104E500096E72049524611E033F8022B24F8022F3E
:104E6000013730E01C492A4608E01C4900205CF06C
:104E70007AFD00283FF4FDAE19493A462046FFF777
:104E80009DFB5AE6154900205CF06DFD00283FF4BB
:104E900027AF14493A46F1E75CF065FD0028D8D108
:104EA000114C05EBC50082302044082203A938F0DC
:104EB000B9FF0198FBF75CFE08EB050304EB051452
:104EC00083F86A0706ABBE42C6DC454485F8829784
:104ED00033E600BF3243080855430808FF4108087D
:104EE00088420808B2420808D8AA00202DE9F041FB
:104EF000144B1B6888B00446F3B11A6804A9D56A3C
:104F000018466A46A847064688B1DFF8448004ACD4
:104F10006D46002735F8022B34F8021B4046013756
:104F2000FDF73CFABE42F5DC08B0BDE8F081064969
:104F30002046FFF743FBF7E7044908B0BDE8F0411E
:104F4000FFF73CBB60410020EA4308080244080820
:104F5000D043080870B5054608460C4659F0FEFCDB
:104F6000024670B1072804D1094821465CF055FD7E
:104F700038B12846064B074A0749BDE87040FFF79D
:104F80001DBBBDE8704002490448FDF707BA00BFE9
:104F90009A3E080809440808144408083E440808D2
:104FA00070B5054608460C4659F0D8FC024670B16B
:104FB000032804D1094821465CF02FFD38B128466A
:104FC000064B074A0749BDE87040FFF7F7BABDE84E
:104FD000704002490448FDF7E1B900BFA23E08084D
:104FE0004C440808144408085C4408082DE9F043C0
:104FF00007469BB008460C4659F0B0FC20220646F6
:10500000002101A85CF0CCFC36B3402E08D03B490F
:105010004023324638461BB0BDE8F043FFF7CEBA16
:1050200001AD04F140084FF0000902222146684614
:105030005CF005FD0023102209A968468DF8029056
:10504000FBF7D8FD099B0DF10202934223D10234F4
:10505000A04505F8010BE8D109AC4122002120460A
:105060005CF09EFC264D002E3BD095F8A462D6B194
:10507000202205F2A52101A85CF016FD98B105F2E9
:10508000A5212046FBF7E8FC1E4A1F492346384667
:10509000FFF794FA04E01A781C493846FFF78EFAB5
:1050A0001BB0BDE8F0831A4B1B78D3B9CEB9194EAB
:1050B00001AB1A4603CAA24230607160134606F182
:1050C0000806F6D101232046124985F8C532FBF7C0
:1050D000C3FC1148FDF708FA10482146FDF75EF9B8
:1050E000DEE795F8C5321BB995F8A432002BF3D052
:1050F00008492046FBF7B0FCEEE700BF6F44080804
:1051000030B50020AD44080814440808914408084C
:1051100038A40020D5B70020B7440808C6440808C2
:105120002DE9F74F834608460C4659F017FCDFF887
:1051300018810646D8F8007028B102463349204647
:10514000FBF71CFD80B93946314852F0C3FB3149A9
:10515000314821EA070152F0BDFB3049304803B025
:10516000BDE8F04F52F0B6BB23782D2B2D4B03BF7B
:10517000013406F1FF364FF0010A4FF0000A4FF0FC
:1051800000094FF0FF3553F8041B51B13246204659
:105190000193FBF7F3FC019B00280ABF4D46002159
:1051A000012109F1010991B9B9F11D0FEBD11E4996
:1051B0002246584603B0BDE8F04FFFF7FFB93B4326
:1051C000C8F8003019491A4B12E01A4913E0114A85
:1051D0000123AB401A40002AF7D007EA0302BAF1D4
:1051E000000FECD027EA0303C8F800301249134B34
:1051F000002A18BF1946124B124803EB8503D3F857
:10520000842603B0BDE8F04FFDF7C8B8613D08083B
:10521000FE440808BDD7771808450808422888E7E3
:10522000144508089C4B0708D3410808F6440808B1
:10523000EF440808D3440808DF440808E644080897
:1052400018450708C3380808944500202DE9F74F92
:10525000019008460E461746984659F07FFB0446D3
:10526000E8B93F483F4DFEF759FA20460CF0C8F91F
:105270003B68184206D020460CF0D4F90146284677
:10528000FEF74CFA0134172CEFD13B6813B93648BE
:10529000FDF764F803B0BDE8F04FFDF767B80246CC
:1052A00032493046FBF76AFC0546A8B93048FDF79D
:1052B00055F82C462F4D20460CF0A2F910EA080FA5
:1052C00006D020460CF0AEF901462846FEF726FA35
:1052D0000134182CEFD1DDE733782D2B03BF0136D5
:1052E00004F1FF34012500254FF0000948F4000BBC
:1052F00048460CF097F92246824601463046FBF7B5
:105300003DFC00BB48460CF07BF91BEA000F1AD0AD
:105310008DB1B9F1170F1CBF3B6840EA030816486E
:10532000C7F80080FDF71AF81248514603B0BDE8EF
:10533000F04FFDF733B8B9F1170F1CBF3D68854337
:105340003D600E48EEE709F10109B9F1180FCFD120
:105350000B490198324603B0BDE8F04FFFF72EB974
:1053600022450808113C08082C450808613D08083A
:1053700033450808123C0808E6440808F6440808C3
:10538000D3410808014A40F202235FE7144100209C
:10539000014B024A5AE700BFFFFF7F000C4100208B
:1053A00010B5044630F08AF828B920460449BDE813
:1053B0001040FFF703B9BDE810400248FCF7EEBF0C
:1053C0003E4508084D450808074B10B50446D3F87C
:1053D000C8023FF0BFFF28B920460449BDE810408D
:1053E000FFF7ECB810BD00BF30B5002058450808E5
:1053F00070B5054608461646FBF79CFC0D4B041E8F
:105400001A780EDB944205DA0B482146FCF7C6FFFA
:10541000204670BD2EB1FF2C03D10848FCF7BEFF1B
:10542000F6E70749013A2846FFF7C8F84FF0FF347E
:10543000EEE700BFD01100106E4508087F45080850
:10544000924508082DE9F04F074691B08248834DF8
:105450000E46FCF7A3FF8249C5F8CCD2002385F89D
:10546000D0320622012309783046402485F8D14203
:1054700007F074FA0A20F5F743FC95F8D0320C2BAC
:10548000DAB240F2E4809DF80C60FE2E2CD0FF2EA4
:1054900015BF0F24152400250125944240F0D78024
:1054A000611EC9B2684648F05DFE04F140030DEB91
:1054B000030414F8413C834240F0C4806A1E012A70
:1054C0009DF80D3012D903F01F0761375C0965485C
:1054D000FCF744FF022D39D0013C042C34D8DFE81E
:1054E00004F00B2D2F3331000225D6E79DF80E7006
:1054F0009DF80F401E46EAE75B48DFF8C491DFF8ED
:10550000C4A1DFF8C4B1FCF795FF5848FCF726FFAB
:105510006C464FF0000814F8011B484608F10108DA
:10552000FEF7FCF8B8F10C0F16D00AFB08F3B3F144
:10553000553FF0D85846FCF711FFECE74C48DCE744
:105540004C48DAE74C48D8E74C48D6E700238DF8BA
:105550003F300DF11F00D0E7FCF708FF022D3AD0D5
:105560006422B6FBF2F102FB11623B464448D2B220
:10557000C9B2FCF713FF85F001035B42DBB2012BDC
:1055800059D8404A404B9DF810104048404E0029E1
:105590000CBF11461946FCF701FF9DF811103D4B59
:1055A0003D4800290CBF31461946FCF7F7FE022D95
:1055B00041D19DF812403948FCF7D0FE8CB1FF2C48
:1055C0001FD00A23B4FBF3F103FB11423448D2B2DB
:1055D000FCF7E4FE08E033483A463146FCF7DEFECD
:1055E000CFE73046FCF726FF9DF813402E48FCF726
:1055F000B5FE44B1FF2C21D02C482146FCF7CEFE4D
:1056000004E02B48EEE72248FCF714FF204E214F20
:10561000DFF89C800DF11305002415F8013F7BB1E4
:10562000FF2B14BF3A464246214622480134FCF77C
:10563000B5FE042CF1D111B0BDE8F08F1C48E3E7B2
:105640003246F1E71C493846FEF7B8FFF3E71B483E
:10565000FCF7F0FEEFE700BFD845080830B50020A2
:10566000D0110010E9450808F44508081A46080852
:10567000FB450808034608080B460808C23A080814
:105680002C460808C1450808B845080863460808BC
:10569000C8450808F94F08087A46080881460808EE
:1056A00095460808484608089D4608088358080893
:1056B000CC450808AD460808B8460808C84608089A
:1056C00017370808ABAAAAAA9A5208082DE9F84386
:1056D000DFF8A49007460C46204659F03FF90646ED
:1056E00058B91D4B1D481A781D4B03EB8203D3F8A4
:1056F0001016BDE8F843FCF751BE02464946204665
:10570000FBF73CFA60B1DFF86480002558F8041B11
:10571000B1B9224638461349BDE8F843FEF74EBFFB
:105720001148124C124DFCF719FE54F8041B19B124
:105730002846FDF7F3FFF8E7BDE8F843FCF716BE8F
:1057400032462046FBF71AFA01350028DED1024B1B
:10575000084C1D70C0E700BF703F0020D14608080C
:1057600018450708D3410808334508082C4B07089B
:10577000123C0808294C0808613D080838B50D4658
:1057800004461A4905222846FBF7F8F968B9184B70
:1057900093F84C2022B9012183F84C1083F84D2056
:1057A000BDE838401348FCF745BE1349032228469C
:1057B000FBF7E4F9A0B90E4D95F84C3063B195F8BC
:1057C0004D304BB10D492046FEF7F8FE002385F819
:1057D0004C3085F84D3038BD0948FCF72BFEF5E715
:1057E00020460849BDE83840FEF7E8BE504F08089B
:1057F00038A40020DB460808A2500808F146080833
:10580000284708083C47080870B5184C94F84C30F5
:1058100005467BB194F84D3063B11549FEF7CEFED5
:1058200028461449FEF7CAFE002084F84C0084F88C
:105830004D0070BD104B93F8C522AAB193F8A42275
:1058400092B903F2A52203F5357503F2C526106857
:1058500051682C4603C40832B2422546F7D10122D2
:1058600083F80F230AF0DEFD0120E2E738A40020D0
:10587000F14608084B47080830B500202DE9F04FE5
:1058800080468BB008460D4659F068F80246B0B322
:10589000A3492846FBF772F9044680BBFCF766FD76
:1058A000A048A14DA14EA24FDFF8C482FCF7C2FD73
:1058B000142051F071FFE110304604F0070201316D
:1058C000FDF72CFF95F81D9095F91C00B9F1000F1C
:1058D0000ED007F035FD4A4601464046FCF75EFD16
:1058E0000134102C05F12405E5D10BB0BDE8F08F93
:1058F00007F026FD01463846FCF750FDF0E7284644
:105900008C4905AA5CF02FF8054620B901464120D4
:10591000FCF703FEE9E78849F9F7ECFF20B987496E
:105920004046FEF74BFEE0E7854E0827002431682D
:105930002846F9F7DFFF002808BF3446013F06F18B
:105940001006F4D154B97F492846F9F7D3FF28B19E
:105950007D492A464046FEF731FEC6E700207549DC
:105960008DF8130005AA5BF0FEFF0646002C4DD013
:10597000002849D0FBF7DEF9031E42DB2279062A14
:105980003AD1E268012101FA03F0104239D0DBB2CA
:1059900047F6FE7040FA03F2D20732D5994001393A
:1059A00008405CF091F80546E0884EF071FE6749CA
:1059B000D0E902230978002918BF1A46217A637AB0
:1059C00005FB0133002712F90390039702EB030A4A
:1059D000584905AA00205BF0C6FF834600283ED147
:1059E0005B49012394B39AF900202046CDE90031A8
:1059F0002946FAF7EFFA78E75D1E13B1A37A9D42C4
:105A0000D2DB54493246A5E7534EFAE768B10DF1AF
:105A10001301FBF769F928B19DF813502846F5F7F3
:105A2000BDFA20B94D49324694E74B4EFAE7284675
:105A3000F5F752FE8146284609F010FF03902846EC
:105A400009F048FFA24607462546C1E7CDE90031E7
:105A50009DF813004A463946FAF700FB45E73649F8
:105A6000F9F748FF064658BBACB13D4FEDB220797F
:105A700072B22946F5F70AFE00283FF436AF0288D5
:105A8000037800933146C2F303233846120BFCF728
:105A900085FC0136EBE7324C7979386872B2F5F75C
:105AA00037FE00283FF421AF028803780093314687
:105AB000C2F303232046120BFCF770FC0136EBE720
:105AC00028495846F9F716FF002853D05846FBF7E7
:105AD00031F9064642B29CB12079E9B2F5F7D6FD1C
:105AE000002849D129462046FAF728F926681E4998
:105AF000CDF800B0034632464046FEF75FFDF4E6BF
:105B000079793868F5F704FEB0BB9DF81330174972
:105B1000CDF800B01A09403203F00F03ECE700BFE4
:105B2000694708086E470808C00200208447080833
:105B3000123C0808FF410808613D0808954708081D
:105B400040060020CB4A0808A947080838A40020CE
:105B500075230108B8470808294C0808C8470808F1
:105B6000DA4708082E450808FB4708081E480808B9
:105B7000F34808084FF0FF3606AF39463046FAF7CB
:105B80007FFF08A94846FAF77BFF4E451CD076B246
:105B900074B18AF8006029462046FAF7CFF82668E3
:105BA00000970246134808AB3146FCF7F7FB9CE62A
:105BB0009DF81320039B10489E701109009708ABB5
:105BC00002F00F024031F0E75CB129462046FAF7B7
:105BD000B5F826680246094808AB3146FCF7DEFBFB
:105BE00083E69DF813200648110908AB02F00F0266
:105BF0004031F3E746480808694808089148080812
:105C0000AC4808082DE9F04F07468DB008460D4610
:105C100058F0A4FE044630B9014601200DB0BDE89D
:105C2000F04FFCF785BD0246A5492846FAF7A6FFC6
:105C300030B9A44938460DB0BDE8F04FFEF7BEBC00
:105C4000A14922462846FAF799FF002854D1FCF7CB
:105C50008DFB9E48DFF8B4A2DFF8B4B2FCF7EAFB94
:105C6000172051F099FD0E271AF9018BB8F1000F9A
:105C700036D041465846FDF751FD00252E46B1006D
:105C800089B2404609F060FE814609F0E9FE90F9CC
:105C9000003004460136CBB10DB9FCF767FB99F82B
:105CA0000630657894F90000894A8A4C03F00203B3
:105CB000002B18BF1446B5B107F042FB0095034610
:105CC000224685483146FCF769FB0125042ED6D1D2
:105CD00015B98248FCF7AEFB013F17F0FF07C3D1AF
:105CE0000DB0BDE8F08F07F02BFB2246034631468E
:105CF0007B48FCF753FBE8E7002476498DF81B400E
:105D000007AA28465BF02FFE18B93846FEF76CFC50
:105D1000E6E70DF11B01FAF7E7FF81460028F4D012
:105D20009DF81B502846F5F739F920B96D493846DA
:105D3000FEF744FCD4E7DFF8DC8123464FF0FF3464
:105D400003EB430218F8022095420BD0002C02DA34
:105D5000002A08BF1C460133152BF1D1002C16DA9E
:105D60006149E4E71C465B4907AA00205BF0FBFDA4
:105D70000646002800F096805149F9F7BBFD30BB7C
:105D80005A4FDFF84C81DFF89091044616E04FF04F
:105D90000009E8E7306896F807A0F5F7C9FFB17980
:105DA000737911F0020F0CBF394641469B08024639
:105DB0000091013351464846FCF7F0FA0134214680
:105DC000284609F05FFD06460028E3D188E74849E8
:105DD00002223046FAF7D2FE4FEA151A0AF1400ABB
:105DE00005F00F0B002845D10390B01CFAF7A2FF75
:105DF000039902460491284601310592039109F066
:105E000041FDDDE90313059A38B93A4900965B462E
:105E100052463846FEF7D2FB62E7C0799042E9D19C
:105E20001F466300B9F1000F31D01A194244567869
:105E3000013E7A1C234414BF2946002108EB0302CB
:105E400008F803107B1C53700AACFF23937039468B
:105E500022462846FAF724FE08AA31462846FAF7D1
:105E60001FFEB74216D1244808AB5A465146FCF7EC
:105E700095FA35E721493046F9F73CFD20B1204934
:105E800000965B465246C4E74FF0FF37C9E74FF034
:105E9000FF36CEE71B48009408AB5A465146FCF744
:105EA0007DFA1DE704EB4404174B0093A04402461F
:105EB00098F8011001232846FAF716F910E700BFF9
:105EC000613D08089547080869470808C848080858
:105ED000A03A0808FF410808E848080809490808E6
:105EE000FA4808080F49080826490808294C0808F4
:105EF0004F49080852490808A44908082E450808CF
:105F00007E490808C24908087523010828C1070806
:105F1000E1480808AC2400203A4908082DE9F04F70
:105F200089B0074605AA08469C495BF01CFD05465A
:105F300030B901464120FDF76DFB09B0BDE8F08F97
:105F40009749F9F7D7FC044600283CD19548964D6F
:105F5000964EDFF89882FCF76DFA142051F01CFC85
:105F600095F9060007F0ECF92968AA8801F13F418C
:105F700001F57E01B2FA82F2890A03464131C2F18B
:105F80001F023046FDF7CAFBE97911B14046FDF723
:105F9000C5FB0134FCF7EAF9602C05F10805DFD1F7
:105FA0007E4905AA00205BF0DEFC8149F9F7A2FCDE
:105FB0000028C2D138467A49FFF724FE784938468E
:105FC000FFF75CFCB9E7DFF8FC91002419F9340015
:105FD00007F0B6F9804601462846F9F78BFC40B138
:105FE00001342B2CF2D173492A463846FEF7E6FAE3
:105FF000A3E76A4905AA5BF0B6FC064690B3FAF738
:1060000099FE05466C4B03EBC4034FEAC40A93F8B0
:10601000EA314BBB002D29DC09EB0A03588893F8C1
:10602000049093F805A04EF033FBEBB2D0F808B023
:10603000009303FB09AA002E00F09A803378002B0E
:1060400000F0968006A93046FAF74EFE002800F0D0
:106050008C809DF8185005BB0BF80A505748FCF788
:10606000E9F96AE70546CDE7002D05DD012B1A4663
:1060700038BF0122954208DD012B514938BF012369
:1060800001223846FEF7C4FB57E7444905AA002021
:106090005BF069FC013D0646BEE72846F4F77EFF4B
:1060A000814600285DD02B09403302930BF80A503B
:1060B00005F00F03434F03934FF00008BB79012B0A
:1060C00038BF012301930026788897F804B097F829
:1060D00005A04EF0DDFA06FB0BA38268D15CA94255
:1060E00022D1444504D10099B1421DD00021D154A0
:1060F000DDE9021234485FFA86FB5FFA88FAFDF7A1
:106100000DFB59465046FDF7B1FF444509D12F48D4
:10611000FDF704FB50465946FDF7A8FF2C48FDF754
:10612000FDFA2C48FCF786F9019B0136B342CBDC23
:1061300008F10108B8F12B0F07F10807BED1D9F813
:106140000010B9F80420244801F13F4101F57E0117
:10615000B2FA82F2890AC2F11F024131FCF71EF93C
:10616000EBE63846FEF740FAE7E61C4932463CE7E4
:106170001BF80A30013573B11A09194903F00F03EE
:10618000403206A8FAF704FC06AB16482A464146F8
:10619000FCF704F9D1E6144BF7E700BFFF4108080C
:1061A00069470808E8490808201D0020264A080811
:1061B000314A0808354A080818450708574A0808A8
:1061C000514A0808FC460708694A0808B93A08080D
:1061D0008D4A0808B1510808974A0808B34A0808C8
:1061E000093A0808CF4A08085536080882580808AE
:1061F00020B10078B0FA80F0400970470120704764
:106200002DE9F74F81460846FFF7F2FF0E46054697
:1062100070B1002401A9204651F0EEFB0134014683
:106220004846FFF7EDFF122CF4D103B0BDE8F08F24
:106230000846FAF77FFDC4B2112C71D8701C3D4D91
:106240003D4EF9F786FE05EB4408670098F810A369
:106250008346B8B9AAF102014B424B413D4495F83F
:106260001023B25C002B54D095F81133192040F262
:10627000EE2100FB03133148214603B0BDE8F04F87
:10628000FCF78CB8017830465BF0A1FB78B1032CA9
:1062900094BF002201222A4902EB4202831B0A44D6
:1062A00052FA83F393F8F8A6BAF1030F05D14846E2
:1062B00003B0BDE8F04FFEF797B95846F9F749FE2D
:1062C000F0B1BAF1020FF2D1FAF734FD40F6CA0389
:1062D00080B29842A8BF184640F2EE239842B8BF59
:1062E0001846A0F2EE201923B0FBF3F088F8110352
:1062F000AAF1020253425341EA1982F810A3ADE712
:10630000BAF1020FF4D1484603B0BDE8F04FFEF7F2
:10631000A7B90C48214603B0BDE8F04FFCF73EB8E2
:10632000094911232A46484603B0BDE8F04FFEF75D
:106330006FBA00BF30B500204CD20708E34A080806
:1063400018450708F34A0808004B08082DE9F041F2
:10635000054686B00846FFF74BFF0F46064640B19C
:1063600000235C491A46012006B0BDE8F041FCF765
:106370009BBA0846FAF7DEFC1328044600F3A18016
:1063800006254543781C8DF81760F9F7E2FD524E5B
:10639000074660B1FAF7CEFCC0B213F09FFB30B1F4
:1063A0007319027983F8042601238DF817303846D3
:1063B000F9F7CFFD074668B1FAF7BCFC0D2809D8FC
:1063C000062303FB046383F805069DF817300133A9
:1063D0008DF81730DFF8FC80A91C0DF1170241443D
:1063E0003846FAF7ABFCF9F7B4FD074668B1FAF79F
:1063F000A1FC012809D89DF81730062202FB04628F
:10640000013382F808068DF817303846F9F7A1FDF8
:1064100080B1FAF78FFCC0B213F060FB50B19DF869
:1064200017300179062202FB0462013382F8091653
:106430008DF817309DF81720042A4FF006032FD14E
:1064400003FB04630022A3F80826062505FB046568
:1064500022F0F6F995F8040613F024FB95F80716D8
:1064600095F8067619234FF46172804695F809066F
:1064700013FB012613FB072713F014FB437998F84D
:106480000520039395F808360097CDE9016313487A
:1064900095F805362146FBF781FF06B0BDE8F0818F
:1064A000052A05D103FB0463002283F80926CCE703
:1064B000062ACAD008EB0502002348F8053093806D
:1064C000C3E7074913233246284606B0BDE8F0412A
:1064D000FEF79EB93CAA002038A400205C380808CA
:1064E000514A08082DE9F04780468CB00846FFF76E
:1064F0007FFE054640B1002359491A4601200CB0E1
:10650000BDE8F047FCF74CBACDE909000B900791C4
:1065100007A854495BF0FAF9064651F051F9431CBB
:1065200004460ED12B460A2208A93046FAF762FB30
:10653000089B1B782BB9C4B2132C96BF333444B2DA
:1065400064B220460BF07CF8054628B94046FEF7B9
:106550004BF80CB0BDE8F08742498DF8284007A8F9
:106560005BF0D4F9B0B300230A221946FAF742FBD4
:1065700002260990DFF8EC90DFF8F0A000274946EA
:1065800007A85BF0C3F9F8B1FAF7D4FB364A002349
:1065900052F8041B88421FD1DBB20AEB8302D2F807
:1065A000A421904210D1022F20D0032F23D05A1EB5
:1065B000012FD2B215D00B2A03D88DF8293001361D
:1065C000F6B20137042FDAD1052E1AD84046FEF76D
:1065D00047F8BEE70126CDE70133102BD8D10023C1
:1065E000DBE7052AEDD88DF82A30E8E7092BE8D853
:1065F0008DF82C30E3E79A1E0D2AE2D88DF82B3067
:10660000DDE709AB03CB286018686960A860204605
:1066100051F0DCF9154A9DF82B1002EB810103467D
:10662000D1F8A41104919DF82C1002EB8101D1F84E
:10663000A41103919DF82A1002EB8101D1F8A41155
:1066400002919DF8291002EB81020021D2F8A421C9
:106650000192099A00920846054AFBF78BFE78E7FB
:1066600030A90020FF410808BC4607081845070864
:10667000753808082DE9F04F0346A1B00846FFF72A
:10668000B7FD054628B1184621B0BDE8F04FFDF72B
:10669000E7BFDFF8C4920B90FF238DF82830D9F8BC
:1066A000C832ADF83000CDE9050093F838200D90E0
:1066B0008DF838200F90ADF84000119309910746EE
:1066C0004FF0FF38934909A85BF020F9044618BB46
:1066D000914F01460AAC0B0190481A57002310F95C
:1066E000016BB24240F0D28010464E1C51F06EF960
:1066F000314602463846FBF751FE022E4FF00101AB
:10670000E9D19DF938A09DF92830534540F0C58066
:106710008348FBF743FE4DE02378002BD2D0032FB4
:10672000D4BF00260126062F00F2A980DFE807F07B
:106730000447509104475000042F10D07949204657
:10674000FAF740FA58B14FF480600DF03DFD002893
:1067500000F0B58190F90400012306930AE0724924
:106760002046F9F7C7F870B9D9F8C83293F938005C
:10677000042F22D0119B119320AB03EB061606F8D1
:10678000580C01379EE7204651F01AF80028EFDA3E
:1067900001230A2212A92046FAF72CFA40B2002857
:1067A00003DB129B1B78002BE2D060482246711C51
:1067B000FBF7F4FD21B0BDE8F08F0023DBE72046B6
:1067C000FAF7B8FA20AB03EB061646F8540CD8E7F4
:1067D00057492046FAF7F6F95649B0F1000A204623
:1067E00018BF4FF0010AFAF7EDF908B14AF0020AB2
:1067F0003301DFF868C1079320AB03EB0616BCE852
:106800000F0006F850AC12AE0FC6BCE80F000FC662
:10681000BCE80F000FC69CE8030086E803000026D2
:106820000DF1480AB346DAF8001020465BF026F96D
:1068300010B19AF804301E430BF1010BBBF1070FA6
:106840000AF1080AEFD1079B80336B4403F84F6CC1
:1068500097E739492046F9F74DF8A0B13749204666
:10686000F9F748F800288CD02046FAF763FA032895
:10687000804686D901463248FBF790FD9AE73148B9
:106880002246082194E7012305937AE70133072B79
:106890007FF425AF2C4801318AE70B9B1BB9AAF185
:1068A00014025542554100235F1CE368002B62D15E
:1068B00094F900B058460AF005FFD4F8049018B1D6
:1068C0000668002E40F08B80B9F1000F237A14BFC8
:1068D0004E464FF46146666023B91C48FBF75EFDE7
:1068E00003232372627A2AB1194807923946FBF7CB
:1068F00055FD079A0292237ACDE9006300231A46D8
:10690000194658460DF0ECFCE06048BB114839468A
:10691000B2E700BFFF410808844B08088933070825
:10692000A14B0808234B08082E4B0808324B0808D7
:106930004D4B080826500808C84108082E4508088D
:10694000504B0808684B08088F4B0808BA4B0808DA
:10695000D54B0808F04B080830B50020184C070844
:106960005849594A5948B9F1000F18BF0A463346E9
:106970003946FCF7D3FE022F04F110044FF0010357
:1069800092D1119E0D9F4DB15148FBF753FD3368D5
:106990001B6A1BB14F493A4630469847059B002B6E
:1069A00050D04D49474BBAF1140F18BF19464B4808
:1069B000FBF7F4FCBAF1140F09D1059B002B43D06F
:1069C0003368DB691BB14649002230469847069B75
:1069D000002B43D100223146384650F009FFE660D3
:1069E000B9F1000F2CD04946304601F06DFE3D4A0A
:1069F000B3683D483946FBF7D1FC94F80890B9F1EB
:106A0000000F0CD03279914509D038484B463946B1
:106A1000FBF7C4FC336849469B6930469847637A64
:106A200023B1727932483946FBF7B8FCF36A002B80
:106A3000A1D030483946FBF7B1FC0023F3629AE756
:106A4000204AD5E71F49B2E7B8F1000FBFDB336832
:106A5000DB69002BBBD028494246B6E706F012FAA4
:106A60000520F4F74DF9DFF89490DFF894A00025A5
:106A70004FF0030B9AF80030AB42ABD919F8014F35
:106A8000C4B1204608F026FF804698B12046F4F7AE
:106A900085FAEBB2044610B180F806B0C371204607
:106AA0000121F4F7CFF998F80630DB07204603D52B
:106AB000F4F7B6FB0135DDE7F4F7ACFBFAE74FF08E
:106AC000FF3049E6294C0808084B08080C4C080818
:106AD000C24C0808C9860108164B0808EB4C080888
:106AE0006DFF0008114B08082A4C08084F4C080895
:106AF000724C0808A94C080801FD0008F324002086
:106B0000D01100102DE9F04380468BB00846FFF706
:106B10006FFB0F46044640B100235E491A46012030
:106B20000BB0BDE8F043FBF7C1BF0846FAF702F926
:106B30001D28054600F3A5800A264643781C8DF8DB
:106B40002740F9F706FA10B101238DF82730F9F73D
:106B500000FA514C074668B1FAF7ECF80D2809D84D
:106B60000A2303FB054383F834039DF827300133E0
:106B70008DF82730DFF81C91711C0DF12702494474
:106B80003846FAF7DBF8F9F7E4F9074668B1FAF79F
:106B9000D1F8232809D89DF827300A2202FB0542A4
:106BA000013382F837038DF827303846F9F7D1F9E9
:106BB000074668B1FAF7BEF80D2809D89DF82730C6
:106BC0000A2202FB0542013382F838038DF8273090
:106BD0009DF82730062B0CD009EB06020023404617
:106BE00049F80630536013810BB0BDE8F043FDF760
:106BF00037BD0A2606FB054600233846A6F83A3379
:106C0000A6F83C33F9F7A5F9074618B1FAF792F858
:106C1000A6F83A033846F9F79CF930B1FAF78AF842
:106C20000A2303FB0543A3F83C031C4B4FF0FF3240
:106C30005A600A2303FB05424FF46170B2F83C33FB
:106C40000693B2F83A33059392F83833049392F8E6
:106C50003733039392F83613192313FB0101029182
:106C600092F8351313FB0103019392F83433009328
:106C700000210B4A2B460846FBF77CFB0BB0BDE816
:106C8000F08308491D23224640460BB0BDE8F0437F
:106C9000FDF7BEBD64B8002030B5002034060020EA
:106CA00092380808514A08082DE9F14FDFF894B1ED
:106CB00006460D462846FFF79BFA074640B10023DB
:106CC00059491A46012001B0BDE8F04FFBF752BF09
:106CD000564905222846F9F751FF60B9524B002268
:106CE0001A601A611A621A631A641A651A661A67B8
:106CF00001B0BDE8F08F042259462846F9F73EFF5F
:106D000004462846002C42D1F9F723F9074600280B
:106D1000EED057F023FEDFF830A15FFA80F85AF882
:106D2000049BB9F1000F07D141492A46304601B012
:106D3000BDE8F04FFDF742BC424649463846F9F7F8
:106D40001DFF013484460028E9D1374A0346154621
:106D500000210133082B42F8101BFAD1354B03EB0D
:106D6000C40257682FB93448344D4946FBF716FB27
:106D7000A0E713F834E0F445F5DA07EB0C130FCB7A
:106D800005EB0C1484E80F000CF1010CF3E7F9F7A4
:106D9000D1FF072804463DD82846F9F7DAF8074618
:106DA00058B3F8F749FE204B03EB041383ED000AB8
:106DB00001253846F9F7CDF8074638B1F8F73CFE1B
:106DC000194B03EB041383ED010A01353846F9F73B
:106DD000C0F8074638B1F8F72FFE134B03EB041346
:106DE00083ED020A01353846F9F7B3F838B9304671
:106DF00001B0BDE8F04FFDF733BC0546D9E7F8F721
:106E00001BFE094B032D03EB041383ED030A3FF430
:106E100056AFECE70A4907233A46304601B0BDE8D1
:106E2000F04FFDF7F5BC00BF843F0020C8410808C3
:106E3000D341080890330708E4410808294C0808A2
:106E4000514A0808CE4108082C4B07082DE9F341A8
:106E500005460846FFF7CCF90C46074640B100232B
:106E600033491A46012002B0BDE8F041FBF71EBFCE
:106E700030492046F8F73EFD70B92D4B04224FF4FF
:106E80007A704FF4FA61013A1880598003F10403D3
:106E9000F9D102B0BDE8F0812046F9F74BFF032895
:106EA000064641D82046F9F754F8074698B1F9F755
:106EB00041FF4FF0010804463846F9F74AF820B17F
:106EC000F9F738FFB8F1000F09D1284602B0BDE844
:106ED000F041FDF7C5BB40F2EE248046ECE7A4F29A
:106EE000EE2240F2DC539A4203D8A0F2EE229A42FC
:106EF0000AD9114940F6CA0340F2EE22284602B0F0
:106F0000BDE8F041FDF784BC0C4B0D4A03EB860352
:106F10000021A3F86044A3F86204CDE900403346A1
:106F20000846FBF727FAB4E7064903233A46E5E7A4
:106F300090B90020C84108080E4D080830B500205F
:106F4000C9380808004B0808F0B5074689B008465C
:106F5000FFF74EF90E46054640B100231A491A467E
:106F6000012009B0BDE8F040FBF7E4BE0846F9F7A0
:106F7000E1FE1F2804461DD83046F8F7EAFF014617
:106F800020463EF0E7FB78B10F4803AE314600EBF8
:106F9000840050F0C9FC0D4A009623462946284635
:106FA000FBF7E8F909B0F0BD384609B0BDE8F0409C
:106FB000FDF71ABB06491F232A46384609B0BDE82B
:106FC000F040FDF725BC00BFA0B90020DA38080862
:106FD000514A0808F0B5074685B00846FFF708F99A
:106FE0000E46054640B100231D491A46012005B052
:106FF000BDE8F040FBF7E6BE0846F9F79BFE0F2818
:10700000044623DC3046F8F7A4FF014620463EF054
:1070100087FCA8B1134B04F1200203EB820329463D
:1070200093F87324029293F872240192B3F87034A7
:1070300000930D4A23462846FBF79CF905B0F0BDA6
:10704000384605B0BDE8F040FDF7CEBA07490F233A
:107050002A46384605B0BDE8F040FDF7D9BB00BF71
:1070600020BA002030B50020E4380808514A08084A
:10707000F0B5054685B00846FFF7BAF80B4604465A
:1070800040B100231B491A46012005B0BDE8F0407D
:10709000FBF7E0BE1849184F6A4618465AF063FCE1
:1070A00001AE88B1032C04D12846FDF7D9FA05B00A
:1070B000F0BDF9F73FFE6A4646F8040B394600205A
:1070C00001345AF050FCECE7032CEDD1DDE9014628
:1070D000039F31463A46E0B23EF05EFC18B92846BE
:1070E000FDF782FAE3E705483B4632462146FBF7C7
:1070F00055F9DCE7A0B90020FF410808F638080878
:10710000F0B506468BB00846FFF772F80D46044608
:1071100028B300233E491A4601200BB0BDE8F040D9
:10712000FBF736BF2D2903D0A1F13003092B49D835
:10713000052C05DD30460BB0BDE8F040FDF790BAF8
:107140002846F9F7F7FD0AAB621C03EB440424F868
:107150000C0C15F8013F303B092BFAD9144629785D
:107160000029DFD1062CE5D1BDF81C20BDF91C306B
:10717000072ADFD8BDF91E50A5F5FA7292B2B2F512
:10718000FA6F18D8BDF92070A7F5FA7292B2B2F56D
:10719000FA6F10D8BDF922C065450CDC67450ADBE3
:1071A000BDF924E00EF1640292B2C82A03D8BDF9F9
:1071B0002640112C11DD174930460BB0BDE8F040D8
:1071C000FDF7FCB9202902D101352246C6E7304639
:1071D0000BB0BDE8F040FDF707BA0F4A0C2000FBEA
:1071E000032264B2A2F84852A2F84A72A2F84CC232
:1071F00082F84EE282F84F420846CDE903E4CDE939
:10720000017C064A0095FBF7B5F80BB0F0BD00BF56
:1072100074B700200742080830B500200A39080872
:107220002DE9F04F074689B00846FEF7E1FF8B468F
:10723000054640B100234D491A46012009B0BDE87A
:10724000F04FFBF7C9BF4A4B084693F8A0A693F846
:10725000A19693F88A87F9F76DFD092804467BDC2F
:10726000062646430BF101008DF81F50F8F771FE1A
:107270003E4D834638B1F9F75DFD0D2803D8012353
:10728000A8558DF81F305846F8F763FE834660B165
:10729000F9F750FD504508D8062303FB04535870F6
:1072A0009DF81F3001338DF81F305846F8F751FE16
:1072B000824660B1F9F73EFD484508D8062303FB36
:1072C000045398709DF81F3001338DF81F305046DD
:1072D000F8F73FFE814660B1F9F72CFD804508D3F1
:1072E000062303FB0453D8709DF81F3001338DF83B
:1072F0001F30311D0DF11F0229444846F9F71EFDCC
:107300009DF81F30062B09D0AA1900233846AB512F
:10731000938009B0BDE8F04FFDF7A2B96343EA18C6
:107320004FF461765079192111FB006005901079B6
:1073300011FB00610491D178039191780291527808
:107340000192EB5C009300210A4A23460846FBF7B2
:1073500011F809B0BDE8F08F074909232A463846DD
:1073600009B0BDE8F04FFDF753BA00BF78410020E7
:1073700038A4002054390808514A08082DE9F74F6D
:1073800005460846FEF734FF0B46044618B9334A53
:1073900092F860752FB9284603B0BDE8F04FFDF7AD
:1073A00023B92F49DFF8C890DFF8C8A001AA184612
:1073B0005AF0D9FA264610B905F070FD08E056B922
:1073C000012201462846FEF713F8421C04461AD152
:1073D00003B0BDE8F08FF9F7ADFC2F28834636D80F
:1073E0000FB105F04FFDBBF1060F13D01D4901236E
:1073F00009785FFA8BF2E0B205F0B0FA59464846D8
:10740000FAF7CCFF0027164901AA002001365AF0EE
:10741000AAFAD0E7DAF800301B0114D5FF2C0ED001
:10742000E1B22846FEF70EF8E8E72846FEF70AF82C
:10743000013798F80020F9B28A42F6D8DEE7DFF883
:1074400024800027F5E70848FAF7F4FFD6E7074954
:107450002F222846FDF7B2F8D5E700BF30B500204F
:10746000FF410808D01100103E4508082D4D0808BE
:107470001C4D0808CC3E00202DE9F743074608467E
:10748000FEF7B6FE0B46044628B1384603B0BDE809
:10749000F043FDF7E5B82F49DFF8B89001AA184688
:1074A0005AF061FA26460546A04665B92A4B32468F
:1074B000D3F8C802A1B252F0A3FE68BB27493846F0
:1074C000FDF77CF828E0B8F1000F06D0B8F1010F05
:1074D00025D03846FDF7C4F81EE0284657F03EFA9E
:1074E0001F49064602462846F9F748FB50B31D4996
:1074F00032462846F9F742FB30B31B49324628464C
:10750000F9F73CFB10B3194932462846F9F736FB28
:10751000F0B13846FDF768F803B0BDE8F083B31E5C
:107520005A425A4129463846FDF762FF421C04463A
:10753000F2D001AA494600205AF015FA08F10108D4
:107540000546B2E74646F4E70126F2E70226F0E7F1
:107550000426EEE7FF41080830B50020594D080821
:107560004D4D0808504D0808534D0808564D080861
:107570002DE9F74380460846FEF73AFE0B460546DE
:1075800028B14046FDF76CF803B0BDE8F0832D4903
:10759000DFF8B09001AA18465AF0E5F92F460446E4
:1075A0002E467CB9022DECD1A7F57A73B3F57A7F1C
:1075B00021D925494FF4FA634FF47A724046FDF71A
:1075C00027F9E1E74DB1012D10D001AA494600206D
:1075D0005AF0C9F901350446E3E701222146404645
:1075E000FDF706FF431C0646EFD1CDE72046F9F72D
:1075F000A1FB0746E9E7154B1B68B8B25B689847E3
:10760000FF2EBCEEC00A124B0BD1124AF8EE407AA4
:107610001278A24212DC10EE101A0F48FAF7BEFEE2
:10762000B2E7F8EE407A03EB860310EE102A0B481F
:10763000C3ED007A3146FAF7B1FEA5E7E3EC017A33
:107640000134E6E7FF410808674E08087817001084
:1076500094BA0020D0110010844D0808774D080816
:10766000F8B507460846FEF7C3FDD0B1204BD3F866
:1076700098600136304609F0D5FF34460546F0B92A
:107680000134182CA8BF0024204609F0CBFF054682
:10769000A8B9B442F4D138461649BDE8F840FCF721
:1076A0008DBF0846F9F746FB044609F0BBFF0546C7
:1076B00028B921461048BDE8F840FAF76FBE0C4BD8
:1076C000C3F898400CF0A2FE0C482A462146FAF76F
:1076D00065FE172C09D80A4B0C2202FB043393F8E1
:1076E0003807BDE8F8400CF0CDBE0020F9E700BF38
:1076F00034060020934D0808A74D0808BD4D080822
:107700001845070838B5124D04460846FEF770FDC7
:1077100060B1104B104893F900104B1C0ABF0F4B7F
:10772000C9B21978BDE83840FAF738BE0846F9F70B
:1077300001FB032804D8C0B2FAF72AFA2946E4E785
:1077400020460749BDE838400322FCF737BF00BF99
:10775000294C080834060020D64D0808B83E002001
:10776000E64D0808F0B5032985B005460C461646D7
:1077700014D80B4F3970FAF7F9FD0A492846FFF77C
:10778000C1FF0949224601A8F9F702F901AB3246C7
:1077900008212846FCF790FEFF233B7005B0F0BDA2
:1077A00034060020294C0808D64D080838B5124D7B
:1077B00004460846FEF71CFD60B1104B104893F9D3
:1077C00001104B1C0ABF0F4BC9B25978BDE83840B5
:1077D000FAF7E4BD0846F9F7ADFA032804D8C0B2B9
:1077E00013F0E0FF2946E4E720460749BDE83840AA
:1077F0000322FCF7E3BE00BF294C08083406002032
:10780000D24D0808B83E0020E14D0808F0B5032924
:1078100085B005460C46164614D80B4F7970FAF71A
:10782000A5FD0A492846FFF7C1FF094922466846D7
:10783000F9F7AEF86B46324610212846FCF73CFEBD
:10784000FF237B7005B0F0BD34060020294C0808EA
:10785000D24D08082DE9F74F444BDFF82C911A78E8
:107860005B7889F80130424B00911B7889F8002041
:1078700005460BB904F0A8FE4CF044FF00263D4C31
:10788000B0460D233B4A0099734352F803A050467B
:10789000F9F798F9002841D0B8F1000F01DDFAF7A7
:1078A00065FD35485146FBF739FF00222146284641
:1078B000FCF776FEFAF75AFD237903F01803082B3C
:1078C00046D0102B49D02046FBF735FF294B0D221F
:1078D00002FB0633B3F809004CF0DAFE8346D8B158
:1078E0002046F8F7D9F9DBE90221074602440144B2
:1078F0002046F8F769F978B9019051461F48FBF71F
:107900000DFFDBF80810019A28461346CA192146D4
:10791000FCF7E8FCFAF72AFD08F10108013640F20D
:1079200087239E4204F10D04ABD10020F8F793F9B0
:10793000FF2389F8003089F80130B8F1000F11D128
:10794000009A0F49284603B0BDE8F04FFCF736BE59
:107950000C492846FFF7D6FEB5E70A492846FFF747
:1079600025FFB0E703B0BDE8F08F00BFB83E0020B0
:1079700038A400206054070809410808014E08088F
:10798000D3410808294C0808340600202DE9F74F98
:10799000804608460F4656F0E1FF044620B1012814
:1079A00025D13B782A2B22D1A948AA4EAA4FFAF713
:1079B00041FD0025B1464FF00D0A04F001040AFB19
:1079C00005F3384659F80310FBF7A8FE3146224666
:1079D0004046FCF7E5FD0135FAF7C8FC40F2872385
:1079E0009D4206F10D06EAD103B0BDE8F08F3D21BE
:1079F000384659F0ECFF002800F0238103469A46F0
:107A000013F8012D202AFAD0AAEB070A0130054607
:107A100010F8013B202BFAD0DFF838B25FFA8AFA6F
:107A20004FF000090D2303FB09F352465BF80310E6
:107A3000009138460BEB0304F9F7A0F8064670BB3B
:107A40000099084656F08AFF824528D1277907F029
:107A5000E001402900F0898012D871B366797F4A2D
:107A600002EBC606002796F840230092BA463B4632
:107A7000009ABA4202D9BAF1000F62D02BB12DE0C0
:107A80006029ECD0802900F0A48040467449FCF7BE
:107A900095FD204603B0BDE8F04FFBF74CBE09F161
:107AA000010940F287239945BCD16E493A464046C8
:107AB00003B0BDE8F04FFCF781BD07F00703042BCE
:107AC0001CD10B460A222846F9F794F8D4F8053061
:107AD00083420146D9D32046F8F7F8F90D2303FB7A
:107AE00009F961485BF80910FBF718FE00222146EE
:107AF000404603B0BDE8F04FFCF752BD052B0DD159
:107B000001230A222846F9F775F8D4F80530834294
:107B10000146BADB5B428342B7DCDCE72846F9F773
:107B200009F917F0050F0BBFB4F80520B4F90520CB
:107B3000B4F80730B4F9073090420146A5DB98420B
:107B4000EAE7D6F83C1351F8270060B129460193C3
:107B5000F7F7D0FE019B30B9394620464FF0010AB5
:107B6000F8F7B4F95346013782E76379009307F0D9
:107B70000707013F009BB342B0DDAA4615F8013B61
:107B8000202BFAD02046F8F78DF90546042F04D8AB
:107B9000DFE807F0030E0E141D005046F9F7CAF88F
:107BA000A8552C21504659F012FF0136451CE1E73B
:107BB0005046F9F7BFF825F81600F2E700230A222D
:107BC00000215046F9F716F845F82600E9E70123A9
:107BD000F5E7284656F0C2FEE37994F805A0A779A8
:107BE000DB0706460AD52046F8F75CF9037801461C
:107BF00023B13246284659F010FFE0B9DEB1B74252
:107C000019D32046F8F74EF93A46002159F0C8FE3C
:107C1000B2453FF663AF15493246284659F0FDFE9E
:107C200000283FF45BAF2046F8F73CF9324629467E
:107C300059F05EFE52E70E493A464046FCF7BEFC5C
:107C400023E73946404603B0BDE8F04F02E600BFE7
:107C5000114E08086054070809410808184507082C
:107C60005F4E0808D3410808544E08089A52080885
:107C7000244E080870B5044608460E4656F06EFEBF
:107C80003146054602462046F8F778FF68B9635D3D
:107C90001846F8F75DFF00B933B901352C4420468A
:107CA00001340378202BFAD070BD0020FCE708B522
:107CB00004460948FAF752FBFAF734FB074BD3F8AE
:107CC000C8020CF0EDFA05F079F8012C01D153F05F
:107CD00005FAF4F78BFF00BF6D4E080830B50020A1
:107CE00010B5044608460B46FEF782FA28B9094942
:107CF00003221846F8F742FF28B90748FAF7F4FBC1
:107D00000120FFF7D4FF20460449BDE81040FCF7EE
:107D100055BC00BF794E08087D4E08083C4708084E
:107D20002DE9F74F064601AA08462E49DFF8C48020
:107D3000DFF8C490DFF8ACA059F015FE4FF0000B4F
:107D400004465D46012714BBBBF1000F27D1264C2A
:107D5000002D43D025482946FAF720FB23780BB99C
:107D600004F032FC4CF0CEFC002384F84D30FAF7DE
:107D7000AFFA15B12846F7F76EFF9FB13046FDF711
:107D800043FD78B1FAF7EEF80020FFF790FFBBF162
:107D9000000F0AD02046F8F7CDFF85B2C5B93046AE
:107DA000FCF722FC03B0BDE8F08F41462046F8F70F
:107DB00009FF80B949462046F8F704FF0028EED0B5
:107DC0005F4601AA5146002059F0CDFD0446BAE7AE
:107DD0004FF0000BF5E74FF0010BF2E70448FAF71C
:107DE00083FBBFE7FF41080838A40020A84E08081D
:107DF000CB4E08089F4E0808874F080810B50C4660
:107E0000FDF702FD78B1084B01229A73FAF7AAF840
:107E10000648FAF769FB06492046F7F76BFD10B1F3
:107E20000020FFF744FF10BDB83E0020E14E0808D7
:107E3000103808082DE9F04F93B00E460290A04983
:107E400030461746FFF716FF0546002840F021810F
:107E50009C493046FFF70EFF0546002840F01B8185
:107E600099493046FFF706FF0546002840F0158186
:107E700096493046FFF7FEFE0546002840F00F8188
:107E800093493046FFF7F6FE002805460ABF012455
:107E9000082435467F4207F010078E4928463C43A8
:107EA000FFF7E8FE002800F0FC8044F020048A4B35
:107EB0001B780BB904F088FB4CF024FC14F0090F7C
:107EC00000F050838548FAF70FFB0020FCF728F8F4
:107ED00014F48073059340F0EE808148FAF704FBB8
:107EE0008048FAF7A7FA04F01803182B05D17E484A
:107EF000FAF7FAFA7D48FAF79DFA01230493FAF7A4
:107F000035FA7B497B48FAF749FA7B497B48FAF70F
:107F100045FA04F48473082B07D179490298FAF7DB
:107F20004CFA77490298FDF761F814F08003079343
:107F30000ED1744B93F88425002A734A03F28453BC
:107F400006BF012113460021704A2046FAF712FAB3
:107F50006F492046FBF75EFB6E492046FAF7E8FBC7
:107F60006D492046FAF7D9FA6C4BD3F800A06C4B58
:107F700014F010061D6840F0A0806A48FAF7B4FAC1
:107F80000396694B069399466AEA05034FF0000889
:107F9000099359F804BBBBF1000F21D0099B039A48
:107FA000012707FA08F73B400CBF012100212046BA
:107FB0000893FAF7A5FA65EA0A033B4214BF0121C8
:107FC00000215A4A03905B462046FAF755FC08996F
:107FD000564A00395B4618BF01212046FAF7CAF914
:107FE00008F10108B8F11D0FD3D165EA0A03DFF8E3
:107FF000549108934FF00008069B53F804BB069376
:10800000BBF1000F24D0012707FA08F73D420AD040
:108010006AEA05033B424A465B4614BF0121002140
:108020002046FAF729FC1AEA070F11D0089B039A99
:108030001F400CBF012100212046FAF761FA391ECA
:1080400003905B464A4618BF01212046FAF792F991
:1080500008F10108B8F11D0FCED12A4D344B354A35
:1080600005F2EC512046FAF79BFC079B002B6BD0E6
:10807000134B029822461821FCF71EFA049B002B92
:1080800000F0D4812C48FAF72FFA2C48FAF7D2F9ED
:10809000CCE10124FEE60224FCE60424FAE6812475
:1080A000F8E627492846FFF7E5FD00283FF4FFAE34
:1080B00044F48074FBE6002320E71A4B039360E747
:1080C000074F08080E4F0808164F08081C4F0808ED
:1080D000314A0808C24E080838A400202A4F080870
:1080E000324F08084A4F0808564F08087E4F0808C4
:1080F0009A3E08083E440808A23E08085C44080866
:10810000294C080830B500209A5208088E4F0808FC
:108110009B4F0808A54F08088B3B0808CC48002057
:1081200094450020E84E08089C4B0708AB4F080810
:10813000C24F080830A90020865008089C50080843
:10814000254F0808B74F0808DFF8C0A3DFF8C0B311
:108150009AF800209BF80030BC4F9A4214BF0121CE
:108160000021BB4A20460CBF4FF001094FF0000927
:10817000FAF7C6F99BF80030B64A07EB830380464E
:10818000D3F8103649462046FAF776FB9AF80030C5
:10819000B04A07EB83074946D7F81036AE4F204662
:1081A000FAF7E8F8D7ED007AAC4AF5EE407AF1EE4E
:1081B00010FA0CBF012100212046FAF7DBF8A8498C
:1081C00043463A462046FAF7D5FCA64B05F5117210
:1081D00005F244612046FAF7DBFE26B195F9D63167
:1081E000002B00F02981A048FAF77EF99F48FAF7A2
:1081F00021F900239E4A9F4F9F4D02F59A61204628
:10820000FAF76EFF9D4B9E4A019300923A682968E7
:108210002046FBF7A9F940F202229A4B0193009203
:10822000BA68A9682046FBF79FF9002E40F0068146
:108230009548FAF759F93246944F9548DFF8D4C279
:108240000125002117F8013B10F8018B03F1480EBE
:10825000EE440EF8208C1CF801EB0EF14809E944BD
:1082600009F8108C002D00F0EB80A3EB0E056B429B
:108270006B41013108291D46E4D183F0010100273B
:1082800020468DF83070FAF73BF9824A8DF840703D
:108290000EAB29462046FAF7EFFA7E4A0AAB29468A
:1082A0002046FAF767F87C4A7C4B02F52971204694
:1082B000FAF740FD7A4A7B4B02F529712046FAF71E
:1082C00081FD754A784B02F529712046FAF7C2FD07
:1082D000764B774A77492046FAF7E6FA764A774BA3
:1082E00002F5A9612046FAF7E1FB754A754B02F5E4
:1082F000A9612046FAF7DAFC734B744A74492046A8
:10830000FAF7CAFF734B744A74492046FAF764FFC0
:10831000002E40F097807248FAF7E6F8B346714DA8
:10832000DFF8F481A5F2C4770026394602222846F8
:1083300059F0BAFB00285A4614BF012100212046FB
:1083400095F800A00CBF4FF001094FF00009FAF7B3
:10835000D7F8BAF1020F834640F0E0807B784FF007
:10836000190A40F2EE221AFB032301933B785E4A7E
:1083700018F803300093494633462046FAF77CFA52
:108380006B7840F2EE221AFB032301932B78564AB6
:1083900018F803300093494633462046F9F7EAFFC0
:1083A0000136122E05F1020507F10207BDD10021A9
:1083B0004E4B02982246FCF77FF8210740F1C68019
:1083C0000025E9B2029822460135FFF7CBF9042DCA
:1083D000F7D1474F474D3B782B70059B33B9464843
:1083E000FAF782F845490298FFF78CF9FF232B70C2
:1083F0000026F1B2029822460136FFF707FA042E52
:10840000F7D17B786B70059B002B40F09C803C483B
:10841000FAF76AF839490298FFF7C8F93948FAF7C4
:1084200063F83948F9F79AFFFF236B70002013B007
:10843000BDE8F04FF7F70FBC0B4BDBE6124AFBE64B
:108440002B4616E7DFF898B069E700BF1845070824
:10845000F64E0808C94F0808843F0020D24F08088C
:10846000D046002001420808F04E0808E14F0808F5
:1084700004B700200C41002068490020EE4F080896
:10848000FFFF7F00F54F0808FC4E080870470020EA
:108490003CD00708A8410808A0B90020FA44080801
:1084A00020BA002001500808FC4F080807500808AF
:1084B0003CAA002034BD002064B800200B500808FE
:1084C00090B90020145008081C500808D8AA0020B1
:1084D000E8BE00202550080878410020D847002039
:1084E000004F080804C00020E34A0808074F0808A6
:1084F000B44700203406002029500808294C0808F9
:108500004C50080873500808894F08088C4900200F
:10851000703F0020D03E00204CD207083B781B4A19
:1085200018F803300093494633462046FAF7A4F979
:108530002B78164A18F803300093494633462046F4
:10854000F9F718FF2CE7FF236B7097E5104D0298A1
:1085500029782246FFF706F9697802982246FFF744
:1085600055F98BE5A20706D5094B029819782246E2
:10857000FFF7F8F85AE763077FF558AF044B029806
:1085800059782246FFF742F950E700BFF34A08083E
:10859000B4470020224BB0F5FA6F1A680346A8BF13
:1085A0004FF4FA63B3F57A7FB8BF4FF47A73D2040D
:1085B00016D540F2DC52904215D007EE903A40F2C8
:1085C000DB529042F8EE677A1FD8DFED166A9FED16
:1085D000167A9FED160A77EEE67AA7EE870A7047BD
:1085E000B0F57A7F02D89FED120A704707EE903AF5
:1085F000DFED106A9FED107A9FED100AF8EE677AB2
:1086000077EEE67AA7EE870A7047DFED0D6A9FEDF9
:108610000D7A9FED0D0A77EEE67AA7EE870A70478E
:10862000CC3E002000007A44D62000C000E0824406
:108630000000000000407A44661000400000404204
:1086400000A0BB44D620004000008344704700BF18
:1086500000207047704700BF00207047012070471E
:10866000704700BF704700BF704700BF704700BF32
:108670009FED010A704700BF000000000020704716
:10868000064B1B78834206D9054B00EB400003EBF9
:10869000C003586970470020704700BFD005001024
:1086A0000C050010034B00EB400003EBC003587CAB
:1086B000704700BF0C050010024B1878003818BF37
:1086C00001207047D005001003681B6903B11847EB
:1086D000704700BF2DE9F047DFF870A0BAF800300E
:1086E00004330F469DB201F10908012417F8011B5C
:1086F000AC464FF0000E04FA0EF2ACF104030A404F
:108700009BB219D100EB830901339BB29C45C9F898
:108710001420F7D10EF1010E0CF1040CBEF1080F7C
:108720001FFA8CFCE7D120354745ADB2DED10023DE
:10873000AAF80030BDE8F087868900EB8302013398
:108740009BB263455661F8D1E4E700BF50C60020F4
:108750002DE9F047DFF87CA0BAF802300B338846E9
:108760001FFA83FE01F106090024012618F801CB47
:1087700071460025A1F10B039BB23DB1092D20D01C
:108780006A1E06FA02F212EA0C0F1AD0878900EB71
:10879000830201339BB299425761F8D10B1D00EB64
:1087A000830301350C310A2D5C6089B2E2D10EF1F0
:1087B000780EC8451FFA8EFED8D1AAF80240BDE84F
:1087C000F0871A1D013300EB82029BB28B4254608A
:1087D000F7D1E3E750C600202DE9F0410E78057B84
:1087E000F6430446F6B200F1100300F1380243F8F4
:1087F000045F9342FBD12822002104F13C0059F090
:10880000CFF84FF000084FF0140C4FF0050E46FA69
:108810000EF303F00103002B0CBF0A271927434472
:108820001EF0010F0CEB07015FFA83F814BF284616
:10883000002089B2634604EB830201339BB28B4272
:108840005061F8D10EF1FF3E6744BEF1FF3F1FFAC1
:1088500087FCDCD118F0010F14BF19210A210CEBA1
:10886000010080B2634604EB830201339BB2834272
:108870005561F8D14A1E92B20CF1010313440CF178
:1088800002009BB205490433024492B204EB830315
:108890008A80002159602261BDE8F08150C6002025
:1088A00070B5094CA36873B10546002606E09968C7
:1088B0001A681E73A1609047A36823B15A68AA1A68
:1088C000002A1846F3DA70BD50C600200022FFF7D8
:1088D000B1BA0122FFF7AEBA2DE9F84F00261F4DBD
:1088E000DFF88090DFF880A007460C46B0462046AF
:1088F000FDF77EFCD5F800B048B921465846F8F798
:1089000061F920B968682146F8F75CF980B15846EA
:10891000F9F724FD696811B15046FAF7FFFEA9681E
:1089200011B14846FAF7FAFEF9F720FD4FF00108B9
:1089300001363A2E05F11005D9D12046FDF758FC35
:1089400048B9B8F1000F06D1224638460449BDE8BF
:10895000F84FFBF733BEBDE8F88F00BF3C75070842
:10896000EA500808E4500808DE500808F8B5354C0D
:108970002368002B53D00A2801D00D284DD1324D49
:108980002B7B0BB1F9F7F2FC304E2321304659F026
:108990001EF808B1801B2060236800226BB902B169
:1089A0002360F9F7AFFC2B7BEBB1BDE8F84028481A
:1089B000F9F7D4BC01220B46F0E7591E705C202861
:1089C000F8D08AB90022234C204FF2543B26013EB6
:1089D0000CD13146204B9C4211D2E3682068984765
:1089E0006B7B002BDDD1F8BD2360EBE721683846B7
:1089F000FFF740F901460028ECD11034E7E72B7B64
:108A000023B116491648FBF753FCCAE71548F9F796
:108A1000A5FC0E48F9F70EFDC3E7FF2BE3D8A0F144
:108A200020025E2ADFD80BB92028DCD05A1C226035
:108A3000064AD054044B1B7B002BD4D0BDE8F84031
:108A4000F9F710BF6CAD002050C600206CAC0020C0
:108A50000B3808083C750708DC780708FE50080842
:108A60001A5108082051080808B5254B1B68DB047B
:108A70000AD5B5EE400AF1EE10FA12D19FED210AA7
:108A800057F0FEFE80B208BDDFED1F7AB4EEE70AB4
:108A9000F1EE10FA1CDA9FED1D0A57F0F1FE80B2DC
:108AA00008BDDFED197AB4EEE70AF1EE10FAE5D46D
:108AB0009FED177AB4EEC70AF1EE10FA14D870EEF3
:108AC000677A9FED147A9FED140AA7EE870AE4E710
:108AD00070EE677A9FED117A9FED110AA7EE870A73
:108AE00057F0CEFE80B208BDDFED0E7A9FED0E7A14
:108AF00070EE677A9FED0D0AA7EE870ACDE700BFFB
:108B0000CC3E00200080BB440000404200007A447C
:108B100000E0824466BEFFBE0060BB4438DFFF3E1B
:108B200000407A440000834466BEFF3E00A0BB4480
:108B30002DE9F843CF4B1E6816F004072DED048B8A
:108B400040F01F819FEDCC8ACC4C16F0200605D05A
:108B500094F8DC6016F0020640F0AB8094F81D310A
:108B6000DFEDC78A94F81C2113F0010340F0B780B1
:108B7000002A40F09980D4ED487A9FEDC27ADFED6B
:108B8000C26A67EE877A94ED4A7AE8EE267A38EE82
:108B9000477AC4ED487A84ED497A66B1012284F8B7
:108BA0001E2194F83021D4F8E030C4F82C31012A89
:108BB00018BFC4F82431B54B93F80080B8F10D0FFD
:108BC0000BD1D4ED387A9FEDB27AB24B67EE877A4B
:108BD000FDEEE77A17EE902A9A809FEDA77AAE4DC8
:108BE000B0EE489A0023D4ED4F7AD4ED506A94ED5C
:108BF0004E8A37EE677AE6EE877A37EEC87AC4EDAA
:108C00004F7AA6EE878A85ED008A84ED4E8A0BB1F5
:108C100084ED498A94ED517AD4ED537ADFED9F5A71
:108C2000D4ED546A94ED520A84ED518A38EE477AB5
:108C3000B0EE676A97EE256AE6EE867A37EEC07A7E
:108C4000C4ED537AA6EE870A84ED520A84ED550AE4
:108C500057F016FE02B282EAE273A3EBE2739BB214
:108C6000092B40F2FC80002AACBF0A380A3005B25A
:108C7000B8F10D0FA4F8585100F0CF80B8F1240FCF
:108C800000F0E280B8F1380F05D1B0EE480A57F095
:108C9000F7FD804B9880BDEC048B002E18BF374643
:108CA00084F85A71BDE8F88384F81E3184F81C31C9
:108CB00061E7D4ED3B7AB4F8F030F8EEE77AC4ED32
:108CC000387A002B7DD1DFED6E8A94F81D3194F84F
:108CD0001C2113F001034FF001063FF449AF002AB5
:108CE00067D0D4ED4A9A694B94F81E9193F80080AE
:108CF00038EE699A002E49D0B9F1000F73D094ED87
:108D0000380AD4ED4B7A644D30EE670AB8F10D0F96
:108D100085ED000A07D1DFED627A20EE270A57F0D1
:108D2000AFFD5C4B988094F83031002B40F0998077
:108D300095ED007A002F3AD094F831319FED596AC1
:108D400077EE487A06EE903A77EEA97AF8EEE66A80
:108D5000F0EEE77A67EEA67A3B46F4EEC67AF1EEDD
:108D600010FAC4BF28EE866AC6EE278AF7EE007AAC
:108D700077EEE87A67EE897AE8EE877AB0EE677A7E
:108D800031E73E4C012794ED348ADEE6B8F10D0F51
:108D900037D0414DDFED388AB9F1000FC3D1002F34
:108DA00064D094F83031002B5ED1B0EE497A0123C3
:108DB00019E7D4ED489A0123C4ED4A9A84F81C318E
:108DC00091E707EE903ADFED356A9FED377AF8EEDE
:108DD000E77AC6EEA78AF4EEC78AF1EE10FA88BFEA
:108DE000F0EE478A71E7002F60D094ED380A70EEFC
:108DF000487A012377EEA97A84F81E31C4ED4B7AC4
:108E000081E7254DDFED267A95ED000A20EE270A51
:108E100057F036FD1F4B9880BCE7DFED207A9FEDC1
:108E2000200ADFF8708068EEA77A29EE000AFDEECE
:108E3000E77A17EE903AA8F8003057F021FDA8F82D
:108E40000650A8F8020026E7DFED157A94ED490AEE
:108E500020EE270A57F014FD0E4B58801BE7002523
:108E600006E7022B02D00FB1012B9ED095ED007AC0
:108E70000123B8E6A4AD00200000000050C6002089
:108E80009A99993ECDCC4C3FCDCC4C3E82240020CB
:108E90000AD7233C84240020AC4600200000C842AE
:108EA000CDCCCC3D00401C466666663FB8F10D0F48
:108EB000064DDBD1DFED067A95ED000A20EE270A9C
:108EC00057F0DEFC034B9880D0E700BFAC46002093
:108ED000CDCCCC3D842400204E4B1B681B0600D417
:108EE0007047F0B54C4C2DED048BD4F8683185B04B
:108EF00013B104F5AE7098470023CDE90033CDE9F6
:108F00000233D4F86C21454869469047009BD4F859
:108F10008421BDF90460A4F870619D1A03D105B0E5
:108F2000BDEC048BF0BD94F88C219DED039A94ED7B
:108F3000647A9DED020A002A394A67EE498A92ED69
:108F4000008AB4F88E21E0EE088AF7EE007A29EE66
:108F5000088AFFEE006A18BFF0EE667AA0EE078A74
:108F600068EEA78A1AB394ED667AD4ED697A94ED27
:108F7000676AD4ED6A6A78EEC78A38EE678AA6EE29
:108F8000287AE6EE887AD4ED658A94ED688A84EDD5
:108F9000667A37EE685A77EEC85AE6EE058AA6EE8C
:108FA000A58AC4ED697AC4ED658A84ED688A1D4A94
:108FB00084ED5D0A127884ED5E9A1C2AC4ED5F8A06
:108FC00084ED608AC4F88431A9D1DFED179A20EED0
:108FD000290A57F055FC29EE290A044657F050FC9F
:108FE00028EEA90A074657F04BFC00231A4666F301
:108FF0000F0364F31F4367F30F020C4C60F31F422F
:1090000028EE290AC4E9003257F03AFC6581208134
:1090100085E700BFA4AD002050C60020ACC70020EB
:10902000D00600208224002000007A4484240020FE
:1090300070B5234C2378012B00D070BD214B1B68E9
:10904000002BFAD0204D2B6828465B6898470028F3
:10905000F3D01E4B1E4E1A68338892889A421ED354
:109060001C49096800224968EA622A6803FB01F189
:109070002846D36898472B689B6813B128469847C1
:10908000D8B1154A3388526801333380002AD4D0CE
:109090001368928859690A420DD05A8370BD0E4BED
:1090A0000E495B68097800222270002BC5D0890721
:1090B0009A881B68F1D41A8370BD52F0E1F9E0E799
:1090C0005E39002094220020982200205839002088
:1090D0005C39002050390020E4220020E0220020EA
:1090E0002DE9F047A84C2DED048BA3682046984746
:1090F000002800F0BB80B4F90E30A17D06EE903A56
:10910000B4F9103007EE103AB4F9123007EE903A85
:10911000F8EEE66AB8EEC77AF8EEE77A0929C4ED08
:10912000126A84ED137AC4ED147A00F0A380974E8E
:1091300004F148002DF010FAB28DB36A002A40F015
:10914000A580934A934D1268520700F1E880B3F965
:109150000020D4ED147A94ED128AD4ED138A06EE31
:10916000102AB3F90220B3F9043006EE902A07EE74
:10917000103A894B894A93F80080B4F8443092F849
:10918000D273B8EEC66AF8EEE66AB8EEC77A38EE81
:10919000468A37EEC79A78EEE68A07EE903A338829
:1091A00084ED128AF8EEE79AC4ED138A84ED149ADE
:1091B000002B40F0FF80B8F1040F00F0E88195ED3E
:1091C000766AD5ED776A95ED787A85ED768A38EE10
:1091D000466A78EEE66A39EE477A26EE296A66EE46
:1091E000A96A27EE297A84ED156AC4ED166AC5EDE1
:1091F000778A84ED177A85ED789A94ED137AD4ED19
:10920000167A94ED126AD4ED156A27EE077A67EEA6
:10921000A77AA6EE067AB8F1040FE6EEA67A94EDE8
:10922000146AD4ED176AA6EE067AE6EEA67AB1EED7
:10923000C70AB1EEE77AD4ED006A26EE800A26EE80
:10924000878A84ED180A84ED198A0CD1DFED548ADF
:10925000544D20EE280A57F013FB28EE280AA88068
:1092600057F00EFB2881012384F86830BDEC048B95
:10927000BDE8F087454E04F1200104F148002DF0CF
:1092800003F9B28DB36A002A3FF45BAFB2F5C87F31
:1092900000F061813F4DD4ED127A95ED6B7AD4EDFB
:1092A000136A94ED146AB8EEC77A4FF0000C37EEEB
:1092B000277AD5ED6C7AC4F848C0F8EEE77ABDEEAF
:1092C000C77A77EEA67AD5ED6D6A85ED6B7AF8EE02
:1092D000E66AFDEEE77A76EE866A17EE901AC5ED3D
:1092E0006C7AFDEEE67A4FF0000E012AA3F800E05A
:1092F00017EE100AC4F84CC017EE907AA3F802E0FB
:10930000C5ED6D7AC4F850C0A3F804E000F0078200
:10931000013AB2851E4A126852077FF518AFB5F8B8
:10932000B821322A00F0C280002A40F0BB8195F8B3
:10933000D621002A3FF40BAFDFF870C0D5F8D0215A
:10934000B4F80CE0D5E972178CFB0298D217C2EB87
:109350002812A2EB0E029A808CFB01E2C917C1EB26
:10936000221119808CFB0721FA17C2EB21125A80B7
:109370000D4B00200122D881C3F80A2085F8D601C0
:10938000F8F74AFEB36AE2E68817001048170010A3
:10939000CC3E002050C60020822400205413001030
:1093A00000007A448424002020AA00201F85EB516D
:1093B0000AD7233C002F00F0C380D6ED027A96ED49
:1093C000037A96ED010A38EE678AE8EE077A95EDA2
:1093D000768AC6ED027A77EEC06AA6EE870A30EE8C
:1093E000488A86ED010A28EE298A84ED120A84ED66
:1093F000158A85ED760A002F00F08F80012F00F08E
:109400003B81D6ED057A96ED067A96ED040A95ED48
:10941000778A78EEE78A012FE8EE877A77EEC06ADE
:10942000C6ED057AA6EE870A30EE488A86ED040A74
:1094300028EE298A84ED130A84ED168A85ED770AD1
:1094400000F00781022F00F0228196ED087AD6ED18
:10945000096A96ED070A95ED788A79EE477A022F28
:10946000A6EEA77A77EE407A86ED087AA6EEA70AEE
:1094700030EE488A86ED070A28EE298A84ED140A20
:1094800084ED178A85ED780A7FF4B7AEB8F1040F42
:109490007FF4B3AE57F0F4F91FED3B0ABC4D28EE54
:1094A000000A688057F0ECF9E880A6E6D4ED127A5D
:1094B000D4ED136AB7491A68C9689FEDB77AC5F841
:1094C000BC21FDEEE77AFDEEE66A0022C5F8C41184
:1094D0009988C5ED727A84ED127AF0EE477A1A8097
:1094E000C5ED736A84ED137AA5F8C0115A8094ED26
:1094F000147AB5F8B87177EE877A0022FDEEE77A34
:109500002265012F4FF00002C5ED747A9A8000F0B9
:109510002B81013FA5F8B87109E7B8F1040F7FF47A
:1095200070AF57F0ADF99FED9D0ADFF8649228EE19
:10953000000AA9F8020057F0A3F9A9F8060060E7AD
:10954000B8F1040F7FF439AFB0EE480A57F098F93C
:109550008F4B188031E7D4ED126A94ED137AD4ED75
:10956000147A8F4DFDEEE66ABDEEC77AFDEEE77A1E
:1095700000200021A064C5ED6B6A198085ED6C7A2E
:10958000E064C5ED6D7A598020659980C0E697B397
:10959000D5ED767A85ED768A38EE678A012F28EE4A
:1095A000298A84ED158A00F0A080D5ED777AC5ED83
:1095B000778A78EEE77A022F67EEA97AC4ED167AF9
:1095C0003CD1B0EE490A57F05BF9D5ED787A9FEDC2
:1095D000730A6F4E85ED789A79EE677A00B267EE7E
:1095E000A97A308027EE800AC4ED177A708057F090
:1095F00047F9F08001E6B0EE480A57F041F9D5EDA1
:10960000767A9FED660A624E85ED768A78EE677A05
:1096100000B267EEA97A308027EE800AC4ED157A91
:10962000708057F02DF9D5ED777AF08078EEE77AF3
:10963000C5ED778A67EEA97AC4ED167AD5ED787A0A
:1096400085ED789A79EE677A67EEA97AC4ED177A94
:10965000D3E5B8F1040F7FF4F8AE57F011F99FEDA0
:109660004F0ADFF82C9128EE000AA9F8020057F003
:1096700007F9A9F80600E8E6B8F1040F7FF4C1AED7
:10968000B0EE680A57F0FCF8414B1880B9E6B8F123
:10969000040F7FF4DAAEB0EE490A57F0F1F83C4B14
:1096A0001880D2E6D5ED727A94ED127AD4ED136A71
:1096B000F8EEE77A002177EE877A0022FDEEE77A6E
:1096C000A164C5ED727AD5ED737A1A80B8EEE77AA7
:1096D000D5ED747AE16437EE267AF8EEE77ABDEEDE
:1096E000C77A5A8085ED737A01E7B0EE680A57F0C1
:1096F000C7F8D5ED777A9FED290A254EC5ED778A13
:1097000078EEE77A00B267EEA97A308027EE800A19
:10971000C4ED167A708057F0B3F8F0808EE7DFF86A
:1097200084C0B4F80C80C8378CFB07A9FF17C7EBBF
:10973000E917C830A7EB08079F808CFB0087C0178C
:10974000C0EBE710C83118808CFB010CC917C1EBC6
:10975000EC1159800F4BC3F80A20A3F80EE0F8F77C
:109760005BFCB28DB36AD3E50B2085F8D42185F874
:10977000D5710AF087FEB36AD5F8BC111960054AA5
:10978000B5F8C0119980D5F8C411D160C1E600BF09
:109790008424002020AA0020000000000AD7233CD7
:1097A00050C600201F85EB514B4B1B68190700D496
:1097B00070472DE9F0472DED108BDFF83C81474CC9
:1097C00098F80010D4F8F431D4F8E421582982B084
:1097D0000546C4F8E401187800F0D081012800F0B3
:1097E0008F823F49D4F8EC31A1F58070984798F802
:1097F0000070582F08BF3B4B80F00100C0B208BF7B
:109800005881002840F09D82B4F9E83294F8B412EF
:1098100007EE903AB4F9EA32F8EEE77A07EE103A3A
:10982000B4F9EC32C4EDBD7A07EE903AB8EEC77ADF
:10983000F8EEE77A0123092984EDBE7AC4EDBF7AF8
:1098400084F8F03241D028482CF086FE94F800933A
:10985000B9F1000F54D1DFF8A4A0244EB6F90830B6
:1098600094EDBD9A94EDBE8AD4EDBF8A07EE903A8E
:10987000B6F90A30F8EEE77A07EE103AB6F90C308E
:1098800039EE679A07EE903AB8EEC77AF8EEE77AC3
:1098900038EE478A78EEE78A572F84EDBD9A84ED3B
:1098A000BE8AC4EDBF8A00F07181582F00F0088293
:1098B0000F4B5B6801228AF80020002B40F04782A2
:1098C00002B0BDEC108BBDE8F0870A4901F13C0005
:1098D0002CF0DAFDBAE700BFA4AD002050C600208E
:1098E00038C900208424002044C90020F8A90020A1
:1098F000D006002008C9002082240020BC180010D7
:10990000D4F8043394F801235B1B002B40F38581CA
:10991000DFF8A0A3DAED017ADAED026A9AED037AB4
:10992000002A00F0FA81DB4EDB4B1B683BB1DB4ABF
:10993000998812781B68D2074CBF1983598394ED1C
:10994000BE1A94EDBD4AD4EDBF9A94EDCB0AD4ED86
:10995000DB7AD4EDC32AD4EDD0DA94EDCC3A94ED91
:10996000D5EA94EDD12AD4EDDCEAD4EDCD4AD4ED9C
:10997000D6CA94EDD2CAD4EDDA3A94EDDDFA94ED7C
:10998000CEBAD4EDDEFA94EDC88AD4EDC78A21EEC2
:10999000017AB0EE62AAA4EE047A64EE2D6AA9EE12
:1099A000A97A21EE0E6A67EE005AE7EE036A25EE09
:1099B000A75AA4EE026AA5EE85AA66EEAE1AC7EE15
:1099C0008A5AF0EE4A0AC4EDDB5AC6EE8A5AA7EE6E
:1099D000246AE6EEA10AF0EE436A86EE209AE5EEEE
:1099E000C56A61EE2C7AF0EE455AE4EE0C7AC4EDCD
:1099F000CC6A66EEA16AE3EE215A69EEA33AE0EE84
:109A0000056A26EE0F5A73EEA77AB0EE600AA6EE4C
:109A1000050AB0EE646AE7EE0B7AA5EEC96AF0EECD
:109A200040AAE6EE056A84EDCD6A27EEAF6AE4EE61
:109A3000855AE7EE86AAF0EE624AE3EE864AB0EE79
:109A4000613AF7EE003AA2EE053AA9EE612A83EEFA
:109A5000AA9A62EEAAAAC7EE80BA80EE2ADA20EEAF
:109A6000220AD4EDC97A84EDD12AC0EE80AA62EE32
:109A7000A00A2AEE8F0A61EE277A84EDDD0A8AEECB
